:1000000000200020F949030889E602089DE602085D
:10001000B1E60208C5E60208D9E6020800000000C1
:10002000000000000000000000000000EDE60208F3
:1000300001E7020800000000C95A000843E900086F
:100040000D4D0308114D0308154D0308A7EC0208D8
:100050001D4D03080FEE020859E90208E9EA0208FB
:1000600075EB0208314D0308354D0308394D03087F
:100070003D4D0308414D0308454D0308494D030814
:100080004D4D0308514D0308554D0308594D0308C4
:100090005D4D0308614D0308654D0308694D030874
:1000A0006D4D0308714D0308754D0308794D030824
:1000B0007D4D0308814D0308854D0308894D0308D4
:1000C0008D4D0308914D0308954D030819E702086B
:1000D0009D4D0308A14D0308A54D0308A94D030834
:1000E00013EC020873ED0208B54D0308B94D03087F
:1000F000BD4D0308C14D0308C54D0308C94D030894
:10010000CD4D0308D14D0308D54D0308D94D030843
:10011000DD4D0308E14D0308E54D0308E94D0308F3
:10012000ED4D0308F14D0308F54D0308F94D0308A3
:10013000FD4D0308014E0308054E0308094E030850
:100140000D4E0308114E0308154E0308194E0308FF
:100150001D4E0308214E0308254E0308294E0308AF
:100160002D4E0308314E0308354E0308394E03085F
:100170003D4E0308414E0308454E0308494E03080F
:100180004D4E0308514E030838B50020ADF800006D
:10019000044601F0AEFF05464FF48051204602F0C0
:1001A0000CFA0A21284602F091F900E0641C062CA2
:1001B00012D2DFF8080D215C8DF800102018007AAB
:1001C0008DF80100022300AA7221072002F089F8AD
:1001D0000028EBD1002032BD012032BD2DE9FC41C9
:1001E0000746884602F04CFB04460020ADF80400A8
:1001F000DFF8CC5C288C0646B8F1000F02D03843FB
:10020000288401E0B8432884012000900DF1060302
:10021000AB227221062002F0BEF8002801D1002096
:10022000C5E1288C0E2800F2A681DFE810F00F004F
:10023000A4011C00A4013F00A4013F00A401B700D9
:10024000A401B700A401B700A401B70080208DF875
:10025000040000208DF805009DF8060000F0FD0068
:100260008DF8060087E116F00C0F01D001206875AB
:1002700081208DF8040001AEEE207070022301AAE7
:100280007221092002F02DF8002801D100208EE112
:100290007078E87080208DF80400032070709DF85D
:1002A000060000F0FD008DF8060064E1304600070E
:1002B00001D4022E01D1012068759D208DF8040023
:1002C00001AE0C207070022301AA7221092002F0F5
:1002D00008F8002801D1002069E19E208DF8040073
:1002E0000C207070022301AA7221092001F0F9FF8D
:1002F000002801D100205AE181208DF80400FD2062
:100300007070022301AA7221092001F0EAFF00287F
:1003100001D100204BE17078E8708E208DF8040048
:10032000287A002812D00C218F2002F076FB0421BD
:100330008F2002F048FB3021902002F06EFB30212C
:10034000902002F040FB4520707011E00C218F20BE
:1003500002F063FB08218F2002F035FB3021902052
:1003600002F05BFB1021902002F02DFB82207070C8
:10037000022301AA7221092001F0B3FF002801D154
:10038000002014E180208DF80400272070709DF873
:10039000060000F0FD008DF80600ECE016F00807FE
:1003A00001AE4FD102F052FC01206875A4208DF8F7
:1003B000040000207070DFF88C0D00210170022312
:1003C00001AA7221092001F08CFF002801D1002030
:1003D000EDE0A5208DF8040000207070DFF8680DB6
:1003E00000210170022301AA7221092001F079FF86
:1003F000002801D10020DAE0A7208DF804000020B9
:100400007070DFF8480D00210170022301AA7221EB
:10041000092001F066FF002801D10020C7E0A920D3
:100420008DF8040000207070DFF8980D0021017035
:10043000022301AA7221092001F053FF002801D1F3
:100440000020B4E081208DF80400FE2070700223AB
:1004500001AA7221092001F044FF002801D10020E7
:10046000A5E07078E8708E208DF80400287A0028C6
:1004700012D00C218F2002F0D0FA04218F2002F03C
:10048000A2FA3021902002F0C8FA3021902002F028
:100490009AFA4F20707011E00C218F2002F0BDFA03
:1004A00008218F2002F08FFA3021902002F0B5FA57
:1004B0002121902002F087FA84207070022301AA83
:1004C0007221092001F00DFF002801D100206EE00B
:1004D000002F20D1B4F88A00B4F88C10401AE883B9
:1004E000B4F88A108900A98389B2FF2901DBFE21B3
:1004F000A98380B28100652902DB6420E88301E0E2
:100500008000E883A98BE88B0A1AEA8392B20FF283
:10051000A40001F070FEA6208DF80400287A0028BF
:100520000AD06021A32002F078FA4121A32002F032
:100530004AFA5720707009E06021A32002F06DFA9A
:100540004121A32002F03FFA8B207070022301AA00
:100550007221092001F0C5FE002801D1002026E00B
:1005600080208DF80400672070709DF8060040F030
:1005700002008DF80600022301AA7221092001F071
:10058000B0FE002801D1002011E0AB208DF804005E
:100590009DF806008DF80500022301AA72210920AA
:1005A00001F09FFE002801D1002000E00120BDE8FD
:1005B000F6810000233E6755703D25642C674C6F23
:1005C0003D25640010B534220021DFF8A00C02F0B4
:1005D000CFFEDFF8EC480120A07102F0D3FE02F05C
:1005E00057FA01202073DFF8D00D0021017010BDF3
:1005F00010B582B00FF25C0001F0FDFD0020ADF8F7
:10060000000080208DF8000000AC03206070022301
:1006100000AA7221062001F064FE002818D0DFF83D
:10062000A008817A00290DD08C218DF800100021BE
:1006300061708170022300AA7221062001F051FE30
:10064000002805D0FFF7BEFF01210020FFF7C6FDFF
:1006500013BD0000233E484C5300000010B582B08B
:100660000FF2400001F0C7FD0020ADF80000044685
:1006700000E0641C052C12D2DFF8700D215C8DF8AF
:1006800000102018007A8DF80100022300AA7221C0
:10069000072001F026FE0028EBD1002016BD012026
:1006A00016BD0000233E50525000000030B583B00C
:1006B0000FF2880001F09FFD0020ADF804008DF8D6
:1006C0000600DFF8FC47607180208DF8040001AD62
:1006D00003206870022301AA7221072001F001FEA5
:1006E000002801D100203EBD8C208DF804000020A0
:1006F0006870A070022301AA7221072001F0F1FDA9
:10070000002801D100203EBD012060720146042076
:10071000FFF764FD002801D100203EBD01200090BC
:100720000DF10603E5227221072001F034FE0028B6
:1007300001D100203EBD01203EBD0000233E5052AD
:100740004F00000000B583B00FF2640001F053FDCC
:100750000020ADF806008DF8040080208DF806001A
:1007600003208DF8070002230DF1060272210720F5
:1007700001F0B7FD002801D100200EBDDFF84007D1
:10078000002141720420FFF729FD002801D100203B
:100790000EBD0120009001ABE5227221072001F07F
:1007A000FAFD002801D100200EBD01200EBD000081
:1007B000233E5052430000000120704730B583B003
:1007C00004460020ADF80400DFF8F456A87B0028AA
:1007D0002CD1A87A002802D0287C207031E001209A
:1007E00000900DF1050393227221072001F0D3FD43
:1007F00000280DD09DF80500800722D5012000902B
:1008000001AB9C227221072001F0C5FD002801D117
:1008100000203EBD9DF80400697951FA80F080B255
:10082000400820709DF8040068710AE0012808D192
:10083000DFF8380A41696A798918491021704069DE
:10084000687101203EBD2DE9F04391B0044602F0ED
:1008500017F8054601F04DFC06460020ADF80800EB
:10086000ADF80C008DF80A00012000900DF10A038C
:1008700093227221072001F08EFD002801D1002073
:1008800025E20220009003AB94227221072001F0A0
:1008900082FD002801D1002019E2DFF824769DF8BE
:1008A0000D009DF80C1041EA0020DFF8181D4843A8
:1008B000F978C1F580713A79DFF80C3DD25C12FB12
:1008C00001F140F24232514390FBF1F0797B002973
:1008D00002D0B97A002901D1B86208E0B86AF97D7E
:1008E0004A1CFA75062902DB00217973F975397AF9
:1008F00000290CD141F6593188422DDB0121397292
:10090000F86200203876FFF773FE0120DFE1F96A14
:10091000411A44F62162914215DA40F6B831884214
:1009200018DA9DF80A20920614D53A7E531C3B76BD
:10093000C92A04DABA7A002A0ED188420CDA88422F
:1009400001DA00213972F86200203876FFF750FE94
:100950000120BCE1002038769DF80A00800640F1B5
:10096000B5810020B873012000900DF10A03932295
:100970007221072001F00FFD002801D10020A6E11F
:100980009DF80A0080071BD50120009003AB9C2234
:100990007221072001F0FFFC002801D1002096E120
:1009A0009DF80C00797951FA80F080B240086070AF
:1009B0009DF80C00F8739DF80C007871607838741D
:1009C000387B002802D00020387371E1DFF81C8DDD
:1009D000607888F80000B87900280AD002F062F840
:1009E000002806D1B87A002803D0607802F06CF8AD
:1009F0007AE0787A002839D0B87AB978084335D1C6
:100A0000002030758C208DF808000DF10809202099
:100A100089F80100B870022302AA7221072001F0B0
:100A200060FC002801D1002051E189208DF80800E8
:100A3000002089F80100022302AA7221072001F098
:100A400050FC002801D1002041E18B208DF80800E6
:100A5000B5F88A0089F80100022302AA7221072052
:100A600001F03FFC002801D1002030E1B87A0028D5
:100A70000ED105F18A004288B5F88A100FF2542091
:100A800001F0B9FB61780FF25C2001F0B4FB2BE0C0
:100A9000414684B06846182203F05EF80FBC02F0AD
:100AA00082FC04A802F0E5FCDFF8C49C484604A9D7
:100AB000342203F051F899F81C00002807D03422A2
:100AC0004946DFF8A80703F072F80120787009F1B1
:100AD0001C00417D88F81410817D88F81510007D78
:100AE000002801D0FFF76EFD787A002800F0E08042
:100AF000B87A002840F0DC806078B5F88A10884227
:100B000031D3307D00282ED10120F871207020785B
:100B1000307589208DF808000DF1080905F18A006B
:100B2000408889F80100022302AA7221072001F0FF
:100B3000D8FB002801D10020C9E08B208DF80800E7
:100B4000FF2089F80100022302AA7221072001F088
:100B5000C8FB002801D10020B9E061780FF29010A5
:100B600001F049FBA4E005F28A00418862789142D5
:100B700031D3317D01292ED10120F8710020207060
:100B80002078307589208DF808000DF108090020C3
:100B900089F80100022302AA7221072001F0A1FBBB
:100BA000002801D1002092E08B208DF80800B5F8D4
:100BB0008A0089F80100022302AA7221072001F0AD
:100BC00090FB002801D1002081E061780FF228100D
:100BD00001F011FB6CE0B5F88A106278914235D3D0
:100BE000317D002932D1797C01292FD10120F87182
:100BF00000202070207830750020787489208DF8CE
:100C000008000DF10809002089F80100022302AA5A
:100C10007221072001F065FB002801D1002056E079
:100C20008B208DF80800B5F88A0089F801000223AE
:100C300002AA7221072001F054FB002801D10020F4
:100C400045E00FF2BC0001F0D6FA31E0617842884D
:100C500091422DD3317D01292AD1797C012927D1D7
:100C60000021797489218DF808100DF10809408858
:100C700089F80100022302AA7221072001F031FB4A
:100C8000002801D1002022E08B208DF80800FF20F1
:100C900089F80100022302AA7221072001F021FB3A
:100CA000002801D1002012E00FF25C0001F0A3FA4D
:100CB0000120009003ABE5227221072001F06BFBBD
:100CC000002801D1002002E0012000E0002011B046
:100CD000BDE8F083233E55703D25642C4C6F3D25C7
:100CE00064000000233E505241572025640000005C
:100CF000233E503120256400233E503220256400DD
:100D0000233E526554483100233E52655448320018
:100D10002DE9F84304460D46694EB07C002805D005
:100D200000F01EFF0020F0743075C5E001F0A8FD52
:100D3000804600273846ADF800002078072823D1E8
:100D40006078FF2820D12946601CFFF737FD6078C6
:100D5000B8F88A10884208D3012020706278217880
:100D60000FF2601001F047FA0CE0B8F88C006178DF
:100D7000884207D338462070627821780FF24410F9
:100D800001F039FA012097E00020F074307529460F
:100D90002046FFF758FD00280DD0707A00280AD0B1
:100DA000F079002807D00FF2301001F024FA00206B
:100DB000F07101203075B07A002877D0DFF8648DAB
:100DC000D8F8189009F10C00417DC068D9F80C20C2
:100DD000801800F04DFA002868D0DFF8DC050078B4
:100DE000411E8941C90FF1747078002801D000209C
:100DF0007070707A002857D0D9F80C0040780DF147
:100E0000000989F80100B18B814218D201F071F913
:100E1000007D002813D1707E401C7076C0B202287D
:100E20002DD100207076012701F063F93946017554
:100E300099F801100FF2A80001F0DDF91FE099F810
:100E40000100F18B884218D201F053F9007D01288E
:100E500013D1707E401C7076C0B202280FD10020E2
:100E60007076012701F045F90021017599F801100C
:100E70000FF2780001F0BFF901E000207076002F3A
:100E800012D0D8F81C8001F034F9007D8DF80000F4
:100E900008F10C00427D00A9C068D8F80C30C018D9
:100EA00002F085FE012030750020307003F004FF51
:100EB00000283FF469AF307DBDE8F28384870020CD
:100EC0009C860020233E536C65657020414443207E
:100ED0002564202564000000233E5055500000008A
:100EE000233E67757031202564000000233E67753E
:100EF0007032202564000000F8B507460020ADF8E8
:100F0000000001F0BDFC0546DFF8304D01206074A3
:100F10003878A5F88A0005F28A0678787080B5F8E6
:100F20008A00002802D07088002808D10FF29400AF
:100F300001F061F97820A5F88A00002070808920EE
:100F40008DF8000000AF70887870022300AA72212B
:100F5000072001F0C6F900280DD08B208DF8000085
:100F6000B5F88A007870022300AA7221072001F0E8
:100F7000B8F9002801D10020F2BD7288B5F88A10B6
:100F80000FF2480001F037F9B5F88A007188401A6D
:100F9000E083B5F88A108900A18389B2FF2901DBBB
:100FA000FE21A18380B28100652902DB6420E083F9
:100FB00001E08000E083A08BE18B401AE0830120F8
:100FC000F2BD0000233E5054483D3000233E5448BB
:100FD00053455420256420256400000080B50FF29D
:100FE0001801072004F0D0FA0FF230010A20BDE802
:100FF000044004F0C9BA00005D060008AD06000810
:1010000045070008B907000800000000110D00089E
:10101000F90E000800000000000000005D06000856
:10102000AD06000845070008B907000800000000E9
:10103000BD070008F90E00080000000000000000D5
:1010400010B582B00FF2540001F0D5F80020ADF8D1
:101050000000FFF799F8002803D10FF2480001F0D3
:10106000CAF8002400E0641C0B2C12D2DFF8840DB7
:101070002118097B8DF80010205C8DF801000223F7
:1010800000AA7221062001F02CF90028EBD10020E3
:1010900016BD03F045F8012016BD0000233E47456C
:1010A00050000000233E47504641494C00000000DC
:1010B00038B50FF29C0001F09EF80020ADF800005A
:1010C00080208DF8000000AC03206070022300AA8D
:1010D0007221062001F005F9002801D1002032BD5F
:1010E0008C208DF8000000206070DFF8505BA87045
:1010F000022300AA7221062001F0F3F8002801D192
:10110000002032BDA3208DF80000DFF8E80CC07885
:101110006070022300AA7221062001F0E2F8002884
:1011200001D1002032BD0120A872FFF74BFA012146
:101130000820FFF753F8002801D1002032BD01201C
:1011400032BD0000C74F0120C84F0120C94F012008
:10115000233E47454F00000010B582B00FF26800F3
:1011600001F049F80020ADF8000080208DF8000063
:1011700000AC03206070022300AA7221062001F057
:10118000B0F8002801D1002016BDDFF86C0C00215A
:1011900081720820FFF722F8002801D1002016BD37
:1011A0009F208DF8000000206070022300AA7221A9
:1011B000062001F096F8002801D1002016BD01207C
:1011C00016BD0000CA4F0120233E474543000000E2
:1011D0000120704730B58DB0DFF8605AA87900283B
:1011E00014D001F05FFC002810D0DFF80045201D6E
:1011F0000FC801F053FD01F05EFC002832D0002042
:10120000A871012060752075A0752BE0A8790028D1
:1012100028D1DFF8D844214684B06846182202F06D
:101220009BFC0FBC02F0F2F800A802F022F9DFF8F4
:101230004055284600A9342202F08EFC05F11C001E
:10124000417D2175817D6175007D002801D0FFF70A
:10125000B9F9287F002805D034222946DFF81C0D73
:1012600002F0A5FC01200DB030BD0000844C01202F
:1012700010B584B0044602A8002101600846ADF80C
:1012800004000120009001AB93227221062001F09E
:1012900082F8002800F088809DF8040010F0040017
:1012A00004D1DFF89819497800297DD0002806D0AC
:1012B000DFF888094178002901D1012181730120DB
:1012C00000900DF10503AE227221062001F063F8B3
:1012D000002869D09DF80500002817D00420009050
:1012E00002ABFC227221062001F055F800285BD0E9
:1012F000DFF8F8039DF80810416002A94A7882607F
:101300008A78C260C9780161FFF764FFDFF86C1C5E
:101310000A78DFF828094378002B227007D00022D2
:101320006270A270E27022716271A2710BE04A6970
:1013300062708A69A2704A68E2708A682271CA681B
:1013400062710A69A2710A6AE2714A6A22728A6A41
:101350006272CA6AA2724A7FE272DFF8242C1278A3
:101360002273DFF8202C12786273DFF81C2C1278BD
:10137000A273DFF8182C1278E273DFF8142C1278BD
:101380002274DFF8102C12786274DFF80C2C1278BB
:10139000A274C27BE274002202700878042801D192
:1013A00010460870012000E0002004B010BDDFF8F6
:1013B000480AC07C70470000CC49012080B5052850
:1013C00002D1084600F002F8012002BD80B5017884
:1013D00041F04103DFF8C41BCB70027801780FF6AF
:1013E000DC3000F008FF012002BD000094870020DF
:1013F00070B584B004460020019002A8002101606D
:101400000E460FF6CC3000F0F6FE01210820FEF764
:10141000E5FEA0208DF8040001AD3046687002237F
:1014200001AA7221062000F05CFF002801D130469D
:10143000C5E0A1208DF80400FF206870022301AAF6
:101440007221062000F04DFF002801D13046B6E0A1
:10145000AB208DF8040001206870022301AA7221DC
:10146000062000F03EFF002801D13046A7E0012011
:1014700000900DF1060380227221062000F08BFF00
:10148000002801D130469AE080208DF804009DF8B4
:10149000060040F045006870022301AA7221062070
:1014A00000F01FFF002801D1304688E0A3208DF80E
:1014B0000400DFF84009C0786870022301AA722195
:1014C000062000F00EFF002801D1304677E0012011
:1014D00000900DF10703AF227221062000F05BFFA0
:1014E000002801D100206AE09DF80700C0070BD555
:1014F0000420009002ABFC227221062000F04BFF7A
:1015000000280CD100205AE03046461CB0F57A7F06
:10151000DDDB0FF6C42000F06EFE00204FE09DF8EA
:101520000800207002A8417861708178A170C078AD
:10153000E070012000900DF1060380227221062048
:1015400000F029FF002801D1002038E080208DF82C
:101550000400DFF8A408417A002905D09DF80600B0
:1015600000F0BF0068700CE09DF8061001F0BB01B0
:101570006970C07A002804D19DF8060000F0BA0016
:101580006870022301AA7221062000F0AAFE00283A
:1015900001D1002013E0AB208DF80400002068701A
:1015A000022301AA7221062000F09BFE002801D12F
:1015B000002004E000210820FEF710FE012004B006
:1015C00070BD0000D8D00100742000080FF6A821DB
:1015D000062003F0D9BF1CB50FF6082000F00BFE63
:1015E00000208DF80400ADF80600044600E0641CFD
:1015F000052C13DADFF8A809215C8DF806102018F5
:10160000007A8DF8070002230DF1060272210920ED
:1016100000F067FE0028EAD1002016BD01200090EE
:1016200001ABD6227221062000F0B5FE002801D1C0
:10163000002016BD9DF804100FF6B01000F0DBFD81
:10164000DFF8B4079DF80410C9098176012016BDA2
:1016500030B583B0DFF8A047A07E002804D00FF695
:101660009C1000F0C8FD03E00FF6981000F0C3FDD9
:101670000020ADF8040080208DF8040001AD0320A7
:101680006870022301AA7221092000F02AFE0028B6
:1016900001D100203EBD8F208DF804000B20687022
:1016A000022301AA7221092000F01BFE002801D1AB
:1016B00000203EBD032020710120A075E07201468C
:1016C0000220FEF78BFD002801D100203EBD012045
:1016D00000900DF10603E6227221092000F05BFE66
:1016E000002801D100203EBD01203EBD344F012025
:1016F00000B583B00FF6141000F07DFD0020ADF8AA
:10170000060080208DF8060003208DF807000223D4
:101710000DF106027221092000F0E3FD002801D13D
:1017200000200EBD0120009001AB8F227221092004
:1017300000F031FE002801D100200EBDDFF8B80610
:101740000021C1720220FEF749FD002801D10020CE
:101750000EBD0120009001ABE6227221092000F0AD
:101760001AFE002801D100200EBD01200EBD000090
:10177000E84B0120012070472DE9F04184B0044678
:101780000020ADF804000290DFF89803456A0020BD
:1017900085F85E00DFF86066B07D012803D0707DBB
:1017A000002840F090800220009001AB942272212A
:1017B000092000F0F0FD00282DD09DF80400A07154
:1017C00001AF7878E0710220009001AB962272217F
:1017D000092000F0E0FD00281DD09DF804002070D5
:1017E000787860700220009001AB98227221092065
:1017F00000F0D1FD00280ED09DF80400A07078788C
:10180000E0700220009001AB9A227221092000F0C2
:10181000C2FD002801D1002097E09DF8040020714E
:1018200078786071F0782072307960726078217811
:1018300041EA0020E178A27842EA01216279237925
:1018400043EA0222E379A77947EA032302AF00972C
:1018500000F0CCF800281BD1B07D012834D1002045
:10186000B075DFF840075B210170002141708521D0
:1018700081700021C170AE21017100214171702180
:1018800081710121C171EE210172002141721BE0C1
:101890000020B075DFF80C07217801706178417085
:1018A000A1788170E178C17021790171617941710C
:1018B000A1798171E179C171217A0172617A4172F4
:1018C0000298706238E037D0DFF8D80601782170CE
:1018D000417861708178A170C178E17001792171DE
:1018E000417961718179A171C179E171017A2172C6
:1018F000407A6072002070756078217841EA00209B
:10190000E178A27842EA01216279237943EA02224E
:10191000E379A77947EA0323F77894F808C086F8B3
:1019200003C096F80480647A347102AC009400F02D
:101930005DF8F77086F80480029840F6845188427A
:1019400002D1012085F85E00012004B0BDE8F081DD
:101950001CB504460020ADF806008DF804000120F7
:10196000009001AB8F227221092000F014FD0028A5
:1019700001D1002016BD9DF8040000F0FC008DF898
:101980000400012C0AD0042C04D0102C1FD0402CB1
:1019900022D026E040F001008DF804008F208DF861
:1019A00006009DF804008DF80700DFF84C449DF810
:1019B000040000F00300207102230DF106027221E1
:1019C000092000F08EFC00280DD1002016BD40F04B
:1019D00002008DF80400E1E740F003008DF80400F8
:1019E000DCE7002016BD0120607316BD2DE9F04133
:1019F0009C4614460D460646A8192018A0EB0C007C
:101A0000401C47103FB2002F00D50027DFF8E81335
:101A100008790FF26062805CC978C1F5807110FBB3
:101A200001F240F6DC2E0EFB02F88902B1F5803F90
:101A300001D34FF6FF71C9000A22B1FBF2F1102861
:101A40002DD18B422BD30120FFF782FF002840D1FC
:101A5000E91B0698B74206DA0268F31B4FF4B47626
:101A600006FB03220260AF4205DA02684FF47A7384
:101A700003FB01210160A74201DA016801600168EE
:101A8000002901D50021016040F2A641B8FBF1F127
:101A90000268B2FBF1F101600120BDE8F08110287D
:101AA00008D1BCF1640F05DA4020FFF751FF002890
:101AB0000FD1CDE7402802D164398B4204D20128EE
:101AC000C6D1BCF1640FC3DA1020FFF741FF002834
:101AD000BED00020E1E70FF2C451092003F054BD4D
:101AE000C54988740120704710B5DFF8BC44202038
:101AF0002070002060700A20A0700020E0700A2092
:101B00002071002060713220A0710020E072072255
:101B10002146DFF8980402F04AF8002060720120A4
:101B200010BD00000860002000B583B000A80021AF
:101B30000A4606C00722DFF870140DF1010002F01A
:101B400036F8A0208DF80000082300AA7221072093
:101B500000F0C7FB002801D100200EBD01200EBD02
:101B600000B583B000208DF80400DFF83C04417B11
:101B7000012903D100F0B0F901200EBD418AFF29EF
:101B80000CD000290DD0C27A521CC272491E41826B
:101B9000417AD2B2914201D20021C17200F015F80F
:101BA00005E0818A41820021C17200F00EF8012017
:101BB000009001ABE3227221072000F0ECFB00282B
:101BC00001D100200EBD01200EBD38B50020ADF8BA
:101BD0000000DFF8D443608A002801D1A07A607247
:101BE0000722E07AC0EBC000DFF8C013411820469E
:101BF00001F0DDFFFFF798FF80208DF8000000ADB9
:101C000081206870022300AA7221072000F069FB7E
:101C1000002801D1002032BDA7208DF80000208AC5
:101C20006870022300AA7221072000F05AFB0028E6
:101C300001D1002032BD012032BD00009C86002071
:101C400030B585B0044600208DF80C00ADF80E00CC
:101C50006079029020790190E0780090A378627812
:101C600021780FF2B03000F0C6FA0120009003ABEB
:101C700080227221072000F08EFB002801D1002075
:101C800061E0C94D9DF80C0028720120009003AB63
:101C90008F227221072000F07EFB002801D1002056
:101CA00051E09DF80C00A8730120009003AB902236
:101CB0007221072000F06FFB002801D1002042E0D4
:101CC0009DF80C00E87300F0A6F88F208DF80E0048
:101CD0000DF10E050B20687002230DF10E0272212A
:101CE000072000F0FEFA002801D100202BE0902010
:101CF0008DF80E000120687002230DF10E02722192
:101D0000072000F0EEFA002801D100201BE0A84DCA
:101D10008122FF21284601F02BFB80222146681CEE
:101D200001F045FF0020287081232A4672210720F8
:101D300000F0D7FA002805D10FF2F02000F05BFA8E
:101D4000002000E0012005B030BD80B501780F29EA
:101D500004DA954A527A521C8A4205DA0FF2D820E8
:101D600000F049FA002002BD4278202A01DB20223F
:101D700042700022C2704271C1EBC1018B4A202324
:101D80008B54891800224A704278002A01D100221F
:101D900001E05200521E8A7182788A70C278CA703D
:101DA00002790A7140794871012002BD7E48417A6A
:101DB000491C417281720120704738B504467A4D42
:101DC0006C82FFF791FE002C00D0AC8221460FF20E
:101DD000782000F010FA012032BD734948730120C9
:101DE0007047744908700120704772480078704746
:101DF000000000001C8700209C86002080B56A49F6
:101E000008730A7B52000A8201460FF24C2000F050
:101E1000F2F9012002BD00B583B00020ADF8060044
:101E20008DF8040080208DF8060001208DF8070051
:101E300002230DF106027221072000F052FA002859
:101E400001D100200EBD102000905B4BA02272211A
:101E5000072000F0A0FA002801D100200EBD0120CB
:101E6000009001AB80227221072000F094FA002834
:101E700001D100200EBD01200EBD00B587B00020AD
:101E8000ADF8000001A8142103F0CAFD80208DF8F0
:101E9000000001208DF80100022300AA7221072012
:101EA00000F01FFA002801D1002013E0102242495F
:101EB0000DF1050001F07BFEA0208DF80400112338
:101EC00001AA7221072000F00CFA002801D100209D
:101ED00000E0012007B000BD30B583B00020ADF8B0
:101EE00004008DF80600304C217A0FF27C1000F0CF
:101EF00082F90020FFF7F4FD002060736072FFF7A5
:101F0000BCFF8F208DF8040001ADA07B6870022318
:101F100001AA7221072000F0E4F9002801D1002075
:101F20003EBD90208DF80400E07B6870022301AA7A
:101F30007221072000F0D5F9002801D100203EBD14
:101F400080208DF80400207A6870022301AA722193
:101F5000072000F0C6F9002801D100203EBD012075
:101F600000900DF10603E3227221072000F013FA1E
:101F7000002801D100203EBD01203EBD844C01203F
:101F800054500120C74F0120C84F0120C94F0120E4
:101F9000CA4F012055500120565001201C870020B7
:101FA000A487002048510120AC4F0120544101205A
:101FB0008C3C012069530120A8500120233E474555
:101FC0002043552025782025782025780000000022
:101FD000233E4753454C4600233E475354455252F7
:101FE00000000000233E4C4947500000233E4C4374
:101FF000484950203078257800000000233E3E4CB0
:1020000049474F00233E4C49474F0000233E4C496F
:10201000474300004D424420256420256420256468
:102020002025642025642025640000004D6F626532
:10203000616D2057460000004D6F6265616D20485C
:102040006F70204661696C004D4220486F70436F8D
:10205000756E7420256400004D6F6265616D204CC3
:10206000656E3D25640000004D4220436C6F736532
:10207000202564000104104041100008B110000840
:1020800059110008D111000800000000AF1300082A
:1020900000000000F1130008BD130008D715000868
:1020A00051160008F116000875170008000000001E
:1020B0007917000800000000000000000000000088
:1020C000BFF34F8FDFF81C07016801F4E061DFF810
:1020D000442711430160BFF34F8FFEE710B5DFF8CF
:1020E00038474FF48E720021204601F041F9204616
:1020F00010BDDFF82407704710B5FFF7EFFF044667
:1021000000231A461146084600F06FFAC046C04642
:1021100001F060FD204600F019F801F0B2FF204602
:1021200000F0D0F9204600F015F8204600F01FF826
:1021300000F093F900206072A072E0722073012019
:1021400060730020E075A073012010BD0021C171F3
:10215000017231E010B50446DFF88C0601F0E6FDAF
:10216000DFF8B80601F0E2FD0120607110BD10B586
:10217000044601F046FE0120A07110BD38B50446AA
:10218000012501F0F1FE012804D12846E07000206D
:10219000A0700AE0022804D10020E0702846A07058
:1021A00003E00020E070A0700546284632BD80B5EF
:1021B00002F058F8012002BD10B50446E07902F0A3
:1021C0008FF90121217010BD70B504460025E67914
:1021D000E171FFF7F1FF002807D02046FFF7BAFFB3
:1021E0002046FFF7C4FF012503E0E6712046FFF714
:1021F000E3FF284670BD0EB470B5C1B0054600A817
:102200004FF4807103F00CFCFFF773FF044645ABFD
:102210002A464FF4807100A803F00AFC00A803F0DE
:1022200025FC451C00A82818002100F8011CDFF837
:10223000F0653078401C30707078F021084202D090
:10224000992003F02FFC03F09AFC7078401C70700A
:10225000207E2818FF2810DA207E002803D0207E58
:1022600000190A2101762A4600A9207E001919309A
:1022700001F09DFC207E2818207600A803F0E8FEDF
:102280007078F021084202D0992003F00BFC70789E
:10229000401E7070C0B2002801D103F06AFC04F047
:1022A000C2FA41B070BC5DF810FB0428DFF83C05B1
:1022B00003D8DFF8341501607047DFF8601501605E
:1022C0007047DFF82C1551F82000007F002807D058
:1022D000DFF8500501784A1C0270032900DBEFE6A5
:1022E00070472DE9F84305460E4617464FF00208A1
:1022F000DFF82C456078F021084202D0992003F0E5
:10230000D1FB03F03CFC6078401C60709DF800003D
:10231000401E8DF8000017F8019B2846FFF7C5FF07
:1023200000AB4A463946304602F0F2F9002810D098
:102330006078F021084202D0992003F0B3FB607866
:10234000401E6070C0B2002801D103F012FC0120D1
:102350001FE05FFA88F8424629460FF2D440FFF7A3
:102360004AFF4046A0F101080028D9D16078F02149
:10237000084202D0992003F095FB6078401E6070FF
:10238000C0B2002801D103F0F4FB2846FFF799FF03
:102390000020BDE8F2832DE9F04704460D461646BD
:1023A0001F46DFF85084089888F80000DFF8709422
:1023B00099F80100F021084202D0992003F072FB45
:1023C00003F0DDFB99F80100401C89F8010020466C
:1023D000FFF76BFF4FF0020A434632463946284664
:1023E00002F046FA002813D099F80100F0210842C3
:1023F00002D0992003F056FB99F80100401E89F89D
:102400000100C0B2002801D103F0B3FB012022E09B
:102410005FFA8AFA524621460FF22040FFF7EBFEA0
:102420005046A0F1010A0028D6D199F80100F02108
:10243000084202D0992003F035FB99F80100401EB4
:1024400089F80100C0B2002801D103F092FB2046B8
:10245000FFF737FF0020BDE8F08703F00DBAF8B5AD
:10246000044602270025DFF888630DE039464F1E39
:10247000C9B200290AD1002804D120690121A9404C
:102480008843206102276D1C162D10DA56F82500AE
:10249000006E006880470128E8D121690122AA4026
:1024A0001143216156F8251001220A77E3E72069DC
:1024B000032803D0022801D0012802D140F4805023
:1024C0002061F1BD02F01CBB02F075BB81B000229F
:1024D000ADF80220ADF80020C079042808D0062805
:1024E00009D008280AD009280BD00A280CD00EE001
:1024F0004FF4C8600DE04FF448600AE04FF4C85054
:1025000007E04FF4FA5004E042F2107001E041F2AB
:102510007070ADF802200DE0BDF80020521CADF83F
:102520000020BDF800208242F6DBBDF80220521CDC
:10253000ADF80220BDF802208A4203D20022ADF895
:102540000020EEE701B07047417230B589B004F069
:1025500085FA0446FFF7CDFD054600A8242103F0C7
:102560005FFA0020ADF8220001900A208DF80800E3
:1025700000208DF809008DF80A00687A00280DD037
:10258000002C18D000208DF80000052001900B20B1
:102590008DF8080000A806F0AFFA0CE0002C0AD075
:1025A00001208DF80000052001900B208DF8080017
:1025B00000A806F0A1FA09B030BD02F018BB02F085
:1025C00020BB01210846F8E701210846F7E7022170
:1025D0000120F2E702210120F1E702F01DBB10B556
:1025E0000446FFF786FD447510BD2DE9F04782B023
:1025F0000C4615462F46264680464FF47A714FF01A
:102600003C0C4FF4616918FB09F216FB0C22BA1856
:1026100001FB0232DFF8E0E19EF900A01AFB09F9A4
:102620009EF901A01AFB0C9C9EF902904CFA89FCC1
:10263000BEF9039001FB0C919EF808C0BCF1000F9D
:1026400022D144EA00012943194302D001218EF826
:1026500008108EF80000B8F1000F04D59EF80000B5
:1026600018308EF800008EF801408EF80250AEF857
:10267000033000933B4632469EF900100FF2EC10F7
:10268000FFF7B9FDBDE8F38791420DD3A1EB020C32
:10269000ACF2D17CDFF89091CC45DAD30FF2A810E0
:1026A00002B0BDE8F047A6E5D3D2A2EB010CACF234
:1026B000D179DFF874A1D145CBD363460FF29810DE
:1026C00002B0BDE8F04796E510B504002FD004F045
:1026D0007BFA4949CA68002A00D0841AB1F803205D
:1026E000A218A1F8032012B2B2F57A7F06DBA2F598
:1026F0007A72A1F803208A78521C8A7091F902201C
:102700003C2A04DB3C3A8A704A78521C4A7091F9A0
:1027100001203C2A04DB3C3A4A700A78521C0A70B9
:1027200091F90020182A01DB00220A70C86010BD50
:102730003149052201F000BA0FB410B52DED028B1E
:102740002E4C104606F016FB2D4A2E4B06F02AFBA7
:10275000206161619FED2C8B049806F00BFB53EC1C
:10276000182B06F01FFB20606160059806F002FB45
:1027700053EC182B06F016FBA060E1609DF81C00DE
:10278000207604F118009DF81D1041709DF81E1070
:1027900081709DF81F10C1709DF820100171BDF867
:1027A000210000EE100AB8EE400A10EE100A06F002
:1027B000CBFB174A1D4B06F0F5FA06F0EDFBC4F80B
:1027C0001D00BDF82300A4F821009DF8250084F821
:1027D0002300BDEC028B10BC5DF814FB07492422DA
:1027E00001F0AAB90CED00E000540040E0870020A1
:1027F000086000206C530120B8500120E84D0120F2
:10280000FCA9F1D24D62503F8DEDB5A0F7C6B03EA8
:102810003BDF4F8D0400FA055C300120005800407A
:10282000CC8600206B5301205F4C2605976EA23F9B
:102830004957452025642025640000004952452061
:10284000256420256400000041542D5365745453C1
:10285000312025642025640041542D536574545360
:1028600032202564202564202564000041542D5326
:102870006574542025643A25643A25642E25640045
:1028800000487047D83A012000214FF0804200E014
:1028900092089042FCD3002A09D05318984203D3DF
:1028A000401A801A01EB420149089208F3E70846F2
:1028B0007047002802D400F07F0002E0404240F060
:1028C0008000C0B2704700F07F01802800DB4942E1
:1028D0000846704730B404460D46A54200DA2C463F
:1028E0001546A54200DA2C46A34200DA1C462046D3
:1028F00030BC704730B404460D46AC4200DA2C467A
:102900001546AC4200DA2C469C4200DA1C462046B2
:1029100030BC7047184900224A608A600861C8606C
:10292000704770B50546144CA06821696268236839
:102930009A4214DB91FBF3F6266190FBF3F0FFF76C
:10294000A3FFA060072804DB2846FFF7E3FF002071
:1029500070BDE660256100216160A16070BD521C00
:10296000626069182161E168491B01FB0100A060F8
:10297000002070BD00000000348700200EB4F0B5C8
:102980000999059A4A430092069A4A430192089A85
:102990004A4303921A465143029100A9102201F0C2
:1029A000DBF804B05DF810FB10B40C181C191019FA
:1029B00010BC70470A7822EA0000087070470A7855
:1029C00010430870704730B583B004460D460020B0
:1029D000ADF806000120009001AB224672210720CD
:1029E000FFF7D9FC002801D100203EBD01A92846EF
:1029F000FFF7E5FF8DF806409DF804008DF807000D
:102A000002230DF1060272210720FFF76AFC00285D
:102A100001D100203EBD01203EBD30B583B004464B
:102A20000D460020ADF806000120009001AB2246C3
:102A300072210720FFF7AFFC002801D100203EBD26
:102A400001A92846FFF7B6FF8DF806409DF804005F
:102A50008DF8070002230DF1060272210720FFF70F
:102A600040FC002801D100203EBD01203EBD50F8B1
:102A7000041B61B150F8042BD30744BFA9F1010333
:102A80009A18002342F8043B091FFAD1EFE7704778
:102A9000DFF8D40800210170C170082141708170F5
:102AA00000F015BDDFF8C0080078032801D101202F
:102AB000704700207047DFF8B0080078042801D183
:102AC000012070470020704710B5DFF89C4821783E
:102AD00000290FD10F219F20FFF79FFF06219F2084
:102AE000FFF771FF012020700020E07020710120AD
:102AF000607210BD012950D1617A002952D121792B
:102B000000291AD1E17802290AD06278520882425B
:102B100006D30120E07000F021F9002862D010BD3A
:102B200001295FD0A178490881425BD20220E07080
:102B300000F038F9002855D010BD01291ED1E178E8
:102B400002290AD062785208824206D30120E0703E
:102B500000F092F900280CD010BD012909D0A1780D
:102B60004908814205D20220E07000F0A9F900284E
:102B70006BD1E078012859D000202071022020700C
:102B80000020E0700F219F20FFF747FF09219F20C1
:102B9000FFF719FF0120607210BD022955D1617A3B
:102BA000002902D00020607210BD217900291ED1B9
:102BB000E17802290AD062785208824206D30120C5
:102BC000E07000F012F900280CD010BD012909D0E6
:102BD000A1784908814205D20220E07000F029F96D
:102BE000002832D10020E0700120207110BD0129A1
:102BF00021D1E17802290AD062785208824206D3B4
:102C00000120E07000F07FF900280CD010BD0129F0
:102C100009D0A1784908814205D20220E07000F075
:102C200096F9002811D1E078012802D10020E07047
:102C300010BD002020710F219F20FFF7EEFE032022
:102C400020700020E0700120607210BD38B50020B7
:102C5000ADF80000DFF814472078FFF734FE9D211F
:102C60008DF8001000ADFFF724FE6870022300AA63
:102C700072210720FFF735FB00280ED06078FFF7A0
:102C800022FE9E218DF80010FFF713FE68700223CC
:102C900000AA72210720FFF724FB31BD3FB581B0A8
:102CA000DFF8C4462078032856D101A80FC8FFF7E3
:102CB00011FE054601A80FC8FFF71CFE2179002967
:102CC00020D1E17802290BD06278AA4208DB0120EA
:102CD000E07001A80FC800F05DF900280DD03BE0BE
:102CE00001290AD0A178814207DA0220E07001A808
:102CF0000FC800F0CCF900282ED10020E070012090
:102D0000207129E0012923D1E17802290BD06278D2
:102D1000AA4208DB0120E07001A80FC800F02FFADA
:102D200000280DD018E001290AD0A178814207DAE5
:102D30000220E07001A80FC800F09DFA00280BD116
:102D400000202071E078012802D10020E07003E02B
:102D5000042020700020E07005B030BD10B582B0B6
:102D60000020ADF80000DFF804462078FFF7ABFD47
:102D700010F17B0F01DA002016BD9D218DF80010A7
:102D8000001FFFF796FD8DF801002070022300AAB6
:102D900072210720FFF7A5FA002801D1002016BDF7
:102DA000012016BD10B582B00020ADF80000DFF89C
:102DB000BC452078FFF787FD7C2801DB002016BD8D
:102DC0009D218DF80010001DFFF773FD8DF80100A7
:102DD0002070022300AA72210720FFF782FA002840
:102DE00001D1002016BD012016BD10B582B0002013
:102DF000ADF80000DFF874456078FFF764FD10F16E
:102E00007B0F01DA002016BD9E218DF80010001FF7
:102E1000FFF74FFD8DF801006070022300AA7221B8
:102E20000720FFF75EFA002801D1002016BD01201F
:102E300016BD10B582B00020ADF80000DFF82C45BB
:102E40006078FFF740FD7C2801DB002016BD9E2145
:102E50008DF80010001DFFF72CFD8DF8010060704B
:102E6000022300AA72210720FFF73BFA002801D1B4
:102E7000002016BD012016BD10B582B00020ADF8AF
:102E80000000DFF8E8442078FFF71DFD10F17F0F08
:102E900001D1002016BD9D218DF80010401EFFF7C6
:102EA00008FD8DF801002070022300AA722107207E
:102EB000FFF717FA002801D1002016BD012016BD2A
:102EC00010B582B00020ADF80000DFF8A0442078F3
:102ED000FFF7F9FC7F2801D1002016BD9D218DF858
:102EE0000010401CFFF7E5FC8DF801002070022364
:102EF00000AA72210720FFF7F4F9002801D1002071
:102F000016BD012016BD10B582B00020ADF800003E
:102F1000DFF858446078FFF7D6FC10F17F0F01D13D
:102F2000002016BD9E218DF80010401EFFF7C1FC49
:102F30008DF801006070022300AA72210720FFF7BC
:102F4000D0F9002801D1002016BD012016BD10B512
:102F500082B00020ADF80000DFF810446078FFF781
:102F6000B2FC7F2801D1002016BD9E218DF80010F3
:102F7000401CFFF79EFC8DF801006070022300AA40
:102F800072210720FFF7ADF9002801D1002016BDFE
:102F9000012016BD3FB581B000252846ADF80000E0
:102FA000DFF8C44301986178884217DA6079FFF747
:102FB0008AFC10F17A0F11DBA4218DF80010001F9C
:102FC000FFF777FC00A948706071022300AA722104
:102FD0000720FFF786F9002853D001250298617871
:102FE000884217DAA079FFF76EFC10F17A0F11DB37
:102FF000A5218DF80010001FFFF75BFC00A94870A9
:10300000A071022300AA72210720FFF76AF90028A5
:1030100037D0012503986178884217DAE079FFF705
:1030200052FC10F17A0F11DBA7218DF80010001F60
:10303000FFF73FFC00A94870E071022300AA72214B
:103040000720FFF74EF900281BD00125049861786E
:10305000884219DA207AFFF736FC10F17A0F13DB79
:10306000A9218DF80010001FFFF723FC00A948706C
:103070002072022300AA72210720FFF732F90028EC
:1030800001D1002001E00125284605B030BD3FB543
:1030900081B000252846ADF80000B34CA078019916
:1030A000884216DA6079FFF70EFC7B2811DAA4213A
:1030B0008DF80010001DFFF7FCFB00A9487060713F
:1030C000022300AA72210720FFF70BF9002850D035
:1030D0000125A0780299884216DAA079FFF7F3FB60
:1030E0007B2811DAA5218DF80010001DFFF7E1FB08
:1030F00000A94870A071022300AA72210720FFF7DF
:10310000F0F8002835D00125A0780399884216DA16
:10311000E079FFF7D8FB7B2811DAA7218DF80010A2
:10312000001DFFF7C6FB00A94870E071022300AA4A
:1031300072210720FFF7D5F800281AD00125A078C2
:103140000499884218DA207AFFF7BDFB7B2813DA4E
:10315000A9218DF80010001DFFF7ABFB00A94870F6
:103160002072022300AA72210720FFF7BAF8002874
:1031700001D1002001E00125284605B030BD3FB552
:1031800081B000252846ADF80000774C01986178A1
:10319000884217DA6079FFF796FB10F17F0F11D0A4
:1031A000A4218DF80010401EFFF783FB00A9487092
:1031B0006071022300AA72210720FFF792F800280D
:1031C00053D0012502986178884217DAA079FFF779
:1031D0007AFB10F17F0F11D0A5218DF80010401E51
:1031E000FFF767FB00A94870A071022300AA7221B3
:1031F0000720FFF776F8002837D00125039861787B
:10320000884217DAE079FFF75EFB10F17F0F11D0EB
:10321000A7218DF80010401EFFF74BFB00A9487056
:10322000E071022300AA72210720FFF75AF8002854
:103230001BD0012504986178884219DA207AFFF7BB
:1032400042FB10F17F0F13D0A9218DF80010401E12
:10325000FFF72FFB00A948702072022300AA7221F9
:103260000720FFF73EF8002801D1002001E00125EA
:10327000284605B030BD3FB581B000252846ADF8E1
:103280000000394CA0780199884216DA6079FFF77E
:103290001AFB7F2811D0A4218DF80010401CFFF7E5
:1032A00008FB00A948706071022300AA7221072060
:1032B000FFF717F8002850D00125A078029988421E
:1032C00016DAA079FFF7FFFA7F2811D0A5218DF833
:1032D0000010401CFFF7EDFA00A94870A07102230E
:1032E00000AA72210720FEF7FCFF002835D0012537
:1032F000A0780399884216DAE079FFF7E4FA7F288C
:1033000011D0A7218DF80010401CFFF7D2FA00A9B8
:103310004870E071022300AA72210720FEF7E1FF46
:1033200000281AD00125A0780499884218DA207A5A
:10333000FFF7C9FA7F2813D0A9218DF80010401C8F
:10334000FFF7B7FA00A948702072022300AA722181
:103350000720FEF7C6FF002801D1002001E001256B
:10336000284605B030BD0000C24F01205550012055
:1033700010B5044610460A460146204605F054FEA4
:10338000204610BDDFF860070021C161DFF85C173F
:1033900000220A7701224A7700221046086381F84A
:1033A0002000C87770470FB410B5DFF83C479DF890
:1033B0001D00411E8941C90F6177201D03A91022FC
:1033C00000F0CAFBDFF824079DF81E1041770021AA
:1033D00080F8201001779DF80810002907D1217F7F
:1033E0004A1C227706290EDB012101770BE0002021
:1033F0002077607F00289DF8080002D100F031F9A5
:1034000001E000F09DF810BC5DF814FB0FB438B576
:10341000DFF8D4469DF82400411E8941C90FE177A9
:10342000201D05A9102200F097FBDFF8C0569DF87B
:103430002600687705A80FC8FFF75CFA606168612D
:10344000002085F820002877E07F002804D105A817
:103450000FC800F0AEF909E0A07F002805A80FC84A
:1034600002D000F0DFF901E000F018FA31BC5DF89D
:1034700014FBF8B50446DFF8785605F11C06DFF8B2
:103480006806C17F4A1E9241D20F7275407F411E6D
:103490008941C90FB175DFF85476387F307597F8D8
:1034A00020002877284639461C2200F055FBB87FBB
:1034B000707005F12000DFF83C16102200F04CFB84
:1034C000204629463422BDE8F84000F045BB10B53F
:1034D00082B00020ADF80000A0208DF8000000AC04
:1034E00000206070DFF80C0600210174022300AA9E
:1034F00072210720FEF7F5FE002801D1002016BD3D
:10350000A1208DF80000FF206070022300AA722124
:103510000720FEF7E6FE002801D1002016BD80211D
:10352000A320FFF750FA3C21A220FFF74CFADFF866
:10353000B80500218177DFF8B4050163012016BDCD
:1035400010B50446DFF8A005807F0028204602D091
:10355000BDE810400BE000F03AF8DFF89005C07FBE
:10356000002803D12046BDE8104054E010BD38B516
:10357000DFF87845E07F012828D1DFF86C55201D61
:10358000291D102200F0E8FA04202070A069C72845
:103590000FD1201D0FC8FFF7ADF9A17F814208DAD6
:1035A000012085F8200001460FF25C50FEF723FE53
:1035B00007E0002085F8200001460FF26450FEF776
:1035C0001AFE012084F820000020E07731BD10B5FC
:1035D000DFF81845E17F012909D100F0CBF8002878
:1035E00002D00420E07710BD0020E06210BD002969
:1035F00009D100F0B6F8002802D00220E07710BD13
:103600000020E06210BDE06A411CE1620B2801DB92
:103610000020E06210BD10B5044600F055F82046C9
:1036200000F05DF8204600F065F8204600F06DF8E7
:10363000DFF8B404816A01EB8102D100642291FBBE
:10364000F2F1C26B836B9A4204DA006B052290FBA5
:10365000F2F003E0C06A142290FBF2F0BDE81040E3
:1036600090E038B5044600F014F8204600F01AF84F
:10367000DFF87454A86A00EB8001C800642190FB55
:10368000F1F104EB8400400000F07CF80120687741
:1036900031BDDFF854144FF4FA624A62C8228A62DC
:1036A000FFF738B9DFF84014C82212FB00F2CA62F3
:1036B000322212FB00F20A6300EB800252004A63DE
:1036C0008863C8630864704710B50146DFF8184482
:1036D00004F134020A2000F025F8206410BD10B572
:1036E0000146DFF8044404F13002322000F01AF8F9
:1036F000E06310BD10B50146DFF8EC4304F12C0285
:10370000C82000F00FF8A06310BD10B5FFF709F94D
:10371000642101FB00F4002C02D0204600F013F8D5
:10372000204610BD10B400EBD0735B10146809196B
:1037300000FB0131441C91FBF4F11160591891FB1D
:10374000F0F010BC704710B50146C82900DAC82156
:10375000DFF8944304F124020A20FFF7E3FFA0629C
:1037600010BDDFF88813496A814201DA01207047F1
:1037700000207047DD49896A884201DA01207047DC
:103780000020704740F2DD52904201DB40F2DC50F5
:103790000A2901DA0A2102E0652900DB6421081800
:1037A000401D0A2190FBF1F0C0B2D0494862886206
:1037B000704780B500F004F8CB480121C17701BD06
:1037C0000FB587B0C820019007A883B069460CC820
:1037D0000CC10CC80CC10EBC02A8FFF7CFF8C6483C
:1037E00002A9102200F0B8F90A20019007A883B0BE
:1037F00069460CC80CC10CC80CC10EBC02A8FFF76E
:10380000BDF8BE4802A9102200F0A6F9BC4807A9DD
:10381000102200F0A1F9BB4807A9102200F09CF982
:103820000BB000BD00BF1FB5B04CE07F002802D038
:1038300001280ED01FBD0020A061201D00A910226C
:1038400000F08AF902202070012084F82000E0773F
:103850001FBD201D00A9102200F07EF9012020705C
:10386000A069401CA061C72807D10121AB20FFF748
:10387000D4F80021AB20FFF7A6F8A069C82809DB1F
:103880000020A0610121AB20FFF7C7F80021AB2089
:10389000FFF799F8012084F820001FBD1FB5934C55
:1038A000E07F002803D0012084F8200003E000A876
:1038B0000FC800F037F800A80FC800F00AF8607FC2
:1038C000002805D0206B292802DBBDE81F40C9E095
:1038D0001FBD1FB5854CE07F012804D002280DD004
:1038E000042817D01FBD201D00A9102200F034F9B4
:1038F00001202070A069401CA0611FBD0020A061B4
:10390000201D00A9102200F027F9022020700120BC
:10391000E0771FBD042020700020E077012084F8AC
:1039200020001FBDFFB585B07048016B491C0163C5
:1039300005A883B069460CC80CC10CC80CC10EBCEC
:1039400001A800F025F805A883B069460CC80CC191
:103950000CC80CC10EBC01A800F03BF8694C94E8FF
:103960000F00FFF721F80546624E654F97E80F00FC
:10397000FFF71AF88542304604DA2146102200F09B
:10398000EBF803E03946102200F0E6F809B0F0BD8C
:103990000EB430B588B00446574802900BA882B0E8
:1039A00069460CC80CC10CC80CC10CBCC82103A8CA
:1039B00000F030F8524D284603A9102200F0CCF850
:1039C00020462946102200F0C7F808B030BC5DF848
:1039D00010FB0EB430B588B00446484802900BA8DE
:1039E00082B069460CC80CC10CC80CC10CBC0A21C1
:1039F00003A800F00FF8434D284603A9102200F059
:103A0000ABF820462946102200F0A6F808B030BCDA
:103A10005DF810FB0CB47FB504460D460C9E324693
:103A200008992846FFF77EFE0090321D0999284626
:103A3000FFF778FE019006F10C020B992846FFF77C
:103A400071FE039006F108020A992846FFF76AFE04
:103A50000290204600A9102200F07EF804B070BC4D
:103A60005DF80CFB70B582B00020ADF80000214C71
:103A700094E80F00FEF73EFF401D1C4DFF2802DDBD
:103A8000FF20A87700E0A877A0208DF8000000AE06
:103A9000686A707070782074022300AA722107206F
:103AA000FEF71FFC002801D1002076BDA1208DF873
:103AB0000000A87F7070022300AA72210720FEF781
:103AC00010FC002801D1002076BD8021A320FEF744
:103AD000A4FF3C21A220FEF7A0FF0348012181772B
:103AE00000202863084676BDAC4901201C4C01200B
:103AF000504C012044500120685001208850012082
:103B00007850012098500120233E445F6C6F6E670F
:103B10005F67657374757265203A20256400000044
:103B2000233E525F6C6F6E675F6765737475726575
:103B3000203A20256400000062B38B0708D0521E93
:103B400011F8013B00F8013B00F024808B07F6D10F
:103B5000830740F0208000BF103A07D330B4B1E8AB
:103B60003810103AA0E83810F9D230BC530724BFFF
:103B7000B1E80810A0E8081044BF51F8043B40F831
:103B8000043BD20724BF31F8022B20F8022B44BF9C
:103B90000B7803707047083A07D3B1E80810083A69
:103BA00040F8043B40F804CBF7D25307E4E710B5E4
:103BB0000446FFF7C1FF204610BD8268521C826098
:103BC000426832B10268531C036011704168491E9B
:103BD0004160704730B583B00121032005F0BDFA84
:103BE000DFF8804C204605F051FBDFF87C5C28466E
:103BF00005F04CFB01208DF8040000208DF8050035
:103C000001208DF8060000208DF8070001212846CC
:103C10000183C0460120009000A9284605F092FBD0
:103C2000022128460183C0460220009000A92846B0
:103C300005F088FB01208DF8040000208DF80500B8
:103C4000ADF806004FF48070009000A9284605F0FA
:103C500079FB4FF4807128464183C04601208DF8DE
:103C6000040000208DF8050001208DF806000020DA
:103C70008DF807004FF48050009000A9204605F011
:103C800061FB4FF4805120464183C0460422062147
:103C9000284605F0A5FB04220721284605F0A0FBD5
:103CA00002208DF8040001208DF805008DF8060033
:103CB00000208DF807004020009000A9284605F05C
:103CC00041FB8020009000A9284605F03BFB042220
:103CD0000A21284605F084FB09220321284605F025
:103CE0007FFB02208DF8040001208DF805008DF87F
:103CF000060000208DF807004FF48060009000A9B6
:103D0000284605F01FFB0820009000A9284605F072
:103D100019FB286820F0300040F01000286020686F
:103D200020F0300040F01000206037BD1FB5DFF8F4
:103D30003C4BA04230D101214FF4001005F018FA9D
:103D40000121022005F009FA01214FF4001005F0CD
:103D500030FA00214FF4001005F02BFA0020ADF8E6
:103D600004004BF6FF70ADF806004FF48060ADF82C
:103D70000A004FF48040ADF80C000A20ADF80800AE
:103D8000DFF8CC0C009000A9204605F06CFB012167
:103D9000204605F0CBFB1FBDDFF8B84CA0422FD169
:103DA00001214FF4800005F0E3F90121022005F024
:103DB000D4F901214FF4800005F0FBF900214FF404
:103DC000800005F0F6F90020ADF804004BF6FF7016
:103DD000ADF806004FF48060ADF80A004FF4804063
:103DE000ADF80C000A20ADF80800DFF8640C009074
:103DF00000A9204605F037FB0121204605F096FB7F
:103E00001FBD2DE9F04192B001214FF4805005F023
:103E1000BAF90121084605F0A0F901214FF480000C
:103E200005F09BF9DFF83C4A05221146204605F0D3
:103E3000D7FA05220721204605F0D2FA05220621ED
:103E4000204605F0CDFA05220421204605F0C8FAE7
:103E500002208DF8040001208DF805000020ADF847
:103E600006002020009000A9204605F06BFA802073
:103E7000009000A9204605F065FA4020009000A9B6
:103E8000204605F05FFA1020009000A9204605F0BA
:103E900059FADFF8C44B204605F0AAFBDFF8BC5BFB
:103EA0000020288068600120288100206881E86067
:103EB0000720288200206880DFF8A46B304605F0D8
:103EC00007FCDFF8A07B384605F002FC4FF4806069
:103ED000069000210D9103210E9100210F910A916E
:103EE0000890DFF8180C039008461090099007908E
:103EF0004FF400300C9008460B904FF0C068CDF89E
:103F00000880402005900846049002A9304605F03C
:103F100063FC00200B90CDF80880059005F114009B
:103F2000049002A9384605F057FC00206880294615
:103F3000204605F08CFB01220221204605F0B6FB4D
:103F400001221146204605F0B1FB0121204605F073
:103F5000A1FB0021304605F066FC0021384605F043
:103F600062FC12B0BDE8F08130B589B001214FF09C
:103F7000805005F0FDF8012005F0BEFC01214FF452
:103F8000802005F0EAF80F2005F066FE04461020B8
:103F900005F062FE0546012005F0DCF8002005F082
:103FA000D9F821460F2005F04AFE2946102005F0D9
:103FB00046FE00214FF4802005F0CFF8012005F0E7
:103FC00067F8412005F016F90028FAD04FF4807008
:103FD00005F0AAF8012005F0BAF805F0E0FC3F2052
:103FE000069040F2FF1007900020059005A805F00C
:103FF0008DFC0020029002A905F0F2FC00208DF853
:10400000070001208DF804008DF805008DF80600EA
:1040100001A9002005F05DFD4FF4800005F0FCFED5
:104020004FF48000039000208DF8100008208DF8D8
:10403000110001208DF8120003A805F0ABFE03204B
:104040008DF800000D208DF8010000208DF8020091
:1040500001208DF8030000A805F0EBFE032005F019
:10406000ACFD4FF4804005F062FE4FF4800005F097
:10407000D3FE01214FF4804005F01FFE012009B05E
:1040800030BD10B586B00121084605F066F8012163
:104090004FF4804005F077F800208DF810008DF87F
:1040A000130001200390DFF8BC4703A9204605F068
:1040B00049F90420039003A9204605F043F90021A3
:1040C000084605F0EFFE0221002005F0EBFE00207F
:1040D0008DF8080001208DF80A0001900C208DF861
:1040E000090001A805F056FE042001900C208DF86F
:1040F000090001A805F04EFE042005F08DFE2820E1
:104100008DF800000F208DF8010000208DF80200CE
:1041100001208DF8030000A805F08BFE06B010BD4D
:1041200010B586B00121084605F017F801214FF4BB
:10413000804005F028F800208DF810008DF813005D
:104140004FF40064039403A9DFF8180705F0FAF8A8
:104150000B21002005F0A6FE00208DF808000120AC
:104160008DF80A0001940C208DF8090001A805F0D3
:1041700011FE204605F050FE28208DF800000F208B
:104180008DF8010000208DF8020001208DF8030059
:1041900000A805F04EFE06B010BD30B58DB0044647
:1041A00001214FF4807004F0EEFF00A805F004F93F
:1041B0000A20009003208DF8040000208DF80700ED
:1041C00000A9DFF8A00605F0BDF805F07FFE02A803
:1041D00005F0C1FE4FF48030039002A805F0ADFE5B
:1041E00006A805F0A0FEDFF8DC5A06A9284605F06F
:1041F0007AFE072301222146284605F0BDFE012153
:10420000284605F0FCFE0121284605F0AAFE0DB067
:1042100030BD38B5DFF8AC4A204605F0EBFE4FF470
:104220007A750221204605F001FF002803D12846B7
:10423000451E0128F5DA2046BDE8324005F0EABE09
:1042400080B50021DFF87C0A05F08BFE00214FF4D9
:104250008070BDE8044004F096BFDFF8280B0068CA
:104260007047000038B5040040D0012005F044FB41
:10427000002005F0BCFC4FF40055042005F038FD8B
:10428000012804D12846451E80B20028F5D100EE51
:10429000104AB8EE400ADFED800A80EE800AF0EEA8
:1042A000000A20EE200ADFED7D0A80EE800ABDEED6
:1042B000C00A10EE100A401E80B205F08EFC4FF4CA
:1042C000804005F034FD4FF4800005F0A5FD01208D
:1042D00005F08DFCDFF8AC0A012181600460214605
:1042E0000FF22000BDE83440FDF785BFDFF8940AE7
:1042F00000210160012005F0FFFA0020BDE83240F6
:1043000005F075BC536574525443203D202564006C
:1043100030B4014601200023DFF86C2A1C4694606B
:10432000946814F00C0FFBD10C460B2C55D8DFE829
:1043300004F02054545406192031383F464D9468F7
:1043400044F080049460DFF8444A4FF4C06525606F
:10435000146824F080741460DFF8B44ADFF8305A2F
:1043600025603BE00346DFF8A84ADFF8A85A25603D
:1043700034E094689460DFF8144A4FF4C065256017
:10438000146824F080741460DFF8844ADFF8885AD7
:10439000256023E00223DFF8784ADFF8805A2560A1
:1043A0001CE00323DFF8684ADFF8745A256015E043
:1043B0000423DFF85C4ADFF8C45A25600EE00523C9
:1043C000DFF84C4ADFF8B85A256007E00623DFF82B
:1043D000404ADFF8B05A256000E01846002B4AD06A
:1043E00003EBC3030FF2B8041B19946894601468BC
:1043F00024F080741460146824F0806414609C7845
:104400001D8844EA8514DD786D086D1E44EA054474
:104410001D7944EA05645460DC881D7A2D0745EA5D
:104420008414DFF8BC5A2C60146844F08074146063
:104430001468A401FCD55B7943F4C063DFF84C49F0
:1044400023609368936093689360052904D1916811
:1044500041F09001916005E00A2903D1916841F48F
:1044600080519160916841F002019160916801F082
:104470000C010829FAD1DFF898190968DFF8642AD5
:10448000914207D2DFF8F01A0A6822F4404242F45F
:1044900080420A6030BC704700007A440000004748
:1044A000200110040F03020103F00010060F0102A7
:1044B0000103C00010080F01020103C00010060F25
:1044C00001020103F00010060F01020103C80010F1
:1044D000040F02020103A80010020F0302010300EF
:1044E00016E7002800E0401EFDD170477CB5072686
:1044F000DE4988426BD101208DF804008DF805005B
:104500008DF8060000208DF8070040200090DFF8AD
:10451000885A00A9284604F015FF8020009000A9C1
:10452000284604F00FFF402128464183C0460F2053
:10453000FFF7D7FF402128460183C0460F20FFF731
:10454000D0FF3046461E80B20028ECD1802000907B
:1045500000A9284604F0F6FE402128464183C046C3
:104560000520FFF7BEFF802128460183C0460520B5
:10457000FFF7B7FF402128460183C0460A20FFF716
:10458000B0FF402128464183C0460520FFF7A9FF20
:10459000802128464183C0460520FFF7A2FF022064
:1045A0008DF8040001208DF805008DF8060000202C
:1045B0008DF807004020009000A9284604F0C2FEB4
:1045C0008020009000A9284604F0BCFE73BDDFF8EF
:1045D000841488426AD101208DF804008DF805000A
:1045E0008DF8060000208DF807004FF480640094D9
:1045F000DFF8A45900A9284604F0A4FE0820009082
:1046000000A9284604F09EFE214628464183C04664
:104610000A20FFF766FF214628460183C0460A208C
:10462000FFF75FFF3046461E80B20028ECD108201D
:10463000009000A9284604F085FE214628464183C3
:10464000C0460520FFF74DFF082128460183C046DC
:104650000520FFF746FF214628460183C0460A2071
:10466000FFF73FFF214628464183C0460520FFF75C
:1046700038FF082128464183C0460520FFF731FF57
:1046800002208DF8040001208DF805008DF8060049
:1046900000208DF80700009400A9284604F052FE7F
:1046A0000820009000A9284604F04CFE73BD10B508
:1046B000DFF8E8480121206804F071FF206804F069
:1046C000A3FE2068FFF732FB05E02068FFF70EFF2E
:1046D0002068FFF72BFB4FF40031206804F06AFFDD
:1046E0000028F2D110BD30B40022838A008BDFF89D
:1046F000AC48656843EA00400840000255EA1020D3
:1047000060600840884200D10122104630BC7047EA
:104710002DE9F84F04460D4616464FF420491F7800
:10472000DFF878884FF40031D8F8000004F042FF39
:10473000002808D04846A0F101090028F2D1FFF76F
:10474000B6FF00208CE0D8F8000001884FF6FF5239
:10475000114001800121D8F8000004F0F3FE4FF46D
:10476000805AD1460020C8F80400D8F800B0DFF81D
:1047700030185846FFF7B7FF002805D14846A0F18A
:1047800001090028F1D163E0D146002221465846B4
:1047900004F0F0FE0020C8F80400D8F80040DFF86C
:1047A00004182046FFF79FFF002805D14846A0F1D6
:1047B00001090028F1D14BE03146C9B220460182FF
:1047C000C046D1460020C8F80400D8F80040DFF801
:1047D000D8172046FFF787FF002805D14846A0F1EB
:1047E00001090028F1D133E0012F15D129782046A5
:1047F0000182C046D1460020C8F80400DFF8AC179B
:10480000D8F80000FFF76FFF002823D14846A0F139
:1048100001090028F2D11BE03846471EC0B200282B
:1048200018D015F8011BD8F800000182C046D14607
:104830000020C8F80400DFF87417D8F80000FFF76C
:1048400052FF0028E8D14846A0F101090028F2D122
:10485000002005E00121D8F8000004F07FFE0120CF
:10486000BDE8F28F00000240000402400054004006
:104870002DE9F54F81B00D461E464FF4204837789C
:10488000DFF818474FF40031206804F093FE002849
:1048900008D04046A0F101080028F3D1FFF707FF38
:1048A0000020D3E0206801884FF6FF5211400180BC
:1048B0000121206804F046FE4FF48059C8460020CC
:1048C0006060DFF8DCA6D4F800B051465846FFF728
:1048D0000AFF002805D14046A0F101080028F2D1C6
:1048E00091E000229DF80410584604F043FEC846AB
:1048F00000206060D4F800B0DFF8A8165846FFF733
:10490000F2FE002805D14046A0F101080028F1D1AF
:1049100079E0BDF80810C9B258460182C046C846C1
:10492000DFF88C16206804F045FE002805D14046CB
:10493000A0F101080028F3D165E00121206804F00E
:1049400001FEC84600206060D4F800B051465846C9
:10495000FFF7C9FE002805D14046A0F10108002854
:10496000F2D150E001229DF80410584604F002FEF6
:10497000022FC84639DADFF83C16206804F01AFE28
:10498000002805D14046A0F101080028F3D13AE003
:104990000021206804F0F7FD2068018B012104F05C
:1049A000DDFDC846DFF81016206804F003FE00287D
:1049B00005D14046A0F101080028F3D123E020688A
:1049C000008AC0B228703078401E3070C846206817
:1049D0000188890505D54046A0F101080028F6D1D7
:1049E00011E0012104F0CFFD2BE000206060DFF832
:1049F000CC152068FFF777FE002806D14046A0F1CD
:104A000001080028F3D1002020E0012616E0012F44
:104A10000CD1012E0AD100263146206804F0B3FDE6
:104A20002068818A018B012104F098FD2068818A29
:104A3000490603D5008A05F8010B7F1EFFB2002F3F
:104A4000E5D10121206804F09EFD0120BDE8FE8F24
:104A5000801A06000058004000300140C44D01207B
:104A60008864024010640240DFF854050168082998
:104A700033D1DFF814130A6842F080720A6042688A
:104A8000B2F1806F03D10A6842F080620A600A685E
:104A90009201FCD58A6842F002028A608A6802F0BC
:104AA0000C02082AFAD14268B2F1806F02D10A687A
:104AB0001201FCD5DFF858130968DFF82824914269
:104AC00007D2DFF8B4140A6822F4404242F480426C
:104AD0000A6000210160416070474168B1F1806F58
:104AE00009D1A9490A6842F080620A600A68120185
:104AF000FCD5002141607047000000000C300140EF
:104B0000DFF8C004016841F080510160DFF86804FB
:104B100001688908890041F001010160DFF8A804FB
:104B20000FF205014160704738B5DFF8A0442088D6
:104B300040F004002080FDF7DCFA807A012803D1E0
:104B4000012004F0DCFE02E0002004F0D8FEDFF8D3
:104B500080548021DFF87C0404F0B2FD002818D1D5
:104B600072B68948DFF85814826802F00C020A60B5
:104B7000006800F080604860286840F00400286009
:104B800030BF62B6286820F004002860FFF76CFF91
:104B90000CE0608840F004006080286820F0040089
:104BA000286030BF286840F004002860608840F02A
:104BB0000400608031BDDFF8100440680047DFF872
:104BC0001814012806D010D3032809D005D30428CF
:104BD00009D00AE0DFF8C01307E0DFF8001404E0B2
:104BE000DFF8FC1301E0DFF8FC130846704710B54E
:104BF0000C46FFF7E4FF214689B2BDE8104004F0FF
:104C0000EBBB10B50C46FFF7DAFF214689B2BDE8D1
:104C1000104004F0E3BB0000E0B500238DF808303D
:104C200001238DF80A30002A03D10C228DF80920C7
:104C300002E008228DF8092004283CD8DFE800F0C3
:104C40000315212A2A004FF40060019028208DF8D6
:104C500000000F208DF8010000208DF802000129CE
:104C600021D118468DF803001FE01846019010204E
:104C70008DF8090006208DF800000E208DF8010047
:104C8000EAE70220019007208DF800000F208DF840
:104C90000100E1E70420019008208DF800000F20BA
:104CA0008DF80100D8E78DF8030001A805F072F82F
:104CB00000A805F0BEF807BD4FF40061C64804F037
:104CC00084BB00000020014010B5044601214FF4D0
:104CD000802004F042FA2146102004F0B0FF0021A9
:104CE0004FF48020BDE8104004F037BA10B5012120
:104CF0004FF4802004F031FA102004F0ADFF044698
:104D000000214FF4802004F028FA7B2004F072FA8E
:104D1000002802D099A0FDF76EFA7A2004F06AFA12
:104D2000002802D096A0FDF766FA792004F062FA16
:104D3000002802D093A0FDF75EFA7C2004F05AFA16
:104D4000002802D090A0FDF756FA7D2004F052FA18
:104D5000002802D08DA0FDF74EFA7E2004F04AFA1A
:104D6000002802D08AA0FDF746FA7F2004F042FA1C
:104D7000002802D087A0FDF73EFA04F04DFA204645
:104D8000C0B210BD5451012000380240003C024026
:104D900000127A003EB50C4615460422014602A8D0
:104DA000FEF705FF0422214601A8FEF700FF0422BA
:104DB000294600A8FEF7FBFE02A9002004F010FE21
:104DC00001A9002004F085FE04F07EFE0446864A18
:104DD000002300981946101A63EB0101490241EAC9
:104DE000D051400205F04CF90090844205D2011BDD
:104DF0004FF0004004F03DFF37BDA04207D2C4F59C
:104E00000070009909184FF0004004F032FF37BDE0
:104E100080870020809698000024F40000366E0100
:104E20000048E8012DE9704384B004460D4616465B
:104E300002A9002004F023FE01A9002004F099FE3D
:104E400004F042FE0090684AA2FB00894FEA58280D
:104E500048EAC958A2EB08000090042202A92046A3
:104E6000FEF7A5FE042201A92846FEF7A0FE0422B3
:104E700000A93046FEF79BFEBDE87F83005A620220
:104E800080F0FA0200BD010570B48C1E012C01DA1D
:104E90000C34401E3C216425B0FBF5F5C5EB9005B4
:104EA0004FF4C876B0FBF6F6751940F26F167443EE
:104EB0000C26B4FBF6F46419121940F26D1404FBCD
:104EC00000204A4A101800EB400203EBC200039A8C
:104ED00001FB0020049A01FB002070BC7047000019
:104EE00084380240018793031CB50C460168019188
:104EF000416800918368C2680169491C406900F2F9
:104F00006C70FFF7C1FF2060002016BD10B58EB099
:104F100037480068C405E40D01A9002004F0AFFD86
:104F200000A9002004F025FE9DF8040006909DF8DD
:104F3000050005909DF8060004909DF80100401EB4
:104F400008909DF8020007909DF8030064300990D6
:104F500002A904A8FFF7C8FF4FF47A7010FB04F011
:104F6000400AC0F57A700390029A4FF47A73C11721
:104F7000E3FB02010EB010BD00700040504F520024
:104F800050494E00424F5200534654004957440086
:104F9000575744004C50570000040240E08700205F
:104FA0000100030082000700800007008400070062
:104FB0000400001002000010400000100200030076
:104FC0006C52012040380240545101201800024028
:104FD00010ED00E0003001400000024000080240F7
:104FE000000C02400010024000CA9A3B7505F5FF14
:104FF00028280040506002604160086070470A68DD
:10500000F8E748600160704701684068F9E7F8B563
:105010000600DFF8C05802D505F15800F2BD05F1D1
:1050200058040020296F00E0096805F170029142E0
:1050300004D00C46A2689642F6D10120002840D147
:10504000A86FD0F88070182005F092F80446A6608A
:10505000002F05D0B74203D2B6FBF7F0784300E04B
:105060003046E060002F02D0B74200D23E462661B3
:1050700000202075DFF860683078401C3070707850
:10508000F021084202D0992000F00CFD00F077FDDD
:105090007078401C707005F170012046FFF7AFFF7B
:1050A0007078F021084202D0992000F0FBFC707863
:1050B000401E7070C0B2002801D100F05AFD01F00E
:1050C000B2FB2046F2BD38B5044694F9140000281E
:1050D00029D1DFF804582878401C28706878F0211E
:1050E000084202D0992000F0DDFC00F048FD68780D
:1050F000401C68702046FFF787FF204605F050F8F7
:105100006878F021084202D0992000F0CBFC687842
:10511000401E6870C0B2002801D100F02AFDBDE831
:10512000314001F080BB31BDF8B5044608466FF050
:105130000045FFF76CFF064694F9050094F904104A
:10514000814214D1C01C800005F012F8074694F982
:105150000500012807DB820021683846FEF727FD9D
:10516000206805F01DF827606079C01C607194F913
:105170000400411C2171216841F82060DFF85C07C0
:10518000864202D0307D401C3075002008E0216846
:1051900051F820108A68954201DB1546A160401C39
:1051A00094F904108842F2DBF1BDF8B504466FF0C3
:1051B0000046DFF8202702F1580502F158004FF0B1
:1051C000FF33002704E0664501DB664675467F1C19
:1051D00094F904C067450DDAD4F800C05CF827E004
:1051E000DEF808C0002BEED58C45ECD170463B466E
:1051F0005BB2ECE7002B11D4BCF1010F0EDB06E033
:10520000216801EB8306766841F823605B1C94F902
:1052100004104E1EB342F3DB491E217102F1580106
:10522000884204D0017D491E0175FFF74CFFA5603F
:10523000F1BD10B4C26A836B406C9C68002C02D52F
:105240006FF0004300E01B698468002C02D56FF00A
:10525000004000E00069984200DD1846D2685143E2
:10526000884201DB012000E0002010BC704738B507
:10527000DFF860168A6FD36E012490F90850AC40B5
:105280002343D36601F66C11FFF7B9FE012032BD4E
:1052900010B5DFF84016896FCA6E012390F90840F7
:1052A000A3409A43CA66FFF7AFFE012010BD01205C
:1052B00070472DE9FC4104460D4616461F4604F191
:1052C0002400FFF731FF07EB470004EB800831466D
:1052D00008F13000FFF728FF019598F9340000909D
:1052E0003B46627A94F908100FF2F450FCF783FF02
:1052F000BDE8F3812DE9FC4104460D4616461F46E4
:1053000004F12400FFF751FF07EB470004EB80088E
:10531000314608F13000FFF748FF019598F9340055
:1053200000903B46627A94F908100FF2C850FCF7DF
:1053300062FFBDE8F381C16A8A68012A09DB096955
:10534000012906DA006D002801D5002070470220EF
:1053500070470020704701EB410200EB8201896B2E
:105360008A68012A09DB0969012906DA006D00282B
:1053700001D50020704702207047002070470029A7
:1053800000D5D8E7E7E7012900DA012113460A46EC
:105390008FE7012900DA012113460A46AAE7DFF860
:1053A0003405C06A417A481E8041C00F70471346D9
:1053B0004FF0FF3211467CE713464FF0FF321146A3
:1053C00098E780B5DFF80C050068417A002902D122
:1053D000006E40688047012002BD80B5FFF758FF8E
:1053E000DFF8F0040068417A002902D1006E80687D
:1053F0008047012002BDB1F57A7F01DC4FF47A715C
:1054000013460A464FF4FA7153E7B1F57A7F01DC8F
:105410004FF47A7113460A464FF4FA716AE710B5F1
:105420000446002922D5E06A816801291CDB006955
:10543000012819DA02212046FFF7FBFE002813D1CC
:1054400094F9540010F1010F04D1002084F85400A5
:10545000012010BD002807D1012060774FF0FF30F8
:1054600084F85400022010BD002010BDBDE810409B
:1054700071E74FF0FF3280F85420F8E6DFF854244B
:10548000926FD2F88020A03252420265EFE60029E6
:105490000AD5C06A8168012904DB0069012801DAA4
:1054A000022070470020704755E7B52900DAB42183
:1054B00013460A463C21FCE6B52900DAB42113461E
:1054C0000A463C2116E710B50446002927D5E06AB4
:1054D0008168012921DB006901281EDA03212046A9
:1054E000FFF7A7FE002818D194F95400014611F1E6
:1054F000010F04D1002084F85400012010BD0028C1
:1055000003D1012084F8540010BD012905D14FF0CA
:10551000FF3084F85400022010BD002010BDBDE80B
:10552000104018E74FF0FF3280F85420DFF8A42332
:10553000926FD2F88020B4325242026597E6DFF8CB
:105540009423926FD2F880206432524202658EE634
:1055500013464FF0FF321146ABE613464FF0FF32D1
:105560001146C7E680B5FFF782FEFCF7C2FD0021B9
:105570000175012002BD80B5FFF78AFEFCF7B9FD79
:1055800000210175012002BD2DE9F0410C46D14DED
:1055900055F82060307206F154070FF26C31396112
:1055A000152800F22F81DFE810F0160026003300E6
:1055B00053004300620073008200B2009200A20018
:1055C000C200D200E000EC00F90007011401210143
:1055D00021012101210106F10800062141760A215D
:1055E000817605F67411416040F2DC5181600FF262
:1055F0003430386106E106F10800062141760A21BF
:10560000817605F6507141604FF496718160F9E042
:1056100006F108000C2141761021817605F58051B4
:1056200090314160102181600FF24C303861E9E027
:1056300006F10800072141760B21817605F580519E
:10564000843141600B2181600FF22C303861D9E048
:1056500006F10800062141760A21817605F585517B
:1056600041600A2181600FF210303861CAE006F112
:105670000800062141760A21817605F58051AC317A
:1056800041604FF4FA7181600FF208303861B9E07F
:1056900006F10800142141761821817605F595510F
:1056A0004160182181600FF25C303861AAE006F198
:1056B0000800022141760621817605F59051D4310A
:1056C0004160062181600FF2043038619AE006F1F2
:1056D00008000A2141760E21817605F59051C431EA
:1056E00041600E2181600FF2C82038618AE006F126
:1056F0000800012141760521817605F59051DC31C4
:105700004160052181600FF2E02038617AE006F106
:105710000800052141760921817605F59051B831BF
:105720004160092181600FF2342038616AE006F19E
:105730000800062141760A21817605F59051E43171
:1057400041600A2181600FF2F81038615AE006F1D9
:105750000800012141760521817605F59051F0314F
:10576000416040F2866181604CE006F10800012151
:1057700041760521817605F5CC5141600521816096
:1057800040E006F108000C2141761021817605F5F4
:10579000C851883141601021816033E006F1080072
:1057A000112141761521817605F5C8519831416066
:1057B00040F63401816025E006F1080011214176B0
:1057C0001521817605F50451CC31416015218160A8
:1057D00018E006F10800042141760821817605F5DC
:1057E000C85178314160082181600BE006F1080062
:1057F000012141760521817605F580517C3141609A
:105800000521816006F1080000210175417581754F
:105810000176C1600161417006F128080846C8F8A8
:1058200028004FF0FF3086F854007880062206F1F9
:105830005800FDF79DFD002010E000EB400106EB55
:105840008101002281F8342034314A7005F1580278
:105850004A6006EB800100228A64401C0228ECDBCF
:10586000002086F8280088F8010005F15800C8F8E3
:105870000400FC60BDE8F08110B5164CFDF700F89F
:10588000A067002006E0682111FB00417C3144F84C
:105890002010401C1628F6DB4FF0FF3020666066B3
:1058A0000020A06605F040FF06F0A4FD07F035FAE1
:1058B000FBF794FB07F0BAFBFBF788FEFCF70BF94C
:1058C00007F01EFC07F06DFF07F01FFCBDE810405D
:1058D00007F02CBC08600020CC860020606000200F
:1058E00041442025642025642025642025642C2043
:1058F00025640000524D2025642025642025642065
:105900002564202564000000AF5200086F52000893
:10591000AF520008915200088753000893530008C3
:105920007F5300089F5300086F5200089F530008E0
:105930009152000887530008935300087F530008D2
:10594000C35300086F520008AF520008DB53000831
:10595000AF530008B95300087F530008AF52000846
:1059600073540008AF52000891520008F753000822
:105970000B5400081F540008AF5200087D54000863
:10598000AF52000891520008875300089353000853
:105990008F540008AF52000825550008AF52000888
:1059A00091520008AB540008B9540008C7540008CD
:1059B000AF5200083F550008AF520008915200084E
:1059C00087530008935300087F530008AF52000824
:1059D00065550008AF52000877550008515500087A
:1059E0005B5500087F530008AF5200086F52000853
:1059F000AF520008915200088753000893530008E3
:105A00007F530008AF5200086F520008AF520008E1
:105A100091520008515500085B5500087F5300085B
:105A2000002207F05BBF0268531C036011707047CF
:105A300008B584B00023029311B90093019302E0EA
:105A40000090481E019004AB00A907487844183024
:105A500007F05EFF009909B100220A70002858BFC4
:105A6000029805B000BD00BF53E1FFFF00F1010344
:105A7000810704D010F8011B89B18107FAD10268AF
:105A8000B2F10131914311F0803F04BF50F8042F6F
:105A9000F6E710F8011B11B110F8011BFBE7C01A63
:105AA0007047000000B585B002460FF2140100A84F
:105AB00008F0FAFD00A800F093FB05B000BD00005F
:105AC0004F4525640000000030488168002904BF6C
:105AD00008B008E0EFF30982A2F12802036882E827
:105AE000F84F83685A6000F045FD816859B14A68F3
:105AF00092E8F84F036002F1280282F3098813F458
:105B00007F4F36D07047224822490968401A80F3F7
:105B100008884FF08071C1611F4981617FF0060ED6
:105B2000704701BC2046DFF874E000BDFEE71C486A
:105B3000006818490968401A203820F0070080F3EF
:105B400008884FF0000181F3118862B600F00DF86B
:105B5000FEE74FF0000181F311881249124A0A60F2
:105B60004FF0800181F3118870470E490E4A0A6098
:105B700070474FF0000181F31188704700BF4FF06C
:105B8000800181F31188704700BF0000CC8600209F
:105B9000E01F0020E44C0308F1E900082D5B000839
:105BA0000000000804ED00E000000010EFF30380A7
:105BB0007047BFF34F8FDFF86C06016801F4E061B6
:105BC000DFF8642611430160BFF34F8FFEE770B525
:105BD00082B006460C462046FFF748FF0546202DBA
:105BE00005D10422314600A8FDF7E1FF06E0102DA3
:105BF00016D10222314600A8FDF7D9FF002000E0AF
:105C0000401CA8420EDA015D7829F9D0009A2B4693
:105C10005B1E1B1ADA4002F0010230398A42EFD0D3
:105C2000002076BD012076BDDFF800160160062059
:105C30007047A0F10060B0F53E3F01D801207047E9
:105C400000207047F8B504460D46002000902068FB
:105C5000FFF7EFFF00281AD000A8FFF7E5FF064680
:105C6000002700E07F1CB74211D2009850F837108F
:105C700000EBC700406840422268520810EB420027
:105C8000FFF7A5FF0028EDD02F600120F2BD002016
:105C9000F2BDF8B50C46DFF898150A6D4B6D00257E
:105CA00059082E465F1B062F11D3482707FB0127F3
:105CB0003F6C874200D20D46B84200D20B46E9182D
:105CC000490837467E1C1F2FECD300E06D1C9D4217
:105CD00011D2482707FB05210E6CB042F6D34E6C5B
:105CE0008642F3D34022204608F0F8FC002084F8D6
:105CF00040000120F2BD40220FF20061204608F072
:105D0000EDFC0020F2BDF0B591B0044600250EE098
:105D100032590FF2F45100A808F0C6FC00A8FFF7B2
:105D2000A5FE024600A9381D08F0D8FC6D1C05EB45
:105D3000C500C600305900280BD0371900A9FFF75D
:105D4000A8FF0028E4D0402200A9381D08F0C6FCB6
:105D5000ECE711B0F0BDF8B507460C461546002635
:105D600030460090002F1ED0002C09D1F2BD06EB6A
:105D7000C600C00057F8041B490849004151761C71
:105D80000C2E0FD200A93846FFF75CFF002807D180
:105D90003868FFF74EFF002802D13F1DBC42F1D208
:105DA000BC42E4D23046F2BD70B5DFF888140A4632
:105DB0000B68D21A1368DFF88044A34201D0002098
:105DC00070BDDFF86C44121D22650968091F482266
:105DD000B1FBF2F1616510F1030F02D010F1130F66
:105DE0000AD1DFF85854A86808F0AEFC0646A86847
:105DF00008F0B6FC811905E008F0C0FC054608F083
:105E0000BFFC4119DFF83854A069286005F1480249
:105E1000A06AFFF7A0FF2846FFF775FF012070BDBD
:105E20000EB430B5CCB0044600A84FF49671FFF71D
:105E3000F7FD00254FAB22464FF4967100A8FFF7FF
:105E4000F7FD00A8FFF712FE044609E0DFF8E013B3
:105E5000C86D421CCA6500A9695C08F0F9FC6D1C9C
:105E6000A542F3D34CB030BC5DF810FB38B500242C
:105E7000DFF8BC53E8650FF29840FFF7D1FFDFF879
:105E8000C40301680FF2AC40FFF7CAFFA86C009092
:105E9000AB6B6A6B296B0FF2B440FFF7C1FFE96C83
:105EA0000FF2E040FFF7BCFF6A69A9690FF2E84012
:105EB000FFF7B6FF0FF2F840FFF7B2FF06E0101849
:105EC000021D0FF20450FFF7ABFF641C04EBC4008B
:105ED000C200DB4811580029F1D10FF2F840FFF75A
:105EE0009FFFA86D441E002505E00918BBA0FFF721
:105EF00097FF641E6D1C3C2D09D2002C00D53B245D
:105F0000322000FB04F1D0480A5C002AEDD131BDFB
:105F1000CE48CF490A6802604A6842608A68826057
:105F2000CA68C2600A6902614A6942610A7E826186
:105F3000097F8161C7490A7882614A6842628A683A
:105F40008262CA68C2620A6902634A6942638A69F4
:105F50008263CA69C2638A6EC0F88820BE4A9369A8
:105F6000C0F89830D368C0F88C301369C0F890300E
:105F70005369C0F894300B6FC0F89C304B6FC0F879
:105F8000A0308B6FC0F8A430C96FC0F8A810B34917
:105F90000968C0F8AC10B2490B68C0F8CC304B6847
:105FA000C0F8D0308B68C0F8D430CB68C0F8D83097
:105FB0000969C0F8DC105168C0F8E8101168C0F831
:105FC000E410704770B506460C46994D6FF01E01FF
:105FD000401A14D0083812D0001F05D0001F0ED070
:105FE00008380CD0001F10D104F120002862EFF314
:105FF000148040F00200E862286AA86205E004F11B
:1060000020002862EFF31480E862EFF308806862F2
:10601000EFF305802863EFF300806863FFF7C6FDA8
:10602000A863EFF31080E863EFF311802864EFF3C7
:1060300013806864F1EE100AA864EE64002004E0A6
:1060400054F8201045F82010401C0828F8D370BDE3
:1060500070B5774CA16D3C2901D30021A165A56DD8
:106060003221794A01FB05260A4601463046FDF7F2
:106070009EFD002086F83100681CA06570BD70B5DB
:10608000014674462046FFF79DFFFFF741FF20467B
:10609000FFF78AFE00F09AF8002832D100F034F8B9
:1060A00008F076FBF32008F0EDFB6E484FF000544B
:1060B000002505E02178641C08F0CAFB30466D1C01
:1060C000461CB5F5C03FF5D3532108F0C1FB522162
:1060D000304608F0BDFB741C4121204608F0B8FB97
:1060E000641C4D21204608F0B3FB5F48C046C04603
:1060F00004F10D00FFF7BAFE08F053FB5B4800F017
:106100001FF8BDE8704054E510B508F041FBF320DE
:1061100008F0B8FB564C3820206002E020680830B8
:1061200020602068402807D2002108F040FB0928A1
:10613000F4D0FFF73EFDFCE7BDE8104008F031BBAE
:1061400038B5044608F024FBF32008F09BFB3D48DB
:106150000168204608F060FB241DFF21204608F05E
:1061600077FB641C404D6979204608F071FB641C84
:10617000E978204608F06CFB641C2979204608F079
:1061800067FB641C2978204608F062FB641C697870
:10619000204608F05DFB641CA978204608F058FBF7
:1061A000F521601C08F054FBBDE8314008F0F9BA55
:1061B00080B508F0EDFAF32008F064FBAA212D4821
:1061C00008F046FBBDE8014008F0EBBA0020294981
:1061D0000978F52900D101207047000025730A00D5
:1061E00010B50446FFF742FCC0B2142800DB1320B0
:1061F000024621462048FDF7DAFC4FF0AC3000782B
:1062000010BD80B500F049F8BDE80140D1E480B58B
:10621000FFF7CEFF4FF4C83212490020BDE8084016
:1062200001F045BC0CED00E00400FA056C8600208E
:10623000C0430120FC4F0508FECAFECACC860020E0
:10624000140B012000880020E4D2002074320120C9
:1062500000ED00E020ED00E004E000E0A0ED00E053
:1062600034EF00E00000060864520120F4FF070844
:10627000E8520120FFFF0708CC4F012010B500F0C5
:106280001BF80FF270142046FFF7F0FB0246214680
:106290000020BDE8104001F00ABC80B501214FF498
:1062A000802002F05AFF012003F026FB94210F20EA
:1062B000BDE8044003F0C3BC80B501214FF4802049
:1062C00002F04BFF012003F017FB00210F20BDE877
:1062D000044003F0B4BC10B5002401214FF4802029
:1062E00002F03BFF012003F007FB0F2003F0B4FC9A
:1062F000942800D10124204610BD00004E6F205389
:10630000796D626F6C0000003078253038780000BD
:106310000A0A0A0A3D3D2043726173682044756D84
:106320007020496E666F726D6174696F6E203D3DBD
:106330000A0000004669726D7761726520566572C9
:1063400073696F6E203A2025640A00000A49505391
:1063500052203D20307825782C2041505352203D4A
:1063600020307825782C2078505352203D203078EA
:1063700025782C205046534352203D2030782578F4
:106380000A0000000A6661756C74206D6F646520F8
:106390003D203078257800000A5043203D20307899
:1063A00025782C204C52203D20307825780A00009A
:1063B0000A3C43726173682043616C6C20537461C2
:1063C000636B3E0A0000000030782578202025739A
:1063D0000A0000000A0A3D3D20526563656E742084
:1063E0004C6F67204D65737361676573203D3D0A8F
:1063F00000000000534E414D590000000000000015
:1064000038B5FFF7BCFBDFF830068468DFF82806F4
:1064100000210171FFF7ADFB002C2CD02068002873
:1064200029D0607C2168497CC0B2814223D1256893
:1064300000E00D002968002903D04A7CC0B28242E6
:10644000F7D0FFF79CFBDFF8F0050069A04203D10D
:10645000DFF8E40521680161E06921680160C86135
:10646000E56129682160002900D0CC612C6095F895
:10647000410085F84000FFF77CFB31BD10B5FFF708
:106480007EFBDFF8B8050468DFF8AC05006A201A67
:10649000012832DADFF8A005046A04E0DFF8980585
:1064A0000462FFF766FBDFF898050078C00722D585
:1064B000FFF765FBDFF8880500788007EED5DFF889
:1064C0008005007810F0FD00DFF874150870FFF704
:1064D00050FBDFF86405006A8442FAD0DFF8580503
:1064E0000462DFF858050068401CDFF850150860AA
:1064F000DFF844154862FFF742FB10BD38B50400D1
:106500000020A071206A10F57A606062E0690028BE
:1065100002D02000E1698847FFF72BFBE56809E01E
:10652000E868616A401A002801D5E8686062FFF7F0
:1065300020FB2D68002D1AD0FFF721FB20690028D1
:1065400004D0687C2169497C884212D3287C4007AA
:10655000EDD5E868216A401A0128E1DA280000F048
:106560009EF9FFF70CFB287C0028D9D101E0FFF74A
:1065700006FB31BD70B50400002060700120207062
:1065800008F0FCF80078C0B2CD2802D07D20FFF7DB
:1065900089FAA06800280CD0A068406C002808D0B8
:1065A000A068406C01680800002802D0A06840681C
:1065B000884794F8290000280BD0A06894F8281088
:1065C00080F84010DFF870040079002801D0FFF750
:1065D00017FFDFF870040078002823D0DFF8680484
:1065E0000068DFF85414096A401A002804D5DFF85F
:1065F00054040021017015E0FFF7C1FA08F006FA13
:106600000500FFF7B6FAA068002808D0A068406B24
:106610002818DFF838140968401AA1684863DFF8C1
:106620002C040560A068002808D0A068007C002821
:1066300004D1A068006B401CA16808632069002891
:106640002BD003E030682061FFF793FAFFF797FA49
:106650002669002E27D0357CEDB2002D23D06807A7
:1066600010D5F068216A411A012906DA300000F0DD
:1066700016F9307C002805D10FE0616A411A002923
:1066800000D56062EDB215F0FB001028DAD1B068D9
:1066900080684068007C0028D4D1FFF770FA02E0DF
:1066A0002000FFF72BFFA0790028F9D1DFF8900335
:1066B0000078C00701D5FFF7E1FE00206071206976
:1066C000002839D02069007C002805D02069806826
:1066D00080684068A06001E02069A060A06890F830
:1066E0004C00642802D08020FFF7DCF9A068806AA3
:1066F0000078CD2802D07820FFF7D4F9A068406C4C
:10670000002808D0A068406C41680800002802D02A
:10671000A06840688847A06890F8400084F8280086
:1067200084F82900DFF810038068C06A401CDFF895
:1067300008138968C8620BE0002084F82900002053
:1067400084F828000020A06000202070FFF711FAD4
:10675000200070BD80B508F087F9DFF8F4120978E1
:10676000002806D0022810D009D3042815D010D351
:1067700014E0002902D0A320FFF794F911E00029CA
:1067800002D1A420FFF78EF90BE0A620FFF78AF9CB
:1067900007E0A720FFF786F903E002E0A820FFF753
:1067A00081F901BD10B508F05FF90400DFF8A0021F
:1067B0000078002802D0A020FFF774F9002C05D043
:1067C000022C08D003D3032C09D00CE00EE0A42047
:1067D000FFF768F90AE0A620FFF764F906E0A720B2
:1067E000FFF760F902E0A820FFF75CF910BD80B563
:1067F00008F03AF9002805D0022808D006D303286B
:1068000009D00CE0A320FFF74DF90BE00AE0A62029
:10681000FFF748F906E0A720FFF744F902E0A820B7
:10682000FFF740F901BD80B5DFF80C0200780028C1
:1068300002D19720FFF736F9DFF8FC010078401EFF
:10684000DFF8F4110870C0B2002827D1DFF8E801A2
:106850004068002822D0FFF792F9DFF8DC01406899
:1068600000280BD0DFF8D00101210170DFF8C8014A
:10687000FFF76FF9DFF8C00100210170DFF8B80100
:106880004078F021084202D09920FFF70BF9DFF899
:10689000A8014078002801D1FFF76BF901BD10B5C0
:1068A000816800290CD0DFF89011096AC160816805
:1068B0000A684968002A00D051600A60002181609E
:1068C000017C11F003010174C9B2002945D1DFF840
:1068D00068110969002929D1DFF85C110861DFF826
:1068E0005801007800280CD1DFF84C01012101701B
:1068F000DFF84401FFF72DF9DFF83C0100210170BA
:1069000003E0DFF8340101214171DFF82C01407808
:10691000F021084202D09920FFF7C4F8DFF81801EF
:106920004078002801D1FFF724F916E0427C4B7C27
:10693000D2B29342D0D38142D1D04B7CD2B29A42D0
:106940000BD10300FFE71B68002BDED05C7CD2B2CA
:10695000A242DAD18B42F6D1BEE710BD10B50400D9
:10696000627C35480078401C33490870394800E0A3
:1069700008000168002903D04B7CD2B29A42F7D3B9
:106980002160E061046000290AD0CC61487CD2B269
:10699000904202D194F8410000E0002084F84000C9
:1069A000207C002812D1FFF7EAF82000FFF777FFDC
:1069B00021484078F021084202D09920FFF772F870
:1069C0001D484078002801D1FFF7D3F8FFF72BFFCF
:1069D00010BD10B51848047817480078401C1649B7
:1069E00008701548FFF7B5F813480470124840784E
:1069F000F021084202D09920FFF754F80E48407861
:106A0000002801D1FFF7B5F810BD10B508F032F835
:106A100009480121017007F0B1FE04006846C04634
:106A2000021B203A012A03DBCD212000FCF7A0FC49
:106A300009480121017010BDCC8600203C53012083
:106A40008F530120905301205453012040530120C3
:106A500091530120D886002093530120DFF8C0060F
:106A6000007870472DE9F0418AB0FBF709FF044632
:106A7000DFF8B0562E6842E096F9080007283DD0AE
:106A80000B283BDA062839D006F10807B86C002835
:106A900003D5D4F880100818B8644FF0FF313046A1
:106AA000FA6D926990478046B8F1010F04D197F8CA
:106AB0004C00B96D09698847B8F1020F0BD1797E96
:106AC00038697A688018BA6D52699047002802D0F8
:106AD000304608F0A3F800213046FA6D92699047DD
:106AE000022801D10120B87501213046FA6D926962
:106AF0009047022802D1304608F03CF93668AE4291
:106B0000BAD1D4E91C01002901D100280CD00A20F7
:106B10008DF8080002208DF80000D4F88000ADF850
:106B2000220000A801F0E8FF01200AB0BDE8F081D2
:106B300030B585B004460D46CA208DF8000028887F
:106B4000ADF801000220ADF80300BDF80100001D02
:106B500003F00EFBCDF8090002220DF10301FDF751
:106B600026F802222946DDF80900801CFDF71FF8EF
:106B70002A882146DDF80900001DFDF718F80020DD
:106B8000288000A9DFF8F40D08F016FC05B030BD30
:106B900042F23411081A322801DA0120704700202D
:106BA000704780B5FBF7A5FA407B002804D007F0BA
:106BB0008DFFDFF8A41E086001BD80B507F086FFD9
:106BC000DFF8981E086001BDDFF8900E006870477E
:106BD00010B582B000F10C03D96A896800910422D3
:106BE00000A95C7DDB68C06818182018FCF7DFFF7F
:106BF00013BD30B41488651C1580052565541488B0
:106C0000651C1580635413885C1C1480007A5854EA
:106C100030BC704732B515461C4621884A1C22807C
:106C200037224A5521884A1C2280007A4855022280
:106C300000A920884019FCF7BAFF2088801C20801A
:106C400031BDF8B517461D4600F10C06069CA4B2EE
:106C5000B27D6243C06809182888C019FCF7A7FFF5
:106C60002888B17D614311FA80F02880F1BD30B4ED
:106C700000F110039B7C914203D1006990FBF3F07B
:106C80000DE00C46154603D2281B90FBF3F006E0FE
:106C90000069001B90FBF3F095FBF3F1081880B23C
:106CA00030BC704700F110018A688B7CD2188A6072
:106CB0000069824201D100208860002088737047FB
:106CC00070B582B004460D461E4692B289B2FFF7F7
:106CD000CEFF0090069B324629462046FFF7B1FFC3
:106CE00073BDF8B5044615461E462269002D00D135
:106CF0001546069F0097FFF7E3FF2069854206DAF5
:106D0000009733462A4600212046FFF7D9FFF1BD00
:106D10002DE9FC4104460D461646A169606900282C
:106D200015D500270A4692B289B22046FFF79FFF89
:106D3000804633462A4641462046FFF76BFFA2694C
:106D400000962B4611462046FFF7CBFF2EE08142EE
:106D500016DA01270A4692B2014689B22046FFF7A9
:106D600086FF804633462A4641462046FFF752FFBB
:106D700000962B46A26961692046FFF7B2FF15E035
:106D800002270A4692B2014689B22046FFF76FFFFA
:106D9000804633462A4641462046FFF73BFF009691
:106DA0002B46A26961692046FFF78AFFA06901901E
:106DB000606900903B46424694F908100FF20800C3
:106DC000FBF719FABDE8F3815061636B203D256440
:106DD000202564202564202564202564000000000F
:106DE00070B582B004460D461646A06C012811DA33
:106DF000A07F012811D133462A4601212046FFF702
:106E000009FF0120009033462A46A1692046FFF77A
:106E100018FF02E02046FFF77BFF01233246294698
:106E20002046FFF7E6FEA0696061A36CE26C94F96E
:106E300008100FF20C00FBF7DEF9A06CE06473BDE4
:106E4000666C757368202564202564202564000025
:106E50002DE9F84304460D461646FBF711FD814621
:106E6000FBF747F9804604F10807B87D002802D0F7
:106E70002046FFF7ADFE386C0128C0F28E8098F8EE
:106E80000E00002844D0B87D002800F0CA80786C3D
:106E9000D9F88010401A7864B87E3969FA68531AB4
:106EA000834205D0002A2FD1BA68511A81422BD1D2
:106EB00094F90820397E0FF27010FBF79CF9397EA7
:106EC00000291ED094F908200FF27410FBF793F9F3
:106ED0003869B97E421892B2F96889B22046FFF744
:106EE000C6FE33462A4601462046FFF793FE00962B
:106EF0002B463869B97E4218F9682046FFF7F1FE43
:106F000002E04FF0FF30F8602046BDE8F243C9E6EA
:106F100098F80E00002840F08480786CD9F8801032
:106F2000401A7864012831DA386C7864386BD0F80C
:106F30000C8094F908308268396C0FF22010FBF74E
:106F40005AF9B868B97E90FBF1F0396C91FBF8F111
:106F5000814202DB4FF0FF30F860B86CB97D002948
:106F60000CD0002807D42046FFF79CFE3246294665
:106F70002046FFF7CDFE3869F86052E0002850D473
:106F8000324629462046BDE8F843C1E6B87D0028D0
:106F900047D02046BDE8F24384E6B87D002840D0C3
:106FA00094F9080098F80A1000291BD0072803D08C
:106FB0000D2801D015282FD133462A46012120461D
:106FC000FFF728FE0120009033462A463969204603
:106FD000FFF737FE7A7894F908100FF29400FBF768
:106FE0000AF919E0092809D194F85E10012905D1A0
:106FF0000FF28C00BDE8F443FBF7FDB833462A4698
:1070000001212046FFF706FE0120009033462A4664
:1070100039692046FFF715FE2046FFF743FE386921
:10702000F860BDE8F183000073757370656E6420CD
:107030006669666F2066756C6C2025642025640087
:1070400073757370656E64206669666F2066756C13
:107050006C20322025642025640000006669666F7C
:107060002066756C6C33202564202564202564001F
:1070700041502053757320256420256400000000D2
:10708000233E6C75785F73617420256400000000F6
:10709000F8B504460D46234E376805E02A462146DA
:1070A0003846FFF7D5FE3F68B742F7D1F1BD2DE96D
:1070B000F04104460D46DFF82C6DF76907F10C0826
:1070C00098F81510D8F80C00FA688018D8F85420F1
:1070D0005269904700280AD0012088F81200787A77
:1070E000002804D02A4621463846FFF7B1FEB6698B
:1070F00006F10C07797DF868F26880187A6D52699C
:107100009047002809D00120B874707A002804D074
:107110002A4621463046FFF79BFE0120BDE8F0815C
:107120008B530120746900200288D21C02800A80DF
:10713000704780B50B889B1AADF80030BDF8003061
:10714000002B09D01018012100F8031C022200A90D
:10715000801EFCF72CFD01BD0888C01E088001BD03
:107160002DE9F04FADF68C2D04460D46FBF788FB5C
:107170000746FAF7BEFF804610A840F64821FEF702
:107180004FFC00208DF8020006A82821FEF748FCDD
:1071900001A81421FEF744FC0020ADF800000646CB
:1071A000D7E91C01002902D1002800F0E38398F9F7
:1071B000090008F01DFE002800F0DC8300A9284625
:1071C000FFF7B2FFB0461CE0D7E91C01424609F0C8
:1071D0003DF800F0010011F0000101D100280ED0AF
:1071E00008EB8800DFF8001C01EBC00292F90900EF
:1071F000012804D10DF1020110A8126A904708F18C
:107200000108B8F12D0FDFDB37461AE02888411C52
:10721000298099F8021001552888FFF7B9FC002849
:107220000DD0BDF8002029462046FFF782FF2946F1
:107230002046FFF77DFC00A92846FFF775FF7F1C5D
:107240007FB29DF80200874280F28C832988481C17
:10725000288040F2491010FB07F010AA825C0A5502
:1072600029884A1C2A8010AA00EB020898F801001D
:1072700008552888411C298008F1010999F8011056
:10728000015599F80100032821D0092800F04C810C
:107290000C2800F026811A2800F04A821B2800F0F2
:1072A00059811C2800F078821D2800F066811E2874
:1072B00000F06282252800F0A182262800F0DB82FF
:1072C000282800F0B6822C2800F0E5829EE798F886
:1072D0000100032805D12888411C298099F8021053
:1072E00001552888411C298099F80310015599F807
:1072F0000300C0280DD1B8F83020D8F83210288803
:107300000019FCF754FC2888B8F8301008182880B9
:1073100082E7711C00064ED401A808F104025278DD
:107320003254C9B298F806200A54491CC9B2002246
:107330000A544A1C08F20601D2B24B781354521C6C
:10734000B8F80E30D2B21E0A1654521CD2B21354E0
:10735000521C08F20E03D2B29E781654521CD2B2BE
:10736000DB781354521CD2B298F812301354521CCA
:10737000D2B298F813301354521CD2B28B781354F3
:10738000521CD2B2C9781154511CC9B298F80A20C3
:107390000A54491CC9B298F80B200A544E1CF6B284
:1073A000324601A928880019FCF701FC288850FA08
:1073B00086F0288030E7D8F8052006A8130C33544F
:1073C000C9B2130A0B54491CC9B20A54491CD8F853
:1073D0000920C9B2130C0B54491CC9B2130A0B542F
:1073E000491CC9B20A54491CD8F80D20C9B2130C63
:1073F0000B54491CC9B2130A0B54491CC9B20A5494
:10740000491CD8F81120C9B2130C0B54491CC9B23D
:10741000130A0B54491CC9B20A54491CD8F8272036
:10742000C9B2130C0B54491CC9B2130A0B54491CA2
:10743000C9B20A544A1C08F22701D2B20B7913547C
:10744000521CD2B24B791354521CCB88D2B21E0AB2
:107450001654521CD2B21354521CD2B2097A11548F
:10746000511CD8F81520C9B2130C0B54491CC9B2D1
:10747000130A0B54491CC9B20A54491CD8F81920E4
:10748000C9B2130C0B54491CC9B2130A0B54491C42
:10749000C9B20A54491CD8F81D20C9B2130C0B54A8
:1074A000491CC9B2130A0B54491CC9B20A54491CDD
:1074B000D8F82120C9B2130C0B54491CC9B2130AC5
:1074C0000B54491CC9B20A544E1CF6B2324606A9E6
:1074D00028880019FCF76BFB288850FA86F0288072
:1074E0009AE608F10301B1F90300C0F3072242EA6A
:1074F0000020A1F80300B1F90700C0F3072242EA17
:107500000020A1F80700B1F90500C0F3072242EA04
:107510000020A1F80500092228880019FCF747FB84
:1075200028880930288077E62988084698F80120BD
:10753000032A09D1022208F103010019FCF737FBE5
:107540002888801C288067E6491C298099F8021049
:10755000015561E62888411C298099F802100155DF
:1075600098F8010005287FF457AE2888411C29802F
:1075700008F10401497801554EE608F1030998F82D
:107580000100012840F0C4802888411C298099F816
:10759000041001554FF0000AA1E0CAEB4A1000EBBD
:1075A000090BDBF81800010221F0FF11000A00F0BE
:1075B000FF100843CBF818004FEA3040CBF8180012
:1075C00004220BF1180128880019FCF7F0FA28882A
:1075D000001D2880DBF80800010221F0FF110012D5
:1075E00000F0FF100843CBF80800C0F30F4141EA58
:1075F0000040CBF8080004220BF10801288800198C
:10760000FCF7D5FA2888001D2880DBF80C00010261
:1076100021F0FF11001200F0FF100843CBF80C001E
:10762000C0F30F4141EA0040CBF80C0004220BF1FB
:107630000C0128880019FCF7BAFA2888001D288058
:10764000DBF81000010221F0FF11001200F0FF1022
:107650000843CBF81000C0F30F4141EA0040CBF8DB
:10766000100004220BF1100128880019FCF79FFA82
:107670002888001D2880DBF81C00010221F0FF1182
:10768000000A00F0FF100843CBF81C004FEA30401E
:10769000CBF81C0004220BF11C0128880019FCF710
:1076A00086FA2888001D2880BBF81600010A41EAE6
:1076B0000020ABF8160002220BF1160128880019F1
:1076C000FCF775FA2888801C2880411C298080B22C
:1076D000DBF8201001550AF1010A5FFA8AFA99F8DD
:1076E00004008245FFF659AFB8F84321D8F8451198
:1076F00028880019FCF75BFA2888B8F843110818A5
:107700002880B8F843110FF27820FAF774FD83E56A
:1077100005287FF481AD2888411C298099F8021042
:1077200001552888411C298099F80310015573E5FB
:1077300008F1030198F80100032805D12888421CAC
:107740002A8098F80A200255D1F80100020222F09E
:10775000FF12000A00F0FF101043C1F801004FEAC9
:107760003040C1F80100072228880019FCF71FFAF1
:107770002888C01D28804FE508F103010888020A07
:1077800042EA00200880022228880019FCF70FFA3C
:107790002888801C28803FE508F1030098F8011034
:1077A00001297FF439AD99F80210012918D12988EF
:1077B0004A1C2A8000780855B8F80420D8F806102A
:1077C00028880019FCF7F3F92888B8F8041008187D
:1077D0002880B8F804100FF2BC10FAF70CFD1BE576
:1077E00002297FF419AD29884A1C2A8002780A559B
:1077F00029884A1C2A80C07908550DE52888411C33
:107800002980B9F8021001552888411C2980B9F94E
:10781000021009120155B9F90220D8F8051028887C
:107820000019FCF7C4F92888B9F902100818288053
:10783000F2E42888411C2980B9F8021001552888F3
:10784000411C2980B9F90210091201552888411CF0
:10785000298008F1040149780155B9F90220D8F8C6
:10786000061028880019FCF7A2F92888B9F9021037
:1078700008182880D0E408F103010888020A42EAC7
:1078800000200880022228880019FCF790F9288837
:10789000801C2880C0E408F103082988084698F86D
:1078A000002013072AD5491C298098F8001001559B
:1078B0002888411C298098F8071001552888411C08
:1078C000298098F808100155D8F80900010221F024
:1078D000FF11000A00F0FF100843C8F809004FEA42
:1078E0003040C8F80900042208F10901288800196D
:1078F000FCF75DF92888001D28808DE4520724D507
:10790000491C298098F8001001552888411C2980BD
:1079100098F801100155D8F80300010221F0FF1179
:10792000000A00F0FF100843C8F803004FEA304097
:10793000C8F80300042208F1030128880019FCF7A5
:1079400036F92888001D288066E498F80220D8F8C7
:107950000D100019FCF72BF9288898F80210401830
:10796000288059E4BDF8002029462046FFF7E1FBB6
:1079700008F06CFA0DF68C2DBDE8F08F3C8A0020E3
:107980004F4A483A20415442442073697A653A206C
:10799000256400004F4A483A204150445220736900
:1079A0007A653A20256400002DE9F04105460E462F
:1079B000FAF79FFB0746DFF834442078401C20701C
:1079C0006078F021084202D09920FEF76BF8FEF7AC
:1079D000D6F86078401C607097F81880B8F1000FF6
:1079E00026D03088404480B2FFF7D2F8002803D078
:1079F00031462846FFF79CF83088411C318003212E
:107A000041553088411C318000F80580424607F11D
:107A1000190130884019FCF7CAF83088404430809A
:107A2000FF22002107F11900FBF7A2FC00203876A5
:107A30006078F021084202D09920FEF733F8607890
:107A4000401E6070C0B2002801D1FEF792F8BDE878
:107A5000F041FEF7E8BE0000185301201C5301203E
:107A600038B504460D46FAF744FB817A002909D15E
:107A7000417B002906D129884A1C2A8006220A5502
:107A80000121417331BD38B504460D4628880028D0
:107A90000CD02046FFF788FF29462046FFF7E0FF7D
:107AA00029462046BDE83440FFF742B831BD14B541
:107AB00085B0049101A90022134614461CC10A2175
:107AC000ADF8001004218DF804108DF805000A4669
:107AD00005A90DF10600FCF76AF8042204A90DF1CE
:107AE0000A00FCF764F800A901A8FFF721F806B026
:107AF00010BD80B5FAF7FDFA4FF49671FAF7E6FC7F
:107B000007208DF802000120ADF8000000A90DF15A
:107B10000200FFF70DF801BD2DE9F041DFF8804DBF
:107B20006068002828D0218888421FD002F020FBFE
:107B3000054666682788A6EB07081FFA88F84246BC
:107B4000381900F108012846FCF731F83A4604F1EB
:107B5000080108EB0500FCF72AF83246294604F133
:107B60000800FCF724F8284602F01AFB626804F1CA
:107B700008010520FFF79BFF002060602080BDE822
:107B8000F08180B5FAF77CFE062180F884108430FD
:107B9000417007218170C170017101BD2DE9FC4167
:107BA00005460F469046FAF7A4FA0026D5F80910C4
:107BB0000C1D2A781146012962D00F2933D03529AE
:107BC00037D0802900F08880812900F08F808229B9
:107BD00000F08C80852900F08980862900F086805D
:107BE000882900F083808A2900F088808B2900F0A2
:107BF000A1808C2900F0AD808D2900F0B580DD29B1
:107C000000F0BF80DF2900F0D980F0291AD0F429D4
:107C100023D0F62929D0F82947D0F92935D0FF29D2
:107C200000F0A7805FE0807D2070FFF7AAFF0120B1
:107C30005AE00120FAF7D1F83046FAF7D2F80120DD
:107C4000207051E00422DFF85C1C2046FBF7AFFFF8
:107C50000120FDF739F8012046E0042200F110016F
:107C60002046FBF7A4FF01203EE0032221463046D8
:107C7000DFF8343C9B681B6E1B6A9847012033E099
:107C8000204608F011FB01202EE0B5F80120B5F8E0
:107C90000300C010C0EB0011D5F8050000EB811106
:107CA0002046FBF784FF01201EE03046ADF80400BB
:107CB00001206979012900D10320FCF76EFAFCF755
:107CC000A8FAADF80400FCF7BBFA022201A920468D
:107CD000FBF76DFF012007E0D5F805002070214675
:107CE000304607F0F5F83046BDE8F68130462070A2
:107CF000214602F07F0007F0EBF8F4E70120207046
:107D0000DFF8A40B45683746287F002801D13046AC
:107D1000EAE7687A002803D1286E40688047074662
:107D20002046296EC9698847002FDCD0286E8068FC
:107D30008047D8E70120B5F80310C1F3C101091D40
:107D4000884040F0020020702146012007F0C0F872
:107D5000C9E701782170C17861704179A17080799B
:107D6000E07001202071BFE7204608F0B1FA064616
:107D7000B9E704F10802211D2046FDF753F8012060
:107D8000B2E76879DFF8201B51F82050687A0028A4
:107D900010D0424639462846FFF722F8DFF80C0B90
:107DA00001210170DFF8081B082008F053FB0120B7
:107DB000207001E030462070012095E76879DFF8F7
:107DC000E81A51F82050286995F8221090FBF1F03C
:107DD000401E0090042200A92046FBF7E8FE012087
:107DE00082E70000086000209CDE0020CC86002096
:107DF000F0B593B00646FAF77CF90546FAF740FD70
:107E0000D6F809100C1D3178002208924FF0FF328D
:107E1000099217460A46312A00F01E81322A00F0E4
:107E20002581332A00F03181342A00F03881372A45
:107E300074D0A12A00F06081A22A00F07F81A42AD8
:107E400000F08A81B12A00F02F83B22A00F0CB849F
:107E5000B82A00F09C81C12A00F0CA81CD2A00F026
:107E60008B80CE2A00F0A180D02A37D0D12A2BD007
:107E7000D22A38D0D32A3FD0D42A41D0D62A58D0BB
:107E8000D72A56D0D82A5CD0D92A5AD0DB2A00F07B
:107E90001E81DC2A00F02281F12A5AD0F22A00F059
:107EA0009D80F52A00F0B180F72A00F0C480FA2AFC
:107EB00000F0D984FB2A00F0D984FD2A00F0B080BC
:107EC000FE2A00F0E384C4E000212846FAF73CFBD8
:107ED0000020A873FFF720FE0120BBE00020FCF784
:107EE000F3FE0120B6E001212846FAF72DFB012020
:107EF00008F000FB0120ADE00020A8720120A9E0FD
:107F00000120A872002068730120A873E87A002875
:107F100002D1012008F0EEFA01209BE00022214668
:107F20001046DFF884391B681B6E1B6A98470120D6
:107F300090E0D62901D1012000E00020E872012064
:107F400088E0D92901D1012000E000202873012018
:107F500080E000210CE00A180B5D82F884300229D1
:107F600005D10A5D80F887200A5D80F88820491CC9
:107F70000329F0DB01206DE0002512E0DFF828097D
:107F8000466806EB4506022204EB450106F158005F
:107F9000FBF70DFEB6F95810DFF81809FAF72BF9C0
:107FA0006D1C032DEADB012054E0002512E0DFF810
:107FB000F808066806EB4506022204EB450106F1C7
:107FC0005800FBF7F4FDB6F95810DFF8EC08FAF7A3
:107FD00012F96D1C032DEADB01203BE0297C090628
:107FE00001D4012036E02178A0F88A106178A0F849
:107FF0008C1002212046DFF8B028D269126E9269F7
:108000009047002825D0012024E0032221460120AA
:10801000DFF894389B681B6E1B6A9847012019E0B3
:108020001B2221460720DFF880389B681B6E1B6AE5
:10803000984701200EE0DFF870088669306E80688E
:108040008047002805D0012221460520336E1B6A97
:108050009847002013B0F0BDF9F7C7FE012801D101
:108060000120F7E72046F9F7EBFDF2E7F9F7BDFE4F
:10807000012801D10120EDE72046F9F766FE2078BE
:108080000028E6D0F9F792FEE3E7F9F7AEFE012803
:1080900001D10120DEE72078F9F78FFED9E7F9F763
:1080A000A4FE012801D10120D4E74FF48051002023
:1080B000FAF783FA0120F9F713FD0120F9F791FE91
:1080C0002078F9F79BFEF9F780FD0120C2E7D6F88A
:1080D0000510DFF8E807FAF78EF8BAE7FEF776F84A
:1080E000002802D0FEF793F8B3E7FEF7F4F8002873
:1080F000AFD0FEF7C3F8ACE794F900500422611C3E
:1081000008A8FBF754FDB6F80100062806DB042298
:10811000611D09A8FBF74BFD94F90970042D04D1EA
:10812000DFF884070069A17A81720097099B002219
:108130000899284606F03AFF20708AE794F9005023
:108140000422611C08A8FBF732FD00231A46089997
:10815000284606F09BFF7DE794F900500422611C3D
:1081600008A8FBF724FDB6F80100062806DB042268
:10817000611D09A8FBF71BFD94F909700097099B85
:1081800000220899284606F0DEFF207061E720787B
:108190000146032908D01A2913D0252915D02829EA
:1081A00017D02C2919D01CE060788DF80A0001281E
:1081B00005D1A0788DF80B00204600F039FC012095
:1081C00048E7204600F034FCF9E7204600F030FC98
:1081D000F5E7204600F02CFCF1E7204600F028FCF3
:1081E000EDE794F9011040B207F0D2FEC0B231E7DA
:1081F000207801460E3908D0091F03291CD9091F10
:1082000037D0491E00F0958038E10E208DF8080027
:1082100060788DF80A00A1788DF80B10E2788DF85F
:108220000C200023ADF80D3052B249B240B2FAF73B
:10823000DCF900F0F4FB21E18DF80800122802D1EE
:1082400061788DF80A10132802D161788DF80B102F
:10825000142802D161788DF80C10152802D16078AD
:108260008DF80A0062782178DFF85406F9F7C3FF29
:1082700004E16078A178090401EB0060E17800EB8B
:10828000012021794018CDF80A006179A279120401
:1082900002EB0161E27901EB0221227A8918CDF823
:1082A0000E10627AA37A1B0403EB0262E37A02EBFC
:1082B0000322237BD218CDF81220637B8DF8163071
:1082C000A37B8DF81730E37B8DF81830237C8DF875
:1082D0001930637C8DF81A30A37CE57C15EB032301
:1082E0001BB21D46ADF81B50257D03EB0523657DB4
:1082F0005B19ADF81D30A37D8DF81F30002803D128
:10830000002901D1002A09D00DF10A0184B0684684
:108310001622FBF711FC0FBCFAF70EFA0DF10A0159
:1083200084B068461622FBF707FC0FBC00F0BFFBC9
:10833000A4E060788DF809001D283ED1A0788DF862
:108340001300A07801280ED1E078217911EB0021EB
:10835000ADF80A1089B20A469DF80910DFF86405E5
:10836000F9F749FF8AE002280BD1E078217911EB77
:108370000021ADF80C1089B2DFF84C05F9F73BFF8E
:108380007CE003280BD1E078217911EB0021ADF8D6
:10839000141089B2DFF83405F9F72DFF6EE00428D8
:1083A0006CD1E078217911EB0021ADF8161089B27B
:1083B000DFF81C05F9F71FFF60E0262809D1A07837
:1083C0008DF80E00A078012858D1E0788DF80D00C6
:1083D00054E01C2823D1A0788DF80D00A078012846
:1083E00007D1E1788DF80A10DFF8E804F9F703FF08
:1083F00044E0022807D1E1788DF80B10DFF8D804AB
:10840000F9F7F9FE3AE0032838D0052836D1E178AB
:108410008DF80C10DFF8C404F9F7EDFE2EE02C28DF
:108420002CD1A0788DF81400A078012803D1E07831
:108430008DF80E0022E0022806D1E078217911EBB8
:108440000020ADF8150019E0032806D1E078217965
:1084500011EB0020ADF8170010E0042806D1E078F9
:10846000217911EB0020ADF8190007E0052805D1AE
:10847000E078217911EB0020ADF81B0006208DF883
:10848000280020780B900DF1310002A91822FBF78B
:1084900053FB0B208DF830000020ADF84A000AA8ED
:1084A00000F02AFBC0B2D5E594F9000006F0D3FF36
:1084B000012840F0698120780146032928D0062947
:1084C00065D009292BD00C2945D00D2951D0192967
:1084D00000F090801A2967D01B2900F0A0801C2989
:1084E00000F0DB801D2900F0B3801E2900F0E2803F
:1084F000252900F0FB80262900F0EA80272900F0DA
:10850000FC80282900F020812C2900F0218136E10F
:108510000322611C0DF10A00FBF749FB34E107223D
:10852000611C0DF10A00FBF742FBBDF80A00010ACD
:1085300041EA0020ADF80A00BDF80C00010A41EA4A
:108540000020ADF80C00BDF80E00010A41EA002041
:10855000ADF80E0018E10322611C0DF10A00FBF7D3
:1085600026FBBDF80B00010A41EA0020ADF80B0024
:108570000AE10322611C0DF10A00FBF718FBBDF8AC
:108580000B00010A41EA0020ADF80B00FCE00122DB
:10859000611C0DF10A00FBF70AFB9DF80A100FF2AF
:1085A0004430F9F728FEEFE00B22611C0DF10A00C0
:1085B000FBF7FDFADDF80B00010221F0FF11000AC4
:1085C00000F0FF100843CDF80B004FEA3040CDF823
:1085D0000B00BDF81000010A41EA0020ADF81000C0
:1085E00000239DF914209DF913109DF91200F9F74D
:1085F000FCFFC9E00622611C0DF10A00FBF7D7FA67
:10860000BDF80A00010A41EA0020ADF80A00BDF8F1
:108610000E00010A41EA0020ADF80E00B4E0042289
:10862000611C0DF10A00FBF7C2FABDF80A00010A4D
:1086300041EA0020ADF80A00BDF80C00010A41EA49
:108640000020ADF80C000FF2A820F9F7D4FD9BE054
:108650000922611C0DF10A00FBF7A9FABDF80A0016
:10866000010A41EA0020ADF80A00BDF80C00010A39
:1086700041EA0020ADF80C00BDF80E00010A41EA05
:108680000020ADF80E0000239DF912209DF9111075
:108690009DF91000F9F7A9FF76E060788DF80A00DF
:1086A000A0788DF80B00A27861780FF25020F9F7CE
:1086B000A2FD69E00322611C0DF10A00FBF777FAC5
:1086C000BDF80B00010A41EA0020ADF80B005BE0A9
:1086D0000522611C0DF10A00FBF769FABDF80B00D9
:1086E000010A41EA0020ADF80B004DE00922611CAF
:1086F0000DF10A00FBF75BFA46E00A22611C0DF15E
:108700000A00FBF754FABDF90A00C0F3072141EA59
:108710000020ADF80A00BDF90C00C0F3072141EAC2
:108720000020ADF80C00BDF90E00C0F3072141EAAE
:108730000020ADF80E00BDF91000C0F3072141EA9A
:108740000020ADF810001FE060788DF80A001BE0F3
:108750000822611C0DF10A00FBF729FABDF80C0094
:10876000010A41EA0020ADF80C0000239DF9112018
:108770009DF910109DF90F00F9F737FF04E08DF80F
:10878000080060788DF8090020780146052907D196
:10879000534801210170687A00280ED1084659E437
:1087A00018290AD18DF8080060788DF80900A078A2
:1087B0008DF80A00E0788DF80B0000208DF8280075
:1087C00020780B900DF1310002A91822FBF7B4F9C3
:1087D0000B208DF830000020ADF84A000AA800F008
:1087E0008BF9C0B236E42078052804D13C4800213A
:1087F000017001202EE41A281CD10822611C0DF101
:108800000A00FBF7D4F9DDF80B00010221F0FF119B
:10881000000A00F0FF100843CDF80B004FEA30408B
:10882000CDF80B00BDF81000010A41EA0020ADF8B8
:10883000100004E02C2802D160788DF80A00012095
:108840008DF8280020780B900DF1310002A9182234
:10885000FBF772F90B208DF830000AA800F04CF9F4
:10886000C0B2FFF7F7BB0120FFF7F4BB2078002868
:1088700002D0052805D006E00FF29000FDF7B0FC0D
:1088800001E0FFF749F90120FFF7E4BB04F108021A
:10889000211D2046FCF77EFA0120FFF7DBBB00001C
:1088A000A411012000880020086000208A530120C4
:1088B0008CC1002054490308604903086C4903082F
:1088C000784903088849030898490308A44903081C
:1088D000B0490308BC490308D0490308E449030828
:1088E0008B53012050443A2053432025640000005C
:1088F0004C54205353204144440000004150445202
:1089000020414444202564202564000041505F52EA
:10891000455155455354000076487047F8B50C460C
:108920001646012500282BD106EB8600714901EB84
:10893000C007F868E040C00708D52346FA6831460A
:108940000FF24030F9F757FC0220F2BD4FF0FF3034
:10895000009003462A467968204606F027FB002847
:108960000CD02346FA6831460FF22830F9F743FC61
:10897000F8682946A1400843F8602CE00220F2BDC7
:10898000012828D106EB86005A4901EBC007F86898
:10899000E040C00708D42346FA6831460FF204309D
:1089A000F9F729FC032516E04FF0FF332A467968D2
:1089B000204606F06BFB002807D02346FA683146B4
:1089C0000FF2F020F9F717FC00E00325F868012109
:1089D000A1408843F8602846F2BD07F0E5BA02B529
:1089E0008AB00021ADF8221001910A218DF80810FB
:1089F00000218DF809108DF80A1005218DF800105E
:108A0000019004220AA90DF10900FBF7D0F800201B
:108A1000ADF8220000A800F06FF80BB000BD80B5E3
:108A200008F026FB0FF29C20BDE80240F9F7E3BBFB
:108A300038B5447885780078032822D01A2802D0E7
:108A40002C282AD031BD012C0CD1012009F00EFFB9
:108A5000012322461A210FF2782001B0BDE83040F0
:108A6000F9F7C9BB022C21D1022009F0FFFE022335
:108A700022461A210FF2682001B0BDE83040F9F714
:108A8000BABB012C12D1284608F0FDFA29460FF294
:108A90006420BDE83440F9F7AEBB012C06D129466D
:108AA0000FF25C20BDE83440F9F7A5BB31BD0FB42F
:108AB00080B5002805D10846002802D110460028BC
:108AC00004D00AF020FCC046C04601E00AF004FCD5
:108AD00001BC5DF814FB00222D2809D200EB8003B5
:108AE000044800EBC300C068C840C00700D501229D
:108AF000104670479CDE002030B585B00446012545
:108B000094F90000062800F2A880DFE800F00428AD
:108B10004B667D9EA20004F1090182B068461822CE
:108B2000FBF70AF80CBC94F90810606840B206F034
:108B300039FE02280AD1606800B207F053F8002518
:108B400061680FF2C410F9F756FB8CE0032840F07F
:108B50008A8061680FF2B810F9F74DFB83E0606816
:108B60001A280BD104F1090007F0FFFA237CE26810
:108B7000E17A0FF2A410F9F73EFB05E02C2803D1AF
:108B800004F1090007F0F1FA94F90810606840B2A6
:108B900006F02CFF032866D161680FF29410F9F7F4
:108BA0002AFB60E0618C00A807F036F89DF904000C
:108BB00002280AD1009800B207F014F800250099A5
:108BC0000FF27410F9F717FB4DE003284BD1009911
:108BD0000FF26C10F9F70FFB45E00AF0A1FC022838
:108BE0000AD1606800B206F0FDFF002561680FF24F
:108BF0005810F9F700FB36E0032834D161680FF212
:108C00005010F9F7F8FA2EE0606805280CD12846D4
:108C10000AF04DFD02280DD0032824D161680FF21F
:108C20004010F9F7E8FA1EE002281CD10AF043FED2
:108C30000228F1D1606800B206F0D4FF0025616817
:108C40000FF21410F9F7D7FA0DE0204607F049F8B3
:108C500009E0204607F00CFA05E061680FF2081001
:108C6000F9F7C9FA0025284605B030BD0120704744
:108C70000FB4022004B070470120704700207047F5
:108C800070470000534D4143202564202564202572
:108C900064000000534D4120256420256420256494
:108CA00000000000534D52432025642025642025F8
:108CB00064000000534D5220256420256420256463
:108CC000000000005044205365745354000000001D
:108CD00041542052492D256420256420256400003C
:108CE000415420524920426174202D25642025647E
:108CF0002025640050442055542D256400000000B8
:108D0000534C4D2025640000414C4F462025640003
:108D1000414C4346202564004F4A4820454C2030B2
:108D20007825782030782578203078257800000064
:108D3000524C434620256400504C4F462025640089
:108D4000504C43462025640050414F462025640086
:108D5000504143462025640050504F462025640072
:108D600050504346202564004558204C4D454C202A
:108D700025640000010040F10980F446404200F003
:108D800005F851F000416047010000BF09D0B0FA7A
:108D900080F18840C91CC1F58461090501EBD0212F
:108DA00040057047B0B581EA030C0CF0004C40F26E
:108DB000FF7515EA11541DBF15EA1357AC42AF42B7
:108DC00039E0E41923EA455343F48013C90241F022
:108DD000004141EA505EC7021100A7FB02020028D1
:108DE0004FF00000EEFB01204FF00001E3FB0721F4
:108DF00018BF42F00102401800214941E3FB0E0177
:108E0000A4F580640F0302D252004041494154F15D
:108E100001046CDD470872F1004250F1000051EB93
:108E20000451A1F580115CBF41EA0C01B0BD4CEAD0
:108E300005510020B0BD05EA1357AC4214BFAF4244
:108E400041E050EA410E1CBF52EA430E02E0614687
:108E50000020B0BD24423C441BD15FEA070EF6D08F
:108E6000090302BF01460020AEF1140EB1FA81F7EA
:108E7000AEEB070401FA07FE0C37C7F1200100FA38
:108E800007F7C8404EEA000E23EA455343F4801327
:108E9000A2E733F00043B3FA83F704BFB2FA82FECD
:108EA00077440B3FE41BB7F1200E2FBF02FA0EF3FD
:108EB000BB40C7F1200E22FA0EFE38BF43EA0E0374
:108EC000BA40641C82E750EA410E14BF52EA430ED6
:108ED0006FF000014FF4001717EB430F8ABF1946DC
:108EE00017EB410FB5E74CEA05510020B0BDD4F1B6
:108EF0000104B4F120070FDAC4F12007520828BF9B
:108F000042F0010210FA07F501FA07F7E1BF2A4320
:108F1000E0403843E1400FE0352C98DCC7F12004F5
:108F200052EA400220FA07F218BF42F0010231FA79
:108F300007F0A1400A43002172F1004250F1000005
:108F400051EB0C01B0BD00005FF0FF0C1CEAD051EA
:108F500014BF614506E0C110400721F0E04101F176
:108F60006051704779B900F0004100020AD0B0FAB0
:108F700080FC00FA0CF001F16051A1EB0C5101EB07
:108F8000D0214005704741020CBF40F4E0016FF072
:108F900000010020704700004FEAF17CBCF1E04C7A
:108FA0002CBFBCF5001F11E05FEA4C0C34BFBCF1D4
:108FB0007F5F2EE05FEA9C0C4FEA0C1C4FEA3C0CF2
:108FC000C10071F100414CEB50707047C90241EA99
:108FD0005051C00218BF41F0010141F000414FEA79
:108FE0006C50C0F10900212810D240EACC7CCCF1B1
:108FF000200C11FA0CF070F10040CCF1200C21FA99
:109000000CF00CF0004C40EB0C0070474FEACC70B9
:109010007047490011F5001F04D84FEACC10FF300B
:10902000C0057047C817704762F30F2262F31F42F2
:10903000401810F0030308D0C91A1FD3DB0748BF3C
:1090400000F8012D28BF20F8022D130030B414467B
:109050001546103928BF20E93C00FAD8490728BF37
:1090600020E90C0048BF40F8042D890028BF20F8F3
:10907000022D48BF00F8012D30BC7047C91818BF39
:1090800000F8012DCB0728BF00F8012D7047000024
:10909000DFF8AC1100220A700A70012802D00428FF
:1090A00003D0704701200870704705200870704792
:1090B00064490860704710B463494A6802F00C02C2
:1090C000082A13D10A680B6803F03F03604CB4FB15
:1090D000F3F30A68C2F388125A430B68C3F30143DF
:1090E0005B1C5B00B2FBF3F2026001E0584A0260D5
:1090F0004A6802F0F003574A1B099B5C046824FA93
:1091000003F343604C6804F4E054A40AA45CE34015
:109110008360496801F46041490B895C426822FA26
:1091200001F1C16010BC7047484900F44072B2F5CB
:10913000407F06D10A6822F4F812474B03401A43D5
:109140000A608A6E000552EA1050886670474349EB
:1091500008607047424908607047424A0029116818
:1091600002D008431060704721EA00001060704789
:109170003D4A0029116802D008431060704721EA77
:10918000000010607047394A0029116802D0084376
:109190001060704721EA000010607047344A0029CF
:1091A000116802D008431060704721EA0000106087
:1091B0007047304A0029116802D008431060704798
:1091C00021EA0000106070472B4A0029116802D084
:1091D00008431060704721EA000010607047274A7A
:1091E0000029117802D008431070704721EA00006E
:1091F000107070474109114A012901D1116804E03A
:10920000022901D1116F00E0516F00F01F0021FA17
:1092100000F000F0010070471948016841F08071CA
:10922000016070470021174A1268024200D00121F4
:109230000846704714490870704700000038024023
:1092400070380240800E474204380240083802401D
:109250000024F400B4870020FFFCFF0F3C0E4742BF
:10926000400E474230380240403802404438024005
:109270001038024020380240243802400D380240A5
:10928000743802400C3802400E38024080B527493D
:10929000884209D101210846FFF780FF0021012003
:1092A000BDE80440FFF77ABF2149884209D1012176
:1092B0000220FFF773FF00210220BDE80440FFF702
:1092C0006DBF1C49884209D101210420FFF766FFC8
:1092D00000210420BDE80440FFF760BF1649884222
:1092E00009D101210820FFF759FF00210820BDE81E
:1092F0000440FFF753BF1149884209D101211020D2
:10930000FFF74CFF00211020BDE80440FFF746BFE7
:109310000B49884209D101218020FFF73FFF00213E
:109320008020BDE80440FFF739BF01BD00000240C6
:109330000004024000080240000C024000100240FD
:10934000001C0240F0B4002232E0012393400C687C
:109350001C409C422BD154000325A540ED430668D8
:109360002E40066006680F79A7403E4306600E79DE
:10937000012E01D0022E11D186682E4086608668AB
:109380004F79A7403E438660466826EA0303436060
:1093900043688E799640B6B233434360C3682B402E
:1093A000C360C368CD7905FA04F42343C360521C3B
:1093B000102ACAD3F0BC70474FF6FF71016000213C
:1093C000017141718171C1717047002200690842C9
:1093D00000D00122104670470183704741837047D7
:1093E00010B4CB1000EB830001F007018900036A81
:1093F0000F248C40A3430362036A02FA01F119436C
:10940000016210BC7047000080B5434988420BD10F
:1094100001214FF40010FFF7CCFE00214FF40010A3
:10942000BDE80440FFF7C5BE3C4988420BD101218D
:109430004FF48000FFF7BDFE00214FF48000BDE82F
:109440000440FFF7B6BE364988420BD101214FF4E4
:109450000000FFF7AEFE00214FF40000BDE804401D
:10946000FFF7A7BE01BD7FB504460D46A68800A83C
:10947000FFF721FE02992B48B1FBF0F04FF6C072C6
:1094800032400243A28022884FF6FE731A402280A7
:109490002A68254B9A420AD25200B1FBF2F10A46E1
:1094A00092B2042A00DA0421401C208421E0EB88D7
:1094B0004BF6FF76B34204D102EB4202B1FBF2F16C
:1094C00006E019235A43B1FBF2F141F4804189B21D
:1094D0000A0502D141F0010189B241F4004180B294
:1094E0004FF4967250434FF47A7290FBF2F0401CA6
:1094F0002084A183208840F00100208020884FF63E
:10950000F5310840A9880843698908432080A88963
:109510002989084320817FBD005400400058004045
:10952000005C004040420F00A18601000029018834
:1095300003D041F00101018070474FF6FE721140E7
:10954000018070470029018803D041F480710180B7
:1095500070474FF6FF621140018070470029018873
:1095600003D041F40071018070474FF6FF52114063
:1095700001807047002A02D041F0010101E001F0B2
:10958000FE01018270470029018803D041F4806107
:10959000018070474FF6FF3211400180704700296B
:1095A000018803D041F40041018070474904490C0F
:1095B0000180704782B00246002003460193009369
:1095C00000920A0F01920902090A019A002A03D0A7
:1095D000009A1432009203E0090C009A18320092AB
:1095E000009A12680A4200D0012002B070470000C1
:1095F00080B5254988420BD101214FF48050FFF7F7
:10960000E3FD00214FF48050BDE80440FFF7DCBDCE
:109610001E4988420BD101214FF48040FFF7C9FD5C
:1096200000214FF48040BDE80440FFF7C2BD184957
:1096300088420BD101214FF40040FFF7BAFD002111
:109640004FF40040BDE80440FFF7B3BD01BD028800
:1096500002F441520B881A434B881A438B881A43F1
:10966000CB881A430B891A434B891A438B891A43B7
:10967000CB891A430280828B4FF2FF731A40828398
:10968000098A018270470000003001400038004024
:10969000003C00400029018803D041F040010180D6
:1096A00070474FF6BF72114001807047002A8288D0
:1096B00002D011438180704722EA01018180704706
:1096C00000220089084200D00122104670470000A5
:1096D0000168490849000160002101604160816022
:1096E000C1600161212141616A49884203D16A4810
:1096F0003D21016070476949884204D166484FF4B2
:109700007461016070476649884204D162484FF431
:109710007411016070476349884204D15E484FF07C
:109720007461016070476049884203D15A485F49BB
:10973000416070475E49884203D157485D494160A6
:1097400070475D49884203D153485C494160704786
:109750005B49884204D150484FF03D514160704709
:109760005849884203D158483D2101607047574904
:10977000884204D154484FF47461016070475449E1
:10978000884204D150484FF4741101607047514928
:10979000884204D14C484FF07461016070474E49D3
:1097A000884203D148484149416070474B4988424B
:1097B00003D145483F49416070474949884203D138
:1097C00041483E49416070474649884203D13E487E
:1097D0004FF03D51416070470268434B1A400B689F
:1097E0001A43CB681A434B691A438B691A43CB69F6
:1097F0001A430B6A1A434B6A1A438B6A1A434B6B20
:109800001A438B6B1A4302604269D208CB6A53EA4F
:10981000C2020B6B1A4342610A6942604A68826065
:109820008968C16070470029016803D041F00101D7
:10983000016070474908490001607047002A01D063
:1098400001617047C1607047006800F00100704717
:1098500000221C4B984201D2244800E024488B008F
:1098600001D5406800E0006808402249084200D065
:10987000012210467047134A904201D21B4800E073
:109880001B481C4A0A40890001D5C26070478260AB
:1098900070470000106002400860024028600240EB
:1098A0004060024058600240706002403D0000206D
:1098B00088600240400F0020A060024000003D2070
:1098C000B86002401064024008640240286402400C
:1098D0004064024058640240706402408864024060
:1098E000A0640240B86402403F801CF00060024067
:1098F000006402407D0F7D0F0249086070470249F5
:109900000860704720000E4224000E4270B50446E5
:109910000026DFF83854CA20E8615320E86100F0DF
:1099200018F8002811D0286820F040002860286826
:10993000216808432860A068A860A868616840EAB8
:109940000140A86000F024F80126FF20E8613046BD
:1099500070BD81B000200090DFF8F4030168490673
:1099600013D44FF0FF310160016801F04001009A0B
:10997000521C0092009AB2F5803F01D00029F3D02A
:109980000068800900F0010000E0012001B070478C
:10999000DFF8BC03016821F080010160704781B0ED
:1099A00000200090DFF8A813CA2088615320886146
:1099B000086820F0A0000860086800F02000009A05
:1099C000521C0092009AB2F5003F01D00028F3D05B
:1099D0000868400900F00100FF228A6101B0704769
:1099E000F8B507460E460024DFF85C53002FA86840
:1099F00004D140060AD42046F07007E0400603D5A3
:109A0000307800F0BEF901E02046F0703078002F89
:109A100009D07178090241EA0040B1780843F17831
:109A200040EA01460FE000F0A1F90746707800F027
:109A30009DF9000240EA0747B07800F097F93843F3
:109A4000F17840EA0146CA20686253206862FFF755
:109A500080FF00280FD0DFF8FC0230402860FFF7BD
:109A600097FFA868800605D4FFF799FF002802D069
:109A7000012400E00124FF2068622046F2BD10B5F9
:109A80000C46DFF8C4120968DFF8C82211400A0C3E
:109A900002F03F0323700B0A03F07F03637001F0B1
:109AA0007F01A17002F04001E17000280BD1207805
:109AB00000F067F92070607800F063F96070A078BA
:109AC00000F05FF9A07010BDDFF88C12486A0968D9
:109AD000704770B506460D460024002E06D1687802
:109AE000C10603D500F0EF000A306870002E05D0E3
:109AF000687800F046F9A87800F043F9E878002E7D
:109B000009D06978090241EA0040A9780843297818
:109B100040EA41360FE000F029F90646687800F087
:109B200025F9000240EA0646A87800F01FF9304304
:109B3000297840EA4136DFF82052CA2028625320B3
:109B40002862FFF706FF00280FD0DFF81002304030
:109B50002860FFF71DFF6868800605D4FFF71FFF28
:109B6000002802D0012400E00124FF2028622046C2
:109B700070BD10B50C46DFF8E0110968DFF8DC2194
:109B800011400A0CE2700A0A02F01F02627001F032
:109B90003F02A270490B01F00701217000280BD190
:109BA000E07800F0EEF8E070607800F0EAF86070BD
:109BB000A07800F0E6F8A07010BDDFF89011CA227E
:109BC000CA615322CA610A68D208D2000A600A68D0
:109BD00010430860FF20C8617047DFF88411CA2273
:109BE0000A6153220A610860FF200861704781B052
:109BF00000210091DFF85411CA22CA615322CA61C0
:109C00000028086804D040F480600860012012E059
:109C100020F480600860486800F00400009A521C3C
:109C20000092009AB2F5803F01D00028F3D0486836
:109C3000800800F00100FF22CA6101B0704781B0C6
:109C400000220092474A0092009A02EB80000090A6
:109C50000098016001B0704781B000210091414936
:109C60000091009901EB800000900098006801B01D
:109C7000704738B500242246344DCA23EB61532384
:109C8000EB616B681B0701D406E0521C6B681B0775
:109C900002D5B2F5805FF8D16A68120709D42A6844
:109CA000D20606D408436862FFF779FE002800D088
:109CB0000124FF20E861204632BD244ACA23D36133
:109CC0005323D36100F0040320F00400002911683D
:109CD00005D008431060906B1843906305E021EABB
:109CE00000001060906B98439063FF20D061704734
:109CF0000021174A12681C4B1A40024200D0012171
:109D00000846704710B40021104A936B03F0040317
:109D10001468044003EAD0332343526802EA101067
:109D200002D0000400D00121084610BC7047084949
:109D30000003000C40F080000A6802F0800262EA32
:109D4000000008607047000000280040082800401C
:109D50000C2800407F7F7F00042800403FFFFF0069
:109D600014280040502800407F3F0100002101E0FE
:109D7000491C0A38C0B20A28FADA40EA0110C0B217
:109D80007047010901EB810200F00F0000EB420077
:109D9000C0B2704730B40168CB4321498279002AB0
:109DA00027D00A4614682340136053680468A3430D
:109DB00053600379CC18236805682B4323609368AC
:109DC0000468A3439360D3680468A343D3604379D2
:109DD0000568102B07D1916829439160D16800680C
:109DE0000843D0600AE051FA83F4206828432060D9
:109DF00004E000790C1820681840206030BC7047DF
:109E00000021074A136803405269024202D0002B26
:109E100000D00121084670470249086070470000E1
:109E2000003C0140143C01401949084319490860AD
:109E3000704770B403781A460121C478002C1DD0F5
:109E4000144B1B6803F4E063C3F5E0631B0A44781A
:109E5000C3F10405AC4085780F2646FA03F32B4086
:109E600023431B010C4C1355007842110B4B00F09F
:109E70001F0001FA00F043F8220006E05011084AE2
:109E800003F01F03994042F8201070BC7047000097
:109E90000000FA050CED00E000E400E000E100E065
:109EA00080E100E030B401F00302920021F00301F0
:109EB000054BCC580F259540AC43CC50CC58904026
:109EC0002043C85030BC70470838014080B501219C
:109ED0004FF48070FFF778F900214FF48070BDE8EF
:109EE0000440FFF771B942684C4B1A400B7942EAC3
:109EF00003220B681A4342608268494B1A400B697F
:109F00001A43CB681A438B681A434B7942EA4302DF
:109F10008260C26A22F47002097D491EC9B242EA17
:109F20000151C1627047002101600171417181607E
:109F3000C16001610121017570473A490A683A4BD5
:109F40001A4003681A4343681A4383681A43C06877
:109F50001043086070470021016041608160C1606A
:109F600070470029816803D041F00101816070478A
:109F7000490849008160704770B407240A290BDB47
:109F8000C568A1F10A0606EB4606B44025EA0404BA
:109F9000B3402343C36008E0056901EB4106B440C8
:109FA00025EA0404B3402343036113461F24072B0F
:109FB00009DA436B521E02EB82029440A3439140A4
:109FC0001943416314E00D2B09DA036BD21F02EB36
:109FD00082029440A34391401943016308E0C36A9D
:109FE0000D3A02EB82029440A34391401943C162AF
:109FF00070BC7047816841F08041816070470029E2
:10A00000816803D041F480618160704721F48061F0
:10A0100081607047C06C80B270470000FFFEFFFC9B
:10A02000FDF7FFC004230140E030FCFF0022006880
:10A03000084200D0012210467047000013F0004C87
:10A0400003D55B42524263F100039CEA210C00F00D
:10A05000178010B5644603D34942404261F10001C4
:10A0600000F00EF8640004D34942404261F100015F
:10A07000244203D55B42524263F1000310BD00004D
:10A080001B4213D1094236D12AB18446B0FBF2F00B
:10A0900002FB10C2704709F06FBCFCD30022002302
:10A0A00070470B000200002100207047904271EBC6
:10A0B000030CF6D370B5B1FA81F4B3FA83F52C1B17
:10A0C000A340C4F1200532FA05F63343A2405FF005
:10A0D0000046E64002E05B085FEA3202841A71EB58
:10A0E000030524BF204629467641F4D302000B0025
:10A0F0003000002170BD012ACFD970B5140C20D0DA
:10A10000B1FA81F4B2FA82F5C4F120046419B4F111
:10A110002006D6D3B2405FF00044F440002502E0B0
:10A1200052085FEA3303C61A71EB020E24BF3046B1
:10A13000714664416D41F3D302000B0020002900F9
:10A1400070BD0C46B1FBF2F102FB11452D0445EA4E
:10A150001045B5FBF2F402FB145580B240EA054508
:10A16000B5FBF2F002FB105240EA044070BD000063
:10A1700010B5040010480078002805D10F4809F0F8
:10A1800022FC0D48012101700C4809F052FC20000E
:10A190000AF022FB0400094809F07FFC200010BDF2
:10A1A00010B50400054809F044FC20000AF06EFCDC
:10A1B000024809F072FC10BD945301203050012078
:10A1C000BFF34F8FDFF8B40C006810F4E060DFF8E5
:10A1D000B01C0843DFF8A41C0860BFF34F8FFEE7F4
:10A1E00000B583B00020ADF8040000208DF8060013
:10A1F00000208DF80700012000900DF10603762263
:10A20000D0210020F8F7C7F8002801D1002044E051
:10A2100076208DF804009DF8060050F020008DF89F
:10A220000500022301AAD0210020F8F75AF80028DF
:10A2300001D1002031E0012000900DF107034922F7
:10A24000D0210020F8F7A7F8002801D1002024E051
:10A2500049208DF804009DF8070050F001008DF8AA
:10A260000500022301AAD0210020F8F73AF80028BF
:10A2700001D1002011E076208DF804009DF8060041
:10A280008DF80500022301AAD0210020F8F729F853
:10A29000002801D1002000E001200EBD38B50400E7
:10A2A000F7F727FF0500DFF8040D0078401CDFF802
:10A2B000FC1C0870DFF8F40C4078F021084202D052
:10A2C0009920FBF7EFFBFBF75AFCDFF8E00C407836
:10A2D000401CDFF8D81C4870210089B22800F8F72C
:10A2E000F5F8DFF8C80C4078F021084202D0992038
:10A2F000FBF7D8FBDFF8B40C4078401EDFF8AC1C4D
:10A300004870C0B2002801D1FBF733FCFCF78BFA90
:10A3100031BD10B582B00020ADF80000F7F7E9FEBE
:10A3200004006B208DF8000080208DF801000223CE
:10A3300000AAD0210020F7F7D4FF002801D1002087
:10A3400094E064212000F8F7C1F8FFF749FF0028E6
:10A3500001D100208AE06B208DF8000000208DF8EC
:10A360000100022300AAD0210020F7F7BAFF00283D
:10A3700001D100207AE028212000F8F7A7F8192061
:10A380008DF8000004208DF80100022300AAD021DE
:10A390000020F7F7A6FF002801D1002066E01A2070
:10A3A0008DF8000003208DF80100022300AAD021BF
:10A3B0000020F7F796FF002801D1002056E01B206F
:10A3C0008DF8000018208DF80100022300AAD0218A
:10A3D0000020F7F786FF002801D1002046E01D206D
:10A3E0008DF8000003208DF80100022300AAD0217F
:10A3F0000020F7F776FF002801D1002036E06A2020
:10A400008DF8000000208DF80100022300AAD02161
:10A410000020F7F766FF002801D1002026E06C201D
:10A420008DF800003F208DF801009DF80110DFF845
:10A43000500DF7F7E0FE022300AAD0210020F7F725
:10A4400050FF002801D1002010E06B208DF80000A3
:10A4500040208DF80100022300AAD0210020F7F748
:10A4600040FF002801D1002000E0012016BD017846
:10A47000407850EA012000B2704780B50220009079
:10A48000DFF8003D6B22D0210020F7F784FF002881
:10A4900001D100205BE001200090DFF8EC3C1A22A3
:10A4A000D0210020F7F777FF002801D100204EE0EF
:10A4B00001200090DFF8D43C1B22D0210020F7F7C8
:10A4C0006AFF002801D1002041E001200090DFF860
:10A4D000C03C1C22D0210020F7F75DFF002801D1ED
:10A4E000002034E001200090DFF8A83C1D22D0219C
:10A4F0000020F7F750FF002801D1002027E00120BD
:10A500000090DFF8943C6A22D0210020F7F743FF47
:10A51000002801D100201AE001200090DFF87C3CE7
:10A520003822D0210020F7F736FF002801D1002083
:10A530000DE001200090DFF8683C1922D0210020B6
:10A54000F7F729FF002801D1002000E0012002BD1B
:10A5500080B50020ADF800001A208DF80000DFF86B
:10A56000240C00798DF80100022300AAD0210020DC
:10A57000F7F7B7FE002801D1002090E01B208DF8EE
:10A580000000DFF8000C40798DF80100022300AADA
:10A59000D0210020F7F7A5FE002801D100207EE0A1
:10A5A0001C208DF80000DFF8DC0B80798DF80100AD
:10A5B000022300AAD0210020F7F793FE002801D142
:10A5C00000206CE01D208DF80000DFF8B80BC0798A
:10A5D0008DF80100022300AAD0210020F7F781FEA8
:10A5E000002801D100205AE06A208DF80000DFF831
:10A5F000940BC0788DF80100022300AAD02100201E
:10A60000F7F76FFE002801D1002048E019208DF8EF
:10A610000000DFF8700B80788DF80100022300AA9B
:10A62000D0210020F7F75DFE002801D1002036E0A0
:10A6300038208DF80000DFF84C0B007A8DF801000F
:10A64000022300AAD0210020F7F74BFE002801D1F9
:10A65000002024E06B208DF80000DFF8280B007844
:10A660008DF80100022300AAD0210020F7F739FE5F
:10A67000002801D1002012E06C208DF80000DFF8E6
:10A68000040B40788DF80100022300AAD02100209D
:10A69000F7F727FE002801D1002000E0012002BDCD
:10A6A00010B582B00020ADF80000DFF8D80A0078BD
:10A6B000400612D56B208DF8000000208DF80100B7
:10A6C000022300AAD0210020F7F70BFE002801D1B9
:10A6D0000020C9E03220FFF7E1FD6C208DF800007A
:10A6E000DFF8A00A407810F0F8008DF8010002238E
:10A6F00000AAD0210020F7F7F4FD002801D10020A6
:10A70000B2E06A208DF8000000208DF801000223DD
:10A7100000AAD0210020F7F7E4FD002801D1002095
:10A72000A2E0002400E0641C062C10DA14F11300EF
:10A730008DF8000000208DF80100022300AAD0212E
:10A740000020F7F7CEFD0028EDD100208CE0192085
:10A750008DF8000000208DF80100022300AAD0210E
:10A760000020F7F7BEFD002801D100207CE01A2070
:10A770008DF8000003208DF801004FF4FA642000EA
:10A78000FA281DD0B0F5FA7F13D0B0F57A7F09D042
:10A79000B0F5FA6F19D19DF8010050F018008DF84E
:10A7A000010016E09DF8010050F010008DF8010046
:10A7B0000FE09DF8010050F008008DF8010008E05E
:10A7C0009DF801008DF8010003E09DF801008DF86F
:10A7D0000100022300AAD0210020F7F782FD002803
:10A7E00001D1002040E0FA2C14D0B4F5FA7F0DD04E
:10A7F000B4F57A7F06D0B4F5FA6F0FD103208DF847
:10A8000001000EE002208DF801000AE001208DF821
:10A81000010006E000208DF8010002E000208DF824
:10A8200001001B208DF800009DF80100C0008DF88C
:10A830000100022300AAD0210020F7F752FD0028D2
:10A8400001D1002010E038208DF8000000208DF8A4
:10A850000100022300AAD0210020F7F742FD0028C2
:10A8600001D1002000E0012016BD00B583B000201A
:10A87000ADF8060000208DF804006B208DF806006E
:10A8800001208DF8070002230DF10602D0210120DE
:10A89000F7F727FD002801D1002023E02820FFF74B
:10A8A000FDFC0120009001AB6C22D0210120F7F7C4
:10A8B00072FD002801D1002014E06C208DF8060004
:10A8C0009DF8040010F0C0008DF8070002230DF180
:10A8D0000602D0210120F7F704FD002801D1002055
:10A8E00000E001200EBD2DE9F04F85B004000D0001
:10A8F00016001F000020ADF8040002A8002100226D
:10A9000006C0083806208DF8060038208DF80400AF
:10A9100000208DF80500022301AAD0210120F7F7BD
:10A92000E0FC002802D15FF0FF3070E123208DF8B9
:10A93000040000208DF80500022301AAD021012087
:10A94000F7F7CFFC002802D15FF0FF305FE16A200B
:10A950008DF8040000208DF80500022301AAD02103
:10A960000120F7F7BEFC002802D15FF0FF304EE176
:10A970006A208DF8040004208DF80500022301AA46
:10A98000D0210120F7F7ADFC002802D15FF0FF30A5
:10A990003DE11A208DF8040001208DF80500022306
:10A9A00001AAD0210120F7F79CFC002802D15FF01A
:10A9B000FF302CE119208DF8040000208DF80500EF
:10A9C000022301AAD0210120F7F78BFC002802D135
:10A9D0005FF0FF301BE11B208DF804008DF805406F
:10A9E000022301AAD0210120F7F77BFC002802D125
:10A9F0005FF0FF300BE1FFB2002F0FD01C208DF86D
:10AA000004008DF80540022301AAD0210120F7F7A8
:10AA100068FC002802D15FF0FF30F8E064B2002C3F
:10AA200002D0C820FFF73AFC6A208DF804004420C9
:10AA30008DF80500022301AAD0210120F7F751FC6F
:10AA4000002802D15FF0FF30E1E023208DF8040000
:10AA5000FFB2002F03D008208DF8050002E070201F
:10AA60008DF80500022301AAD0210120F7F739FC57
:10AA7000002802D15FF0FF30C9E00A20FFF70EFC8A
:10AA8000002408E0E4B2002045F82400E4B20020ED
:10AA900046F82400641CE4B2032CF3DB5FF00009E9
:10AAA000B9F1320F6EDA0A20FFF7F8FB02200090AE
:10AAB00002AB7222D0210120F7F76DFC002802D1F1
:10AAC0005FF0FF30A3E002A8FFF7D1FC9DF806106D
:10AAD00090FBF1F8B8F1070F02DA7FF0010096E081
:10AAE00000241AE05FFA8AFA55F82AB05FFA8AFA67
:10AAF00002A810EB4A00FFF7BAFC0BFA80F05FFAED
:10AB00008AFA45F82A001AF1010A5FFA8AFABAF1BC
:10AB1000030FE7DB19F10109641CE4B24445BFDA15
:10AB2000B9F1320FBCDA9DF80600009002AB742236
:10AB3000D0210120F7F72FFC002802D15FF0FF3071
:10AB400065E0FFB2002F1AD05FF0000A5FFA8AFAC0
:10AB5000BAF1030FDEDA5FFA8AFA56F82AB05FFA22
:10AB60008AFA02A810EB4A00FFF781FC0BFA80F08A
:10AB70005FFA8AFA46F82A001AF1010AE6E75FF05E
:10AB8000000AC2E723208DF8040000208DF805009C
:10AB9000022301AAD0210120F7F7A3FB002802D14C
:10ABA0005FF0FF3033E05FF0000A0FE05FFA8AFAEF
:10ABB00055F82A004FF47A714843322190FBF1F0A6
:10ABC0005FFA8AFA45F82A001AF1010A5FFA8AFA4E
:10ABD000BAF1030FEADBFFB2002F17D05FF0000AD3
:10ABE0000FE05FFA8AFA56F82A004FF47A71484368
:10ABF000322190FBF1F05FFA8AFA46F82A001AF146
:10AC0000010A5FFA8AFABAF1030FEADB012005B004
:10AC1000BDE8F08F2DE9F04389B004000D00160067
:10AC200000275FF0010801A8002101605FF0000922
:10AC30000320009001AB0D22D0210120F7F7ABFBE0
:10AC4000002801D15FF0FF385FF0000905E005A89A
:10AC5000002140F8291019F10109B9F1030F11DAA7
:10AC600001A819F800000028F1D001A819F8000087
:10AC7000DFF8C81A11EB400030F8020C05A941F8C2
:10AC80002900E8E75FF000091FE002A850F829005A
:10AC9000DFF8AC1A884207DADFF8A80AF7F7ABFA50
:10ACA000012010FA09F0074302A850F82900DFF844
:10ACB000981A884207DBDFF8940AF7F79CFA01201C
:10ACC00010FA09F0074319F10109B9F1030F2ADA63
:10ACD00055F8290056F82910401A0AF065F902A91A
:10ACE00041F8290005A850F829000028CDD002A875
:10ACF00050F8290005A951F8291090FBF1F0B0F5A2
:10AD00007A700AF051F924F8190034F91900B0F5F5
:10AD1000FA7FD8DDDFF8380AF7F76DFA012010FA6C
:10AD200009F00743CFE7B4F904000090B4F902300A
:10AD3000B4F900203900DFF81C0AF7F75CFA002F9D
:10AD400005D0DFF8140AF7F756FA7FF002084046FC
:10AD500040B209B0BDE8F08338B505000020ADF879
:10AD600000000020ADF80200F7F7C3F90400382016
:10AD70008DF8000000208DF80100022300AAD021E8
:10AD80000020F7F7AEFA002801D1002074E000F0AF
:10AD90002AFB002801D100206EE01F208DF8000062
:10ADA0004B208DF80100022300AAD0210020F7F7E4
:10ADB00098FA002801D100205EE01E208DF80000E6
:10ADC00006208DF80100022300AAD0210020F7F709
:10ADD00088FA002801D100204EE069208DF800009B
:10ADE000C0208DF80100022300AAD0210020F7F72F
:10ADF00078FA002801D100203EE001220121032041
:10AE0000F7F7EBFB0020F7F7EAFB38208DF800009E
:10AE100040208DF80100022300AAD0210020F7F77E
:10AE200060FA002801D1002026E0012028702000CF
:10AE3000407DC046012810D001212000F7F746FBD5
:10AE4000BDF80200401CADF80200BDF80200322837
:10AE5000EDDBDFF80809F7F7CEF901220021032026
:10AE6000F7F7BBFB0020F7F7BAFB00F0B2FB0028B6
:10AE700001D1002000E0012032BD00000CED00E017
:10AE80000400FA0570B58EB0040000A8002100226D
:10AE900006C00838012500260BA800210022002347
:10AEA0000EC00C3808A80021002200230EC00C3868
:10AEB00005A80021002200230EC00C3802A80021A2
:10AEC000002200230EC00C38FFF7D7FA002801D16A
:10AED000002056E0FFF7E4FB002806D00126FFF72C
:10AEE000C4FC002803D100204BE0002049E00123EE
:10AEF00002AA08A90020FFF7F6FC05006DB2012D9B
:10AF000004D0DFF85408F7F776F91CE0012305AA0E
:10AF10000BA97FF01F00FFF7E6FC05006DB2012DC5
:10AF200004D0DFF82C08F7F766F90CE005AA02A9AF
:10AF300000A8FFF76FFE05006DB2012D03D0DFF80A
:10AF40000408F7F758F92670BDF800006070BDF9E5
:10AF500000000012A070BDF80200E070BDF9020010
:10AF600000122071BDF804006071BDF904000012E8
:10AF7000A071E571FFF7ECFA002801D1002000E094
:10AF800001200EB070BD80B5DFF8D407007800282E
:10AF900009D1FFF7BEF9002801D1002004E0DFF855
:10AFA000C00701210170012002BD0000CC860020F5
:10AFB0001CB500208DF806000020ADF80400F7F75E
:10AFC00098F80400012000900DF106036B22D021B7
:10AFD0000020F7F7E0F9002801D1002088E09DF873
:10AFE00006006021084216D06B208DF804009DF801
:10AFF000060010F09F008DF80500022301AAD02161
:10B000000020F7F76EF9002801D1002070E014212C
:10B010002000F7F75BFA012000900DF106036C2287
:10B02000D0210020F7F7B7F9002801D100205FE018
:10B030006C208DF804009DF8060010F0C7008DF814
:10B040000500022301AAD0210020F7F74AF90028C1
:10B0500001D100204CE00A212000F7F737FA1D202B
:10B060008DF8040043208DF80500022301AAD021A9
:10B070000020F7F736F9002801D1002038E01C2025
:10B080008DF8040000208DF80500022301AAD021CC
:10B090000020F7F726F9002801D1002028E0202021
:10B0A0008DF8040080208DF80500022301AAD0212C
:10B0B0000020F7F716F9002801D1002018E01F2022
:10B0C0008DF8040080208DF80500022301AAD0210C
:10B0D0000020F7F706F9002801D1002008E0DFF88A
:10B0E0008406007850F00100DFF87816087001201F
:10B0F00016BD00B583B000208DF806000020ADF825
:10B100000400012000900DF106036C22D0210020E4
:10B11000F7F741F9002801D1002030E06C208DF8CC
:10B1200004009DF8060050F038008DF80500022359
:10B1300001AAD0210020F7F7D4F8002801D100207F
:10B140001DE0DFF82006007880070FD46B208DF813
:10B15000040040208DF80500022301AAD021002020
:10B16000F7F7BFF8002801D1002008E0DFF8F40568
:10B17000007810F0FE00DFF8EC15087001200EBD1D
:10B18000A44B0308185101201C5101201D5101201E
:10B190001E5101201F5101201B510120205101206F
:10B1A0001A51012000B583B000208DF80400002062
:10B1B000ADF806000120009001AB6C22D0210020E8
:10B1C000F7F7E9F8002801D1002014E06C208DF891
:10B1D00006009DF8040050F038008DF807000223A7
:10B1E0000DF10602D0210020F7F77BF8002801D1ED
:10B1F000002000E001200EBD2DE9F04186B00400E2
:10B200000D0004A80021002206C008380020ADF877
:10B210000C000126DFF850050768F6F76AFF804644
:10B22000DFF848050068401CDFF840150860012081
:10B23000009004AB6B22D0210020F7F7ACF8002877
:10B2400001D10020CCE09DF8100040061AD56B20FB
:10B250008DF80C009DF8100010F0BF008DF80D0067
:10B26000022303AAD0210020F7F73BF8002801D1E0
:10B270000020B5E014214046F7F728F9DFF8F00484
:10B28000F6F7B9FF0120009004AB6C22D02100201A
:10B29000F7F781F8002801D10020A1E09DF8100007
:10B2A000382108421ED06C208DF80C009DF810004B
:10B2B00010F0C7008DF80D00022303AAD021002052
:10B2C000F7F70FF8002801D1002089E0052140465A
:10B2D000F7F7FCF8DFF89C04F6F78DFFDFF8980429
:10B2E00001210160EDB2009504AB3B22D02100208A
:10B2F000F7F751F8002805D1DFF88004F6F77BFF57
:10B3000000206DE09DF8110020709DF81000607025
:10B310009DF81300A0709DF81200E0709DF81500D4
:10B3200020719DF814006071002000E0401C062888
:10B3300006D2015DDFF84824825C9142F6D00026F7
:10B34000F6B2012E18D1DFF83C040068401CDFF88B
:10B3500034140860DFF82C040068132804D1DFF8E7
:10B360002804F6F748FF0BE0DFF8180400681428FB
:10B3700006D1FEF725FF03E0DFF808040021016095
:10B3800006222100DFF8F803F8F711FCDFF8DC03F0
:10B390000068C82190FBF1F201FB120000281ED1C9
:10B3A000F86AC0680290F86A80680190B4F90400F5
:10B3B0000090B4F90230B4F90020DFF8BC03016852
:10B3C000DFF8C803F6F717FFDFF8A0030068DFF81F
:10B3D000C013884203DBDFF89403002101600120E1
:10B3E00006B0BDE8F08130B583B001240020ADF88F
:10B3F000060000208DF80400F6F77BFE0500012012
:10B40000009001AB6B22D0210020F6F7C4FF00288A
:10B4100001D100208BE09DF8040040061AD56B2076
:10B420008DF806009DF8040010F0BF008DF80700AD
:10B4300002230DF10602D0210020F6F752FF00286A
:10B4400001D1002073E014212800F7F73FF8D1481C
:10B45000F6F7D1FE1D208DF8060008208DF80700B4
:10B4600002230DF10602D0210020F6F73AFF002852
:10B4700001D100205BE00120009001AB6C22D021C3
:10B480000020F6F788FF002801D100204FE06C2053
:10B490008DF806009DF8040050F080008DF804003F
:10B4A0009DF8040050F007008DF804009DF804009A
:10B4B00010F0C7008DF804009DF804008DF8070017
:10B4C00002230DF10602D0210020F6F70AFF002822
:10B4D00001D100202BE00120009001AB6B22D02194
:10B4E0000020F6F758FF002801D100201FE06B2054
:10B4F0008DF806009DF8040010F0BF008DF80400E0
:10B500009DF8040050F020008DF804009DF8040020
:10B510008DF8070002230DF10602D0210020F6F776
:10B52000E0FE002801D1002001E02000C0B23EBDB5
:10B5300080B50020ADF80000FFF755FF002801D1CD
:10B54000002045E01F208DF800004B208DF8010001
:10B55000022300AAD0210020F6F7C3FE002801D163
:10B56000002035E01E208DF8000006208DF8010037
:10B57000022300AAD0210020F6F7B3FE002801D153
:10B58000002025E069208DF80000C0208DF8010022
:10B59000022300AAD0210020F6F7A3FE002801D143
:10B5A000002015E0012201210320F7F716F83820CA
:10B5B0008DF8000040208DF80100022300AAD02160
:10B5C0000020F6F78EFE002801D1002000E00120C7
:10B5D00002BD80B50020ADF800000122002103204B
:10B5E000F6F7FBFF38208DF8000000208DF80100F1
:10B5F000022300AAD0210020F6F773FE002801D113
:10B60000002058E06B208DF8000000208DF801002C
:10B61000022300AAD0210020F6F763FE002801D102
:10B62000002048E01D208DF8000000208DF801006A
:10B63000022300AAD0210020F6F753FE002801D1F2
:10B64000002038E06C208DF8000046480078032880
:10B6500003D100208DF8010012E042480078022852
:10B6600003D138208DF801000AE03E480078012817
:10B6700003D107208DF8010002E03F208DF8010082
:10B68000022300AAD0210020F6F72BFE002801D1CA
:10B69000002010E069208DF8000000208DF80100E6
:10B6A000022300AAD0210020F6F71BFE002801D1BA
:10B6B000002000E0012002BD80B50178012905D1FC
:10B6C000FFF74AFB00280AD1002009E0017802298F
:10B6D00005D1FFF7D7FB002801D1002000E00120B1
:10B6E00002BD80B50020ADF800001D208DF80000DF
:10B6F0000878002806D140208DF801002648F6F78A
:10B700007AFD05E043208DF801002448F6F773FD2B
:10B71000022300AAD0210020F6F7E3FD002801D182
:10B72000002000E0012002BD80B51D490020F9F78E
:10B730002BFF1C490B20F9F727FF01BDC03203087E
:10B74000003E49004C4C030801EFE700544C03084D
:10B75000444C0308204B03085C4C0308644C03086A
:10B760005750012068530120086000202C5201200E
:10B770006C4C0308744C03087C5201207C4C030879
:10B780005C520120D8520120004C0308BC4B030836
:10B79000A1860100844C0308204C03082C4C0308AC
:10B7A000DCFB0208904A030810B50024DFF8500CB7
:10B7B000007800280AD1FEF7ACFD002801D1002056
:10B7C00007E0DFF83C0C0121017000E001242000BB
:10B7D000C0B210BD1CB500208DF806000020ADF8E9
:10B7E0000400F6F786FC0400012000900DF106032A
:10B7F0006B22D0210120F6F7CEFD002801D10020D8
:10B8000068E09DF806006021084216D06B208DF894
:10B8100004009DF8060010F09F008DF8050002233B
:10B8200001AAD0210120F6F75CFD002801D10020FB
:10B8300050E01E212000F6F749FE012000900DF196
:10B8400006036C22D0210120F6F7A5FD002801D1C6
:10B8500000203FE06C208DF804009DF8060010F0F9
:10B86000F8008DF80500022301AAD0210120F6F787
:10B8700038FD002801D100202CE00A212000F6F735
:10B8800025FE1B208DF8040018208DF805000223EA
:10B8900001AAD0210120F6F724FD002801D10020C3
:10B8A00018E01A208DF8040003208DF8050002230B
:10B8B00001AAD0210120F6F714FD002801D10020B3
:10B8C00008E0DFF8400B007850F00200DFF8341B8E
:10B8D0000870012016BD00B583B000208DF8060069
:10B8E0000020ADF80400012000900DF106036C2249
:10B8F000D0210120F6F74FFD002801D1002030E0D3
:10B900006C208DF804009DF8060050F007008DF8BB
:10B910000500022301AAD0210120F6F7E2FC00284D
:10B9200001D100201DE0DFF8DC0A0078C0070FD449
:10B930006B208DF8040040208DF80500022301AA39
:10B94000D0210120F6F7CDFC002801D1002008E02D
:10B95000DFF8B00A007810F0FD00DFF8A81A0870D0
:10B9600001200EBD00B583B000208DF8040000203A
:10B97000ADF806000120009001AB6C22D02101201F
:10B98000F6F709FD002801D1002014E06C208DF8A5
:10B9900006009DF8040050F007008DF80700022310
:10B9A0000DF10602D0210120F6F79BFC002801D101
:10B9B000002000E001200EBD7FB5040002A8002198
:10B9C000002206C0083800260020ADF80400F6F773
:10B9D00090FB05000120009002AB6B22D0210120DA
:10B9E000F6F7D9FC002801D1002083E09DF808007B
:10B9F000400625D56B208DF804009DF8080010F056
:10BA0000BF008DF80500022301AAD0210120F6F71E
:10BA100068FC002801D100206CE032212800F6F7F4
:10BA200055FDDFF8E409F6F7E6FB002603E0F6B281
:10BA300000203055761CF6B2062EF8DB012059E0C6
:10BA40000120009002AB6C22D0210120F6F7A3FC6C
:10BA5000002801D100204DE09DF808000721084290
:10BA600025D06C208DF804009DF8080010F0F80037
:10BA70008DF80500022301AAD0210120F6F731FC40
:10BA8000002801D1002035E00A212800F6F71EFD2C
:10BA9000DFF87809F6F7AFFB002603E0F6B20020E6
:10BAA0003055761CF6B2062EF8DB012022E0062087
:10BAB000009002AB4322D0210120F6F76CFC002855
:10BAC00005D1DFF84C09F6F796FB002012E09DF84F
:10BAD000090020709DF8080060709DF80B00A070B0
:10BAE0009DF80A00E0709DF80D0020719DF80C0093
:10BAF0006071012004B070BD2DE9F64FADF63C6DCC
:10BB000005000020ADF8080003A81421F9F788FF0C
:10BB1000002608A80021002200230EC00C385FF088
:10BB2000000940F68C1068444FF49661F9F778FFED
:10BB3000FFA8E0304FF49661F9F772FF0BA84FF4BD
:10BB40009661F9F76DFF5FF00008002700240020E0
:10BB5000070000E07F1C032F80F2BA806B208DF875
:10BB60000800781C8DF80900022302AAD0210120C8
:10BB7000F6F7B7FB002801D1002099E13220FEF74B
:10BB80008DFB6A208DF8080044208DF809000223FF
:10BB900002AAD0210120F6F7A4FB002801D1002041
:10BBA00086E1012409E019EB060608A850F82700F1
:10BBB00019EB000008A941F827002000441E0128C5
:10BBC00075DB23208DF8080070208DF80900022312
:10BBD00002AAD0210120F6F784FB002801D1002021
:10BBE00066E14B20FEF75AFB23208DF80800002069
:10BBF0008DF80900022302AAD0210120F6F771FB7B
:10BC0000002801D1002053E10220009003AB7222F2
:10BC1000D0210120F6F7BFFB002801D1002047E129
:10BC200003A8FEF724FC00EE100AB8EEC00A10EEDE
:10BC3000100AFDF789F9DFF8DC27DFF8DC37FDF7BC
:10BC4000B1F809F0B5F98146B9F148000128B4DB33
:10BC50005FF000081DE003A8FEF709FC18EB0601E1
:10BC600040F68C126A4422F811000DF10E00FEF726
:10BC7000FEFB18EB0601FFAAE03222F8110004A82F
:10BC8000FEF7F5FB18EB06010BAA22F8110018F1DC
:10BC90000108C84587DA0620009003AB7422D02142
:10BCA0000120F6F778FB0028D5D1002000E1232001
:10BCB0008DF8080000208DF80900022302AAD02187
:10BCC0000120F6F70EFB00287FF444AF0020EFE0E0
:10BCD000002E01D0340000E001245FF000080020B5
:10BCE0000021C5E9000100200021C5E90201002072
:10BCF0000021C5E9040122E0D5E9000140F68C12DB
:10BD00006A4432F91820D31780185941C5E9000157
:10BD1000D5E90201FFAAE03232F91820D3178018C2
:10BD20005941C5E90201D5E904010BAA32F91820ED
:10BD3000D31780185941C5E9040118F10108B0452D
:10BD4000DADBD5E900012200E317FEF777F9C5E950
:10BD50000001D5E902012200E317FEF76FF9C5E9FA
:10BD60000201D5E904012200E317FEF767F9C5E9EE
:10BD700004015FF00008DDF83C0E00220023C0E95A
:10BD80000023DDF83C0E00220023C0E90223DDF889
:10BD90003C0E00220023C0E9042382E0DDF83C2EA3
:10BDA000D2E90001CDE9000140F68C10684430F979
:10BDB0001800C117D5E90023801A994140F68C126A
:10BDC0006A4432F918A05FEAEA7BD5E90023BAEBAE
:10BDD00002027BEB0303A2FB00AB02FB01BB03FBF4
:10BDE00000BBDDE9000110EB0A0051EB0B01DDF8AF
:10BDF0003C2EC2E90001DDF83C2ED2E90201CDE97A
:10BE00000001FFA8E03030F91800C117D5E902237E
:10BE1000801A9941FFAAE03232F918A05FEAEA7B62
:10BE2000D5E90223BAEB02027BEB0303A2FB00ABD2
:10BE300002FB01BB03FB00BBDDE9000110EB0A00C4
:10BE400051EB0B01DDF83C2EC2E90201DDF83C2E7E
:10BE5000D2E90401CDE900010BA830F91800C1179F
:10BE6000D5E90423801A99410BAA32F918A05FEA98
:10BE7000EA7BD5E90423BAEB02027BEB0303A2FBC6
:10BE800000AB02FB01BB03FB00BBDDE9000110EBD3
:10BE90000A0051EB0B01DDF83C2EC2E9040118F158
:10BEA0000108B045FFF67AAFDDF8400E06600120CC
:10BEB0000DF6446DBDE8F08F2DE9F04389B0040024
:10BEC0000D00160001275FF0000801A800210160A5
:10BED0000320009001AB0022D0210120F6F75BFA8D
:10BEE000002801D15FF0FF375FF0000907E04FFA4B
:10BEF00089F905A8002140F8291019F101094FFA24
:10BF000089F9B9F1030F17DA4FFA89F901A819F87D
:10BF100000000028EBD04FFA89F901A819F80000B9
:10BF2000DFF8F81411EB400030F8020C4FFA89F9F1
:10BF300005A941F82900E0E75FF0000925E04FFA84
:10BF400089F902A850F82900DFF8D414884208DAE9
:10BF5000DFF8D004F6F74FF9012010FA09F050EAA3
:10BF600008084FFA89F902A850F82900DFF8B81438
:10BF7000884208DBDFF8B404F6F73DF9012010FA37
:10BF800009F050EA080819F101094FFA89F9B9F1E5
:10BF9000030F3BDA4FFA89F955F829004FFA89F96E
:10BFA00056F82910401A08F0FFFF4FFA89F902A944
:10BFB00041F829004FFA89F905A850F8290000280E
:10BFC000BDD04FFA89F902A850F829004FFA89F933
:10BFD00005A951F8291090FBF1F0B0F57A7008F03E
:10BFE000E3FF4FFA89F924F819004FFA89F934F977
:10BFF0001900B0F5FA7FC6DDDFF83404F6F7FBF878
:10C00000012010FA09F050EA0808BCE74FFA88F856
:10C01000B8F1000F05D0DFF81C04F6F7ECF87FF05C
:10C020000207380040B209B0BDE8F0832DE9F047BF
:10C030009CB004005FF0010801250CA81821F9F755
:10C04000EFFC06A81821F9F7EBFC02A8002101601B
:10C0500000A80021002206C008385FF0000A18A8D6
:10C060000021002200230EC00C3815A80021002258
:10C0700000230EC00C3812A80021002200230EC09D
:10C080000C3803A80021002200230EC00C38002623
:10C09000DFF8A403D0F80490FEF7EFF9002801D1EF
:10C0A000002049E1FEF7FCFA80465FFA88F8B8F113
:10C0B000010F0AD15FF0010A02AA06A90CA8FFF736
:10C0C0001BFD002805D1002036E1FEF741FA0020D3
:10C0D00032E1FEF7CAFB002801D100202CE1002349
:10C0E00003AA15A90020FEF7FEFB05006DB2012D85
:10C0F00003D0761CD148F6F77EF8002312AA18A9BF
:10C100007FF01F00FEF7EFFB05006DB2012D03D09D
:10C11000B61CCB48F6F76FF818AA15A900A8FFF7C8
:10C12000CBFE05006DB2012D03D0361DC548F6F7D4
:10C1300062F8DDE90601002901D100280BD0DDE914
:10C140000801002901D1002805D0DDE90A010029F4
:10C1500005D1002803D1BC48F6F74DF80836002772
:10C160003AE0FFB20CA810EBC700D0E9002340F280
:10C17000411000218B420FDB01DC82420CD31036D0
:10C18000FFB20CA810EBC702D2E900010200FFB217
:10C190003900AE48F6F72FF8FFB206A810EBC70239
:10C1A000D2E90001029AD317FDF748FF002912DBFC
:10C1B00002DCB0F5C85F0ED34036FFB206A810EB24
:10C1C000C702D2E90001029990FBF1F2FFB23900F7
:10C1D0009F48F6F710F87F1CFFB2032FC1DB36B281
:10C1E000002E1AD100220CE0D2B219EB4203D2B2D7
:10C1F0000CA810EBC206D6E900018000A3F8580095
:10C20000521CD2B2032AEFDBB9F95C30B9F95A20DB
:10C21000B9F958108F48F5F7EEFF84F800A0BDF883
:10C2200000006070BDF900000012A070BDF80200AF
:10C23000E070BDF9020000122071BDF804006071C9
:10C24000BDF904000012A071E571029820720298F5
:10C250000012607202980014A07202980016E07238
:10C26000DDE90C012073DDE90C0100B200126073FE
:10C27000DDE90C010014A073DDE90C010016E07388
:10C28000DDE90E012074DDE90E0100B200126074D8
:10C29000DDE90E010014A074DDE90E010016E07462
:10C2A000DDE910012075DDE9100100B200126075B2
:10C2B000DDE910010014A075DDE910010016E0753C
:10C2C000DDE906012076DDE9060100B200126076A4
:10C2D000DDE906010014A076DDE906010016E0762E
:10C2E000DDE908012077DDE9080100B2001260777E
:10C2F000DDE908010014A077DDE908010016E07708
:10C30000DDE90A0184F82000DDE90A0100B200122B
:10C3100084F82100DDE90A01001484F82200DDE937
:10C320000A01001684F82300FEF712F9002801D153
:10C33000002001E04046C0B21CB0BDE8F08730B537
:10C3400083B004000020ADF8040000203A494D6895
:10C35000697A002907D1286E40688047F5F7C9FE41
:10C360000A21F6F7B3F80220009001AB4122D02158
:10C370000120F6F710F8002801D1002017E09DF801
:10C3800005009DF8041050EA0120032110FB01F084
:10C390004FF47A7190FBF1F015302070002060703E
:10C3A000687A002802D1286E8068804701203EBD4F
:10C3B00080B50178002905D1FFF738FE00280AD1A1
:10C3C000002009E00178012905D1FFF7B8FF002816
:10C3D00001D1002000E0012002BD80B5C0B20628D6
:10C3E00006D10800FFF7ABFF002801D1002000E0D4
:10C3F000012002BD80B518490120F9F7C5F801BD3B
:10C4000057500120685301208C4C0308944C0308BA
:10C410009C4C03082D211FF46C56C53FC034030803
:10C4200030FD1300AC4C030879E2D100B44C030892
:10C43000A44C0308BC4C030808600020C44C03084B
:10C44000CC4C0308D44C0308104C0308404B0308A1
:10C45000D44B0308EC4B0308B44A0308DFF880050B
:10C46000704730B583B00020ADF806008DF80400A9
:10C470000120009001AB002218210220F5F78BFF6C
:10C4800004469DF8040048281FD131208DF806008D
:10C490000DF106050120687002230DF10602182136
:10C4A0001846F5F71EFF00280DD031208DF8060044
:10C4B0000020687002230DF1060218211846F5F7D6
:10C4C00010FF002802D100203EBD002418220021C8
:10C4D000DFF80C05F6F74CFF20463EBD70B582B084
:10C4E0000020ADF8000008F094FD0446DFF8F404E5
:10C4F0008168497AC268527A51180069407A0818EE
:10C50000012801DB012076BDDFF8DC5468780128C2
:10C510001CD032208DF8000000AE01207070022384
:10C5200000AA18211846F5F7DCFE00280CD03120AF
:10C530008DF8000001207070022300AA182118460F
:10C54000F5F7CFFE002803D1002076BD012028702A
:10C55000281D61698847012076BD38B50020ADF8F7
:10C56000000008F056FD0446DFF878048168497A37
:10C57000C268527A51180069407A0818022801DB13
:10C58000012032BDDFF860542878012812D0312014
:10C590008DF8000000208DF80100022300AA182168
:10C5A0001846F5F79EFE002801D1002032BD00207C
:10C5B000687001E000202870281D2169884701204B
:10C5C00032BD80B50020ADF8000031208DF80000AC
:10C5D00000208DF80100022300AA18211846F5F763
:10C5E00080FE002801D1002002BD012002BD7CB5E3
:10C5F00004460020ADF806008DF8040001200090EC
:10C6000001AB002218210220F5F7C5FE05469DF872
:10C610000400482829D131208DF806000DF10606C6
:10C620001F20707002230DF1060218211846F5F73D
:10C6300058FE002817D003200090234660221821BE
:10C640000220F5F7A8FE00280DD031208DF8060055
:10C650000020707002230DF1060218211846F5F72C
:10C6600040FE002802D1002076BD0025284676BD78
:10C670000021DE4A02E00B5C8B54491C1B29FADBCB
:10C68000DB48C0F8D423012070472DE9F04387B080
:10C6900004460D4616461F464FF000084046ADF8CA
:10C6A000040002A841460A460B460EC04FF0050999
:10C6B00006C00120009002AB102218210220F5F7DD
:10C6C0006AFE9DF80810C9070ED501280CD1082074
:10C6D00000900DF10903112218210220F5F75BFEED
:10C6E000002807D140467BE04846A0F1010980B20E
:10C6F0000028DED1BF489DF80810017002A90A7A0F
:10C700004270CA7982704A78C2708A780271CA7897
:10C7100042710A7982714A79C271897901720AE09B
:10C7200002A800EB48008178407810EB012024F843
:10C73000180008F10108B8F1030FF1DBA948D0F89F
:10C740000C8008F10C0999F815202146D9F80C0045
:10C75000D8F80C30C018F7F72AFA404602F05EFA13
:10C7600099F81520D9F80C00D8F80C10411820467B
:10C77000F7F71DFADFF8788205AA2146404608F04F
:10C780009DFE98F9F4023860B8F8EE00288008F2AF
:10C79000EE00418869808188A98081892180C189D2
:10C7A0006180008AA08020882988401A30806088B3
:10C7B0006988401A7080A088A988401AB08031200A
:10C7C0008DF8040001208DF80500022301AA18212C
:10C7D0001846F5F786FD002801D1002000E0012071
:10C7E00007B0BDE8F08330B585B004460020ADF851
:10C7F000040002A800210A460B460EC005250120B0
:10C80000009002AB102218210220F5F7C4FD9DF81C
:10C810000810C9070ED501280CD1082000900DF191
:10C820000903112218210220F5F7B5FD002806D1D1
:10C83000002029E02846451E80B20028DFD16D483F
:10C840009DF80810017002A90A7A42704878207099
:10C8500088786070C878A0700879E0704879207195
:10C860009DF80E00607131208DF8040001208DF8D4
:10C870000500022301AA18211846F5F732FD002809
:10C8800001D1002000E0012005B030BD2DE9F041CC
:10C8900004460025F5F7F4FF0746FFF7DFFD0646DF
:10C8A0005048D0F81080F86E40070BD406F11403FE
:10C8B00006F10C02B11D3046FFF7E7FE002801D15A
:10C8C000284651E098F80A00012848D149480178E3
:10C8D000217041786170C178A1700179E17041796E
:10C8E000217181796171C179A171007AE07140484B
:10C8F000818D2172B0F92C100912617200F12C01A6
:10C900004A88A272B1F902201212E2728A88227356
:10C91000B1F9041009126173B0F8F410A173B0F901
:10C92000F4100912E173F43041882174B0F9021057
:10C93000091261748188A174B0F904000012E074D6
:10C94000284620750FE006EB4500C18804F8151055
:10C9500004EB4501B0F90600001248706D1C032D70
:10C96000F1DB7069A0710120BDE8F081F8B50446E3
:10C970000025F5F785FF0746FFF770FD0646F86EC0
:10C98000000705D52046FFF72EFF002826D109E035
:10C9900006F1140306F10C02B11D3046FFF775FED7
:10C9A000002814D12846F2BD36F8150004F8150009
:10C9B00004EB450036F915100912417006EB4501EC
:10C9C0008A898271B1F90C100912C1716D1C032D95
:10C9D000EADB182231460248F7F7E9F80120F2BDF8
:10C9E000044F012008600020E04F0120B04E0120DC
:10C9F00060F600203C5101207CB504460020ADF8D3
:10CA000006008DF80400F5F774FB05460120009040
:10CA100001AB002218210220F5F7BDFC9DF804109F
:10CA2000482932D131208DF806000DF106061F206D
:10CA3000707002230DF1060218211846F5F751FC1B
:10CA400000281BD031208DF80600002070700223D2
:10CA50000DF1060218211846F5F743FC00280DD009
:10CA600001212846F5F732FD0120009001AB31226B
:10CA700018210220F5F78FFC002801D1002076BD97
:10CA80009DF804002070012076BDFF21217076BD45
:10CA90002DE9F04387B0044604A800210A460B465E
:10CAA0000EC00846ADF80C004FF00509F5F721FB64
:10CAB00005460220009004AB00221821F5F76BFC1C
:10CAC00006469DF81000482840F00B819DF81000A4
:10CAD000207004AF7878607031208DF80C000DF173
:10CAE0000C081F2088F80100022303AA1821184609
:10CAF000F5F7F7FB002800F0F5800320009004AB69
:10CB0000602218210220F5F746FC002800F0EA8098
:10CB10009DF81000A0707878E070B878207131200E
:10CB20008DF80C00002088F80100022303AA1821C8
:10CB30001846F5F7D6FB002800F0D48001200090BD
:10CB400004AB312218210220F5F725FC002800F063
:10CB5000C9809DF81000607531208DF80C0001200F
:10CB600088F80100022303AA18211846F5F7B9FB3B
:10CB7000002800F0B7801E212846F5F7A7FC012009
:10CB8000009004AB102218210220F5F704FC0646A1
:10CB90009DF81000C0070DD5012E0BD10820009084
:10CBA0000DF11103112218210220F5F7F4FB0028E2
:10CBB00006D160E04846A0F1010980B20028DED12C
:10CBC000B87902907879019038790090FB78BA783A
:10CBD00079780FF26C10F5F70EFBB878797811EBD5
:10CBE00000203979FA7812EB0121BA797B7913EBBD
:10CBF000022203461BB21B126371A071084600B2E9
:10CC00000012E0712172104600B200126072A2722E
:10CC10009DF81000E072387A207331208DF80C00F6
:10CC2000102088F80100022303AA18211846F5F7FE
:10CC300058FB002856D01E212846F5F747FC4FF038
:10CC400005090120009004AB102218210220F5F7FD
:10CC5000A2FB06469DF81000C0070ED5012E0CD190
:10CC6000082000900DF11103112218210220F5F780
:10CC700092FB002807D1002035E04846A0F10109C9
:10CC800080B20028DDD1B8790290787901903879A6
:10CC90000090FB78BA7879780FF2C000F5F7ABFA1C
:10CCA000B878797811EB00203979FA7812EB012104
:10CCB000BA797B7913EB022203461BB21B12637312
:10CCC000A073084600B20012E0732174104600B24F
:10CCD00000126074A2749DF81000E074387A207518
:10CCE00000E00026304607B0BDE8F08318B40446E3
:10CCF0000B4611460020032C04D0042C05D0072C31
:10CD000006D008E0184614BC71E4184612BC73E65D
:10CD1000184612BCACE412BC704710B50FF25804B0
:10CD200021460220F8F730FC0FF270010420F8F7DA
:10CD30002BFC21460320BDE81040F8F725BC00007D
:10CD4000474D53312D25642C2025642C2025642C3F
:10CD50002025642C2025642C20256400474D533267
:10CD60002D25642C2025642C2025642C2025642C62
:10CD70002025642C2025640063C40008DDC400085D
:10CD80005BC50008C3C50008000000006DC90008AD
:10CD90000000000091CA0008EDCC000863C4000840
:10CDA000DDC400085BC50008C3C500080000000022
:10CDB0008DC800080000000091CA0008EDCC0008F2
:10CDC0007CB500242046ADF80400F5F792F905463D
:10CDD00020208DF8040001AE20467070022301AAC5
:10CDE000BA210520F5F77DFA002801D1204676BD4D
:10CDF00001212846F5F76AFB641C0120009001AB75
:10CE00002122BA210520F5F7C6FA002801D1002019
:10CE100076BDA4B2B4F5FA7F05DD0FF21C20F5F75C
:10CE2000EAF9002076BD9DF804000006E0D4202039
:10CE30008DF8040002207070034601AABA21052073
:10CE4000F5F74FFA002801D1002076BD012076BD0C
:10CE50001CB504460020ADF804000120009001AB91
:10CE60000F22BA210520F5F796FA002801D10020FB
:10CE700016BD9DF80400BD2834D100F035F8002817
:10CE800001D1002016BD032001E0401E40B2002861
:10CE900007D40FF2BC1151F830108C4201D2002897
:10CEA000F3D120208DF8040001ACA420607002238F
:10CEB00001AABA210520F5F714FA002801D10020B3
:10CEC00016BD10208DF804007F206070022301AA97
:10CED000BA210520F5F705FA002801D1002016BD7A
:10CEE000012016BD002016BD80B50020ADF8000061
:10CEF00020208DF8000000208DF80100022300AAF8
:10CF0000BA210520F5F7EDF9002805D10FF2301010
:10CF1000F5F771F9002002BD012002BD80B58F2018
:10CF2000FFF796FF002801D1002002BD012002BDBD
:10CF300080B5FFF745FF002805D10FF20C10F5F77B
:10CF40005AF9002002BD012002BD80B5FFF7E6FFBF
:10CF5000002801D1002002BD012002BD80B5FFF7ED
:10CF6000C3FF002801D1002002BD012002BD012025
:10CF70007047012070471FB5044601A800210A46EA
:10CF80000B460EC00120009001AB0F22BA210520F4
:10CF9000F5F701FA002821D09DF80400BD281DD125
:10CFA0000520009001ABA822BA21F5F7F4F900287A
:10CFB00001D1002013E09DF80400207001A8417801
:10CFC00061708178A1700021E170C17821710079D0
:10CFD0006071E01C00F006F8012000E0002004B0C1
:10CFE00010BD00004178007840EA01204FF4F07154
:10CFF00090FBF1F000EE100AB8EEC00ADFED070A70
:10D0000030EE200ABDEEC00A10EE100A80B20449CC
:10D010000870000A487001207047000000002A4292
:10D020006453012001207047012070470FF2400136
:10D030000520F8F7A9BA000042522D524600000020
:10D0400042522D434600000042522D50460000003F
:10D050002800000070000000500000006000000088
:10D060008F00000050000000E803000010000000E6
:10D0700031CF00084BCF00085DCF00086FCF00080C
:10D0800073CF000877CF00080000000025D000080B
:10D0900029D0000800207047012070470120704708
:10D0A00038B504460D46F5F724F80521F5F70EFAD4
:10D0B0000020104904E00A680255521C0A60401C16
:10D0C000A842F8DB012032BD0120704701207047E3
:10D0D000094802680A704A70511C016001207047BB
:10D0E00006490A6802704270501C086001207047AF
:10D0F00000000000F8870020E0520120E4520120E7
:10D100000FF234010820F8F73FBA10B50FF22804E7
:10D1100021461220F8F738FA21461320F8F734FA9E
:10D1200021461420BDE81040F8F72EBA0FF208018E
:10D130001520F8F729BA000095D0000899D000080A
:10D140009DD000089DD00008CDD00008A1D00008D7
:10D15000C9D00008E1D00008D1D0000810B50024E3
:10D16000F4F7C7FF007CC00700D50124204610BD9E
:10D1700000B589B000A82421F8F752FC0020ADF8D2
:10D1800022000A208DF8080000208DF809008DF893
:10D190000A008DF800001F20019000A8FBF7ACFCEE
:10D1A000012009B000BD00B589B000A82421F8F71E
:10D1B00037FC0020ADF822000A208DF8080000207E
:10D1C0008DF809008DF80A0001208DF800001F205D
:10D1D000019000A8FBF790FC012009B000BD00B54C
:10D1E00089B000A82421F8F71BFC0020ADF822002C
:10D1F0000A208DF8080000208DF809008DF80A003B
:10D2000001208DF800001F20019000A8FBF774FC9E
:10D21000012009B000BD0120704710B50024F4F7CB
:10D2200068FF007CC00700D50124204610BD00B572
:10D2300089B000A82421F8F7F3FB0020ADF8220004
:10D240000A208DF8080000208DF809008DF80A00EA
:10D250008DF800002020019000A8FBF74DFC012074
:10D2600009B000BD00B589B000A82421F8F7D8FBAB
:10D270000020ADF822000A208DF8080000208DF86B
:10D2800009008DF80A0001208DF80000202001908F
:10D2900000A8FBF731FC012009B000BD00B589B042
:10D2A00000A82421F8F7BCFB0020ADF822000A20DA
:10D2B0008DF8080000208DF809008DF80A00012083
:10D2C0008DF800002020019000A8FBF715FC01203C
:10D2D00009B000BD0120704710B50024F4F709FF24
:10D2E000007C800700D50124204610BD00B589B020
:10D2F00000A82421F8F794FB0020ADF822000A20B2
:10D300008DF8080000208DF809008DF80A008DF8CE
:10D3100000002120019000A8FBF7EEFB012009B0DE
:10D3200000BD00B589B000A82421F8F779FB0020E2
:10D33000ADF822000A208DF8080000208DF80900C1
:10D340008DF80A0001208DF800002120019000A82E
:10D35000FBF7D2FB012009B000BD00B589B000A8E1
:10D360002421F8F75DFB0020ADF822000A208DF89B
:10D37000080000208DF809008DF80A0001208DF8C2
:10D3800000002120019000A8FBF7B6FB012009B0A6
:10D3900000BD0120704710B50024F4F7AAFE007C00
:10D3A00000F00300032800D10124204610BD00B581
:10D3B00089B000A82421F8F733FBDFF86C0301786B
:10D3C00041F0020101700020ADF822000A208DF822
:10D3D000080001208DF809008DF80A1000208DF852
:10D3E00000002220019000A8FBF786FB012009B075
:10D3F00000BD00B589B000A82421F8F711FBDFF8C3
:10D400002813087810F0FD00087014D10020ADF842
:10D4100022000A208DF8080001208DF80900002064
:10D420008DF80A0001208DF800002220019000A84C
:10D43000FBF762FB02E040B208F0CAFC012009B031
:10D4400000BD012070470120704710B50024F4F79B
:10D4500050FE007C00F00700072800D10124204680
:10D4600010BD00B589B000A82421F8F7D9FAAE495B
:10D47000087840F001000870032805D140B208F098
:10D48000A7FC08F0C1FC12E00021ADF822100A212F
:10D490008DF8081000218DF809108DF80A00084653
:10D4A0008DF800002220019000A8FBF725FB012049
:10D4B00009B000BD00B589B000A82421F8F7B0FA82
:10D4C0009949087810F0FE00087013D10020ADF8DB
:10D4D00022000A208DF8080000208DF809008DF840
:10D4E0000A0001208DF800002220019000A8FBF71F
:10D4F00003FB04E040B208F06BFC08F08AFC01205A
:10D5000009B000BD012070470120704710B500240C
:10D51000F4F7EFFD007CC00700D50124204610BDC4
:10D5200030B58BB001A82421F8F77AFA00200090DA
:10D530007E48446C0020ADF826000A208DF80C00CF
:10D5400000208DF80D008DF80E008DF804002320CA
:10D55000029001A8FBF7D0FA0020009004F10C051E
:10D560006A7D00A9E868E368C018F6F720FB01208F
:10D57000A874002008F003FD03F0E7FC01200BB0C5
:10D5800030BD00B589B000A82421F8F749FA002081
:10D59000ADF822000A208DF8080000208DF809005F
:10D5A0008DF80A0001208DF800002320019000A8CA
:10D5B000FBF7A2FA012009B000BD00B589B000A8B0
:10D5C0002421F8F72DFA0020ADF822000A208DF86A
:10D5D000080000208DF809008DF80A0001208DF860
:10D5E00000002320019000A8FBF786FA012009B073
:10D5F00000BD01207047000070B58AB004460E4699
:10D60000FBF78AF90546002000900422214600A875
:10D61000F6F7CDFA01A82421F8F702FA009A31466C
:10D620000FF2C010F4F7E7FD30460C3809284ED849
:10D63000DFE800F0051118253C0C4D4D4D48142035
:10D64000C5F8DC04207001200AB070BD1420C5F8B4
:10D650007C052070F7E705F2DC403C21816208463A
:10D660002070F0E705F2DC4021783C2904D13C2110
:10D67000217021780165E6E700990165E3E72A4812
:10D680000078C10712D50021ADF826100A218DF8C7
:10D690000C1000218DF80D108DF80E0001208DF872
:10D6A00004002220029001A8FBF726FA00993046D8
:10D6B00040B200F012F80090206005F2DC400099C2
:10D6C0008167C0E71420C5F8BC062070BBE70FF2E5
:10D6D0002410F4F790FD0020B6E710B4134AD36B82
:10D6E000126C114C2478002C1AD00F2802D010286C
:10D6F0000BD015E0507A002812D0906B806800287B
:10D700000ED488420DDD08460BE0587A002807D079
:10D71000986B8068002803D4884202DD084600E048
:10D72000084610BC704700006A53012008600020C2
:10D7300012B589B001460C3909292CD8DFE801F06F
:10D74000051F2123231D2B2B2B291F240020ADF87F
:10D75000220001900A208DF8080005208DF80000B5
:10D760000194042209A90DF10900F6F720FA00A896
:10D77000FBF7C2F901200AB010BD2324E6E72024FC
:10D78000E4E72124E2E722240999FFF7A6FF0990A4
:10D79000DCE72B24DAE70FF26400F4F72CFD00201D
:10D7A000E9E780B50FF25C010C20F7F7EDFE0FF210
:10D7B00078011120F7F7E8FE0FF290010D20F7F73E
:10D7C000E3FE0FF2AC010E20F7F7DEFE0FF2C4010C
:10D7D0000F20F7F7D9FE0FF2E0011020BDE804405A
:10D7E000F7F7D2BE4D52322044523D25642C2564B9
:10D7F000000000004D523220534446004D5232206A
:10D80000524346005DD1000871D10008A7D100083D
:10D81000DFD100080000000017D20008F9D5000889
:10D8200000000000000000000DD5000821D5000810
:10D8300083D50008BBD5000800000000F3D5000820
:10D84000F9D5000800000000000000001BD200080D
:10D850002FD2000865D200089DD200080000000009
:10D86000D5D20008F9D50008000000000000000033
:10D87000D9D20008EDD2000823D300085BD30008FA
:10D880000000000093D30008F9D500080000000054
:10D890000000000097D30008AFD30008F3D30008BE
:10D8A00043D400080000000047D40008F9D5000860
:10D8B00000000000000000004BD4000863D4000802
:10D8C000B5D4000805D500080000000009D50008FF
:10D8D000F9D50008000000000000000000B500BFFE
:10D8E000130096469446103928BFA0E80C50FAD889
:10D8F0005FEA417C28BF0CC048BF40F8042BC90731
:10D9000028BF20F8022B48BF00F8012B00BD000003
:10D910002DE9F04FA1B0824602AE002017461D4609
:10D92000029170620DF144080AE017F8011B029899
:10D93000D0470290002800F0DA82706A401C7062C2
:10D94000387808B9706AD4E22528EED10020F0605A
:10D9500030617061B061F061306201E040F001005F
:10D9600017F8011F2029F9D023290DD02B2904D025
:10D970002D2906D030290AD00CE040F0020080B2F8
:10D98000EEE740F00400FAE740F00800F7E740F067
:10D990001000F4E72A290DD129680A1D2A600968B8
:10D9A000F162002904D5494240F00400F16280B2DE
:10D9B0007F1C13E00021F1620BE0F16A6FF000437D
:10D9C000994205D001EB810302EB43013039F1624A
:10D9D0007F1C3A78A2F130010A29EED339782E293A
:10D9E00003D04FF0FF31B1621EE017F8011F2A2962
:10D9F00006D129680A1D2A607F1C0968B16213E0FC
:10DA00000021B1620BE0B16A6FF00043994205D08A
:10DA100001EB810302EB43013039B1627F1C3A789C
:10DA2000A2F130010A29EED330860FF66040397832
:10DA300008F0E2FA08B117F8010B8DF83A009DF8EA
:10DA40003A00682802BF39786829622005D06C281E
:10DA500004BF38786C2803D171208DF83A007F1C00
:10DA600011A8B0603978B1F1250029D01C3800F038
:10DA7000C080001F022840F2BC80133800F0E48010
:10DA8000093800F0B680801E00F07781401E00F05B
:10DA90002081401E022840F2AC80001F00F0198156
:10DAA000401F7BD0401E00F0CF80401E22D0C01E01
:10DAB0000BD0801E00F0C880C01E00F0C58064E15D
:10DAC000F068411CF160252169E12868011D296089
:10DAD0000068B26A7060002A02D5F7F7C7FF07E056
:10DAE000002108F095FA00281ABF7168401AB06A40
:10DAF000306156E12868011D296000210068CDE9E8
:10DB000000014FF03C0E11A87060DDE9000111B971
:10DB100008B9B26ACAB10206120FA0EB0212303283
:10DB2000AEF10103D2B29E463A2AA8BF27320009BD
:10DB300003F8082040EA0170090908BF002804D052
:10DB4000726811AB73449A42E5D311A971447160B4
:10DB5000CEF13C00B16A3061884207DA081AB06140
:10DB60004FF6EF71308E084030861AE1002940F1FF
:10DB7000188196F8301001F01401102940F011813D
:10DB8000F16AF268891AB269891AA1EB000EBEF136
:10DB9000010FC0F20681C6F818E002E19DF83A00D4
:10DBA000622818D0682806D06A280BD06C2819D0B3
:10DBB000712807D016E02868011D29600068716A85
:10DBC0000180EEE02A68101D28601268706AC11793
:10DBD000C2E90001E5E02868011D29600068716A5A
:10DBE0000170DEE02868011D29600068716A01602B
:10DBF000D7E02868C01D20F00700286000F1080267
:10DC00002A60D0E90023CDE90023002B04D5F06879
:10DC1000421CF2602D220DE0308E820704D5F068A0
:10DC2000421CF2602B2205E0C00705D5F068421CBB
:10DC3000F260202200F80820F06811AA80187060B5
:10DC400000A800F0E3F9ACE09DF83A006C2808BFAA
:10DC50002A6811D0712808BF2A6802D02A686A2869
:10DC60000AD1D21D22F007022A60144604F10802EC
:10DC70002A60D4E9002303E0131D2B6000231268FF
:10DC8000CDE90023682808BF92B207D0622808BFF8
:10DC9000D2B203D0742818BF7A2802D10023CDE96C
:10DCA000002396F8300000075FD5DDE90023002B44
:10DCB00008BF002A59D041F02000782855D1F068DB
:10DCC000302200F80820401C421CF26000F80810C6
:10DCD0004BE09DF83A0062280CD0682810D06A28E2
:10DCE0001AD06C2823D0712816D074281FD07A2817
:10DCF0000CD01CE02868021D2A6090F900201AE070
:10DD00002868021D2A60B0F9002014E02868021D6E
:10DD10002A60002302680FE02868C01D20F0070079
:10DD2000286000F108022A60D0E9002304E0286896
:10DD3000021D2A600268D317CDE90023002B04DA04
:10DD4000F068421CF2602D220DE0308E820704D56F
:10DD5000F068421CF2602B2205E0C00705D5F06890
:10DD6000421CF260202200F80820F06811AA8018F6
:10DD7000706000A800F0C0F813E0F068411CF1608A
:10DD800029680A1D2A60096809E0F068421CF260EF
:10DD9000252200F8082021B1F068421CF26000F84A
:10DDA0000810F06AF168401AB169401A3169401AE6
:10DDB000F169401A7169401A316AA0EB010996F8BD
:10DDC00030007F1C400710D420208DF84000002434
:10DDD00009E0012310AA00A9504600F040FC0028E9
:10DDE00040F08580641C4C45F3DBF4680DF1440B76
:10DDF0000AE01BF8011B0298D0470290002876D059
:10DE0000706A401C7062641E002CF2D130208DF8C4
:10DE100040004FF0000BB46909E0012310AA00A9EB
:10DE2000504600F01CFC002861D10BF1010BA3450A
:10DE3000F3DB3469D6F804B00AE01BF8011B029842
:10DE4000D0470290002852D0706A401C7062641E55
:10DE5000002CF2D130208DF840004FF0000BF46917
:10DE600009E0012310AA00A9504600F0F8FB0028A1
:10DE70003DD10BF1010BA345F3DB30697168746987
:10DE800000EB010B09E01BF8011B0298D047029040
:10DE900068B3706A401C7062641E002CF3D130209D
:10DEA0008DF840004FF0000B346A08E0012310AAFF
:10DEB00000A9504600F0D3FBC8B90BF1010BA345F4
:10DEC000F4DB96F8300040077FF53AAD20208DF85E
:10DED0004000002400E0641C4C45BFF631AD012336
:10DEE00010AA00A9504600F0BAFB0028F3D04FF06A
:10DEF000FF3021B0BDE8F08F2DE9FA47064682B029
:10DF000035690A466F2A08BF082705D041F020006E
:10DF1000782814BF0A271027D6E900013C24804640
:10DF20008946642A18BF692A05D1002903DAD8F185
:10DF3000000869EB4909B9F1000F08BFB8F1000FFB
:10DF40000CD1306B50B9082F3BD196F83800000740
:10DF500037D530203B2485F83B0032E0CDE90089FD
:10DF6000FB17404649463A46FCF78AF8B846A8FBF4
:10DF70000023DDE90089A8EB02023032A4F1010A96
:10DF8000D2B254463A2A03DB9DF80830513B9A1826
:10DF90000AF8052080465FEA010908BFB8F1000FC2
:10DFA00003D0F06861198842D8D3082F09D196F8B8
:10DFB0003800000705D5605D302802D0641E30208F
:10DFC0006055C4F13C00B0616119F160316B884269
:10DFD00007DA081A30624FF6EF71308F0840308749
:10DFE00010E000290ED596F8381001F01401102920
:10DFF00008D1716B7269891A326A891A081A012864
:10E00000A8BF306204B0BDE8F08700002DE9F24FF0
:10E0100004468EB0D4E90001CDE9020104AE9DF8BA
:10E02000380040F02000009061280AD0206B0028C2
:10E0300048BF062004D404BF0098672801D10120FE
:10E0400020636168C1F30A5040F2FF7290421CD114
:10E05000080304BF2068002809D10320A0619DF8AF
:10E06000380061381A2836D30FF2346108E00320F3
:10E07000A0619DF8380061381A2829D30FF2186181
:10E08000E0680322F5F758FDB5E1012816DA2046CD
:10E0900007F0EAFF012811DB002700200099612921
:10E0A00020D1E168302201F8012B4A1CE2609DF882
:10E0B0003820612A0CBF782258220FE0626840F2B3
:10E0C000FE3161F31E52471A62604FF0FF30E5E700
:10E0D0000FF2C051D4E70FF2C451D1E70A70616961
:10E0E000891C616110B9002500277BE10098612837
:10E0F00040F09680206B00284CBF2125451CDDE9AF
:10E1000002012DB26E1CD4E900890022002307F021
:10E11000CDFF3ABF89F00040CDE90280CDE9028908
:10E120003F1F8DF810200DF1110801E000F20708E3
:10E13000012E32DBDDE902010022002307F0CEFFD1
:10E140002BD21C2102A807F0E1FFDDE9020106F055
:10E150002FFFF61F8146012E09DBFAF70BFE024660
:10E160000B46DDE9020108F05BF8CDE9020108F297
:10E170000700072105E009F00F0200F8012D4FEA22
:10E180002919B9F1010F01DB491EF4D5491E5CBF05
:10E19000002200F8012DF9D5C8E70DF11100A8EB18
:10E1A00000010DF11106A942B8BF0D462DB228009D
:10E1B0002FD4884206DA04A9411849780829A8BF53
:10E1C0000F2100DA002104AA821800E06D1E12F867
:10E1D0000139401E8B42F9D00F2904D104A94118FE
:10E1E0004A78521C4A70002802D504AE6D1C3F1DAF
:10E1F0002DB2681E0DD481190A783032D2B23A2A73
:10E2000003DB9DF838303A3B9A1801F80129401E8B
:10E21000F2D5206B002840F1E580681E2063E1E024
:10E22000DDE902010022002307F040FF3CBF81F03E
:10E230000041CDE902013FB247F297507843484987
:10E24000DFF820B190FBF1F73FB2C7F10706924625
:10E25000012E19DBDDE90289F00707D552465B463E
:10E2600040464946FAF79EFD80468946761050465C
:10E27000594652465B46FAF795FD82468B46002E7C
:10E28000EAD1CDE9028921E076429046DFF8D890C4
:10E2900012E0F00707D552465B4640464946FAF77A
:10E2A00081FD8046894676105046594652465B4667
:10E2B000FAF778FD82468B46002EEAD1DDE90201AD
:10E2C00042464B4608F06CF8CDE9020100986628FA
:10E2D0000CBF07F10A000620216B4518142DA8BFBA
:10E2E000132530208DF810000DF11106DFF87C9019
:10E2F000012D3DDBDDE9020106F070FE06F10801AB
:10E3000004220A23B0FBF3F303EB8306A0EB4600E1
:10E31000303001F8010D0A20B3FBF0F000EB80066D
:10E32000A3EB4603303301F8013D521EE9D1083D0D
:10E3300001F10806012DDBDBDDE9020106F04EFEEE
:10E34000FAF722FD02460B46DDE9020107F068FFFD
:10E3500000224B46FAF726FDCDE90201CAE700BFCD
:10E36000A0860100000024400000F03F84D79741C0
:10E370000DF11100301A0DF1110602E0401E7F1E52
:10E38000761C31783029F9D00099662902D13FB244
:10E39000791C03E065290CBF01210021226B8D1837
:10E3A0002DB2A842B8BF05462DB229001AD4814229
:10E3B00004DA885D3528A8BF392000DA30208A19B0
:10E3C000521E00E06D1E12F80139491E8342F9D039
:10E3D000392802D1885D401C8855002902D5761E57
:10E3E0006D1C7F1C3FB29DF8381000972BB232464F
:10E3F000204600F003F80FB0BDE8F08F2DE9F043A0
:10E40000054685B01E46D5F8308089461746012E50
:10E4100002DA01260FF28C2749F02000BDF93040C6
:10E42000662808BF641C17D0672840F0818014F16B
:10E43000040FC0F28380444580F2808095F8380054
:10E44000641C000702D44645B8BFB04624B2B8EBFE
:10E45000040848BF4FF00008E868A96924B2012CFD
:10E4600025DA30234A1C0B54B8F1010F03DA95F872
:10E470003810090702D52E211154521CAA6118EB3D
:10E48000040FB8BFC8F1000424B26142A04469621D
:10E49000B045B8BF464636B2EE613246AB69394642
:10E4A0001818F5F749FBA8EB0600A862C0E00818A9
:10E4B000A64218DA32463946F5F73EFBA9697118CB
:10E4C000A961A01B6862B8F1010F03DA95F8380062
:10E4D000000705D5E8682E220A54E869401CE86167
:10E4E000C5F82880A4E022463946F5F725FBA8693F
:10E4F0002018361BB8F1010F03DA95F83810090718
:10E5000003D5E9682E224254401C36B2A861B045BA
:10E51000B8BF4646EB6836B23246E119C018F5F787
:10E520000BFBA8693018A861A8EB060068627FE0C1
:10E53000B9F1610F16D14FF0700918E0464504DAC1
:10E5400095F83810090758BFB046B8F1010848BF20
:10E550004FF00008B9F1670F14BF4FF045094FF0B5
:10E56000650904E0B9F1410F08BF4FF05009A969EE
:10E57000E86817F8013B0B544A1CB8F1010F05DAA3
:10E5800095F83810090758BFAA6117D52E211154E4
:10E59000531CAB61B8F1010F10DB761E36B2B045EB
:10E5A000B8BF464636B2324639461818F5F7C4FAAF
:10E5B000A8693018A861A8EB06006862A869E96834
:10E5C0004718200007F8019B03D42B2007F8010B04
:10E5D00003E02D2107F8011B644200260DF1080815
:10E5E00008E00A2200A807F0FEFF019808F8010BD6
:10E5F000761C009C21B20129F3DA022E06DA49F0DA
:10E600002000652804BF302007F8010B4EB93020E8
:10E6100007F8010B07E0761E02A8305C303007F8DF
:10E62000010B012EF7DAA869E9684018381AE86189
:10E6300095F8380000F0140010280DD16869A96918
:10E640000818696A0818E9690818A96A0818696B3E
:10E650008842BCBF081A286205B0BDE8F083F8B54F
:10E6600004460D4616461F46002004E0E86A401C9A
:10E67000E8627F1E002047B116F8011BA868A0477A
:10E68000A8600028F2D14FF0FF30F2BD686A6C74C8
:10E690007A4C00006E616E004E414E00696E66005D
:10E6A000494E4600300000000CB41CB5044604A8D6
:10E6B00001900A46009401AB00A90748784418303D
:10E6C000FFF726F9009900220A7000285CBF009825
:10E6D000001B16BC5DF80CFB4F73FFFF01B58B07E9
:10E6E00018D1121F21D351F8043BA3F1013C2CEAAD
:10E6F000030C1CF0803C04BF40F8043BF1E79CFA9B
:10E700008CFCBCFA8CF1C1F118018B40CB4040F875
:10E71000043B13E0042A09D311F8013B521E00F810
:10E72000013B5BB18B07F7D1DBE7121D5AB111F842
:10E73000013B521E00F8013B03B1F8D111001CBF90
:10E740000022FAF775FC01BD002801D10A48806853
:10E7500090F84C10642901D0002000E0806A7047D6
:10E76000002801D10448806890F84C10642901D039
:10E77000002000E0406A7047CC86002002487047C5
:10E7800002480149401A7047000000200020002084
:10E790004C48C168002903D54B4901604B490160D1
:10E7A00070474B48016841F000410160704770B507
:10E7B0000446002600290BD0012902D14FF48076AF
:10E7C00006E0022902D14FF4007601E04FF44076D2
:10E7D00000F082F809281ED13D4D286820F44070D1
:10E7E0002860286830432860286820F0F8002860F6
:10E7F000286844F0020108432860286840F480300B
:10E80000286000F069F8296821F002012960296870
:10E8100021F0F801296070BD70B504460D4600F086
:10E820005BF8092813D12A4E306820F4407030601C
:10E83000306840F400703060306840F001003060B3
:10E84000256000F049F8316849084900316070BD21
:10E8500070B505460E4600F03FF8092811D11C4C52
:10E86000206820F44070206020682060206840F01C
:10E87000010020602E7000F02FF82168490849003F
:10E88000216070BD134908607047092011490A686A
:10E89000D20301D5012070470A68D20601D50620AF
:10E8A00070470A68D20501D5022070470A6812F045
:10E8B000EF0F01D0072070470968890700D50820AD
:10E8C00070470000043C024023016745AB89EFCD4F
:10E8D000103C02400C3C024080B509208DF800003D
:10E8E000FFF7D3FF8DF8000003E0FFF7CEFF8DF8B0
:10E8F00000009DF800000128F7D09DF8000002BD3F
:10E900000901002806D500F00F004C4A801800F8D5
:10E91000041C70474A4A8154704710B5401EB0F13C
:10E92000807F01D3012010BD464C60600F214FF065
:10E93000FF30FFF7E5FF0020A060072020600020E7
:10E9400010BD38B5404D2878401C28703F4C2078C9
:10E95000401C2070F7F74BFF07F04CFE2878411E53
:10E960002970002802D19820F7F79CF82078012818
:10E9700004D16068002801D0F7F7F7F82078401E2E
:10E98000207031BD10B5314C6078F021084202D0C2
:10E990009920F7F787F8F7F7F2F86078401C607075
:10E9A00007F082FE2A4800684FF47A71B0FBF1F05C
:10E9B000FFF7B3FF002800D0FEE726482649016094
:10E9C0000E214FF0FF30FFF79BFF6078F0210842E7
:10E9D00002D09920F7F766F86078401E6070C0B2E8
:10E9E000002803D1BDE81040F7F7C3B810BD000000
:10E9F00010B51A4C4FF4005120464183C04630BF39
:10EA00004FF400512046FAF7E7FCF3E710B40F4843
:10EA1000006A0F4909684FF47A72B1FBF2F1104AAB
:10EA20001368CB1A0F4C2468640102D512688B1A44
:10EA3000401C00FB013010BC7047000018ED00E0E6
:10EA400000E400E010E000E091530120CC860020BB
:10EA50008087002008ED00E0000000080010024060
:10EA600018E000E004ED00E0EFF30580002847F037
:10EA70007B86704780B5EFF3108072B60B4909684A
:10EA800051F47F01094A116080F31088084800683A
:10EA900010F4700F02D1A720F7F704F805485FF0D3
:10EAA0000071016004480021016001BD20ED00E01B
:10EAB00088ED00E03CEF00E034EF00E080B5F3F7D4
:10EAC000DFFEDFF874180860012002BD80B5F6F79C
:10EAD0001DFADFF86818D1E90023801A02BDF8B5E5
:10EAE0000446A069E1684518B5F90000B5F902705F
:10EAF000B5F90460B4F9581094F90820012A2AD114
:10EB0000B5EE000A00EE901AF8EEE00A60EE800A18
:10EB1000FDEEE00A10EE901A411A2980B4F95A105D
:10EB200000EE901AF8EEE00A60EE800AFDEEE00AD0
:10EB300010EE901A791A6980B4F95C1000EE901A00
:10EB4000F8EEE00A20EE800ABDEEC00A10EE101AC0
:10EB5000711AA98009E0411A2980B4F85A10791A6B
:10EB60006980B4F85C10711AA980B5F90010C91356
:10EB7000B1EBE03F13D0B4F95810C913B1EBE03F4B
:10EB80000DD00FF2D470F3F736FBB5F90000012871
:10EB900002DBDFF8AC0701E047F6FF702880B5F92B
:10EBA0000210C913B1EBE73F13D0B4F95A10C913DF
:10EBB000B1EBE73F0DD00FF2AC70F3F71CFBB5F9EA
:10EBC0000200012802DBDFF8780701E047F6FF705A
:10EBD0006880B5F90410C913B1EBE63F13D0B4F95E
:10EBE0005C10C913B1EBE63F0DD00FF28470F3F760
:10EBF00002FBB5F90400012802DBDFF8440701E05D
:10EC000047F6FF70A88094F90800002804D100207E
:10EC100000E0401C0328FCDBF1BD0000FEB504460B
:10EC200000A800210A460B460EC0A069E1684518FD
:10EC3000174694F90860052E80F09A80012E02D1C3
:10EC40002046FFF74CFF3046012802D9C01E40F095
:10EC50008A80002E01D14FF6FF77DFF8DC060068CE
:10EC6000301890F88400401E06285ED8DFE800F0D7
:10EC700004101D2936424F00B5F90200009000A88B
:10EC8000B5F90010791A4160B5F90410816056E0B9
:10EC9000B5F90000381A009000A8B5F90210791AE9
:10ECA0004160B5F90410816049E0B5F90200381AF5
:10ECB000009000A8B5F900104160B5F9041081601A
:10ECC0003DE0B5F90000381A009000A8B5F902102F
:10ECD0004160B5F90410791A816030E0B5F902009D
:10ECE000009000A8B5F900104160B5F90410791A38
:10ECF000816024E0B5F90000009000A8B5F9021089
:10ED0000791A4160B5F90410791A816017E0B5F9F4
:10ED10000200381A009000A8B5F90010791A416075
:10ED2000B5F90410791A816009E0B5F90000009086
:10ED300000A8B5F902104160B5F904108160012EF8
:10ED40000AD1002106E050F8212002F30F0240F81A
:10ED50002120491C0329F6DB0098288000A841687F
:10ED600069808068A880002E02D12046FFF7B7FE98
:10ED70000120FEBD70B52DED028B82B08169C268A5
:10ED80008A1890F9081008460A2800F29880DFE8EF
:10ED900000F0062B73969665969696808E00B2F9D3
:10EDA0000240B2F90450DFF8900500689FEDB40A04
:10EDB000B2F9001000EE901AF8EEE00A60EE800A58
:10EDC000C0ED000A00EE904AF8EEE00A60EE800A1C
:10EDD000C0ED010A00EE905AF8EEE00A20EE800A3B
:10EDE000001D80ED010A6EE0B2F90240B2F9045054
:10EDF000DFF844050068061D9FEDA28BB2F9000004
:10EE000000EE100AB8EEC00A10EE100AFAF79CF8ED
:10EE100053EC182BF9F7C6FFFAF7BEF8B06000EE16
:10EE2000104AB8EEC00A10EE100AFAF78DF853EC4B
:10EE3000182BF9F7B7FFFAF7AFF8F06000EE105AA9
:10EE4000B8EEC00A10EE100AFAF77EF853EC182B51
:10EE5000F9F7A8FFFAF7A0F8306134E0002000903D
:10EE6000106800909DED000ABAEECA0ADFF8C804E7
:10EE7000006880ED0C0A26E0DFF8BC040068118809
:10EE8000A0F85A1000F25A00518841809188818080
:10EE900019E0DFF8A404006800F25A001188C1806C
:10EEA0005188018191884181D18881810BE0DFF80F
:10EEB0008804006892F9001080F8681003E00FF2EF
:10EEC000BC40F3F798F9012002B0BDEC028B70BD95
:10EED00070B50D46DFF86C1451F820400026207FF5
:10EEE000002801D1304670BD607A002803D0206E22
:10EEF0008068804706462846216EC96988470546CE
:10EF0000002E02D0206E40688047284670BD012048
:10EF10007047F0B4002A1ED400F11004A57C0669E5
:10EF200092FBF1F76F43B74202DAA263E26304E0B7
:10EF300096FBF5F25143A163E163216C002902D5F0
:10EF4000E26B511AE163E16BDFF8EC231268D2F84F
:10EF500080205118E163002B03D4990701D51030AC
:10EF60000374F0BC7047002904D40021816441611E
:10EF7000816181777047042817D101F10C008A7AEA
:10EF8000012A09D0072242750B228275DFF8B823C7
:10EF9000CA600B21416070471522427519228275A3
:10EFA000DFF8A823CA601921416070472DE9F243B8
:10EFB000804614461A46C146B9F1160F46D2454658
:10EFC000DFF8800350F825600227307F00283DD00D
:10EFD0000846C82802D1B420009003E0422801D19D
:10EFE0003C2000909DF92030002B06D4D80704D592
:10EFF00000993046FFF78BFF3FE000993046FFF75E
:10F0000088FFA9F10C00062805D24146C9B200A824
:10F01000326E9269904731464046FFF7ACFF707AF6
:10F0200000281BD1214649B23046726E12689047C3
:10F0300000280DD0306E40688047002804D1394642
:10F040004F1EC9B20029F5D1002801D1002014E0DB
:10F05000214649B23046726E52689047707A401C21
:10F0600070720D2D08D0224652B200993046736E50
:10F070001B69984700F0C9F80120BDE8F283000041
:10F0800060F61C3A89AD84FA0A74513F2DE9F843C1
:10F0900007460C4615461E46162F08D2A94850F8BA
:10F0A00027804FF0020998F81C00002801D10020A9
:10F0B00047E0C82C01D1B42402E0422C00D13C240A
:10F0C00098F8090001281BD1294649B24046D8F8D2
:10F0D00064209268904700280BD0D8F860008068C0
:10F0E0008047002805D14846A0F10109C0B2002898
:10F0F000F3D1294649B24046D8F86420D2689047F7
:10F1000098F80900002802D0401E88F80900002D58
:10F110000AD10020C8F8480098F80900002803D157
:10F1200031464046FFF71FFF0D2F09D02A4652B245
:10F1300021464046D8F864305B69984700F065F88E
:10F140000120BDE8F2832DE9F84304460D4616463A
:10F150001A462746162F26D27A4951F8208098F869
:10F160001C1000291FD0C82D01D1B42502E0422D6A
:10F1700000D13C250D2801D1012044E09DF920302B
:10F18000002B07D4D80705D52946404601B0BDE875
:10F19000F043BCE606EB460008EB8009D9F83800DE
:10F1A0008068002801D500202DE029464046FFF761
:10F1B000B0FED9F838008068854217D0012D15DBE4
:10F1C0000FF2C410F3F717F8324652B2D9F83800EC
:10F1D00081684046D8F864305B699847324652B23D
:10F1E00029464046D8F864301B699847A7F10C00BF
:10F1F000062805D229462046FEF79AFA012002E0A9
:10F2000000F003F80120BDE8F28370B56FF000460E
:10F2100034464F48016804E08A68A24200DA144686
:10F2200009688142F8D14B4D2878401C28706878D5
:10F23000F021084202D09920F6F734FCF6F79FFC43
:10F240006878401C6870B44200D100243A4E30689F
:10F25000C467D0F8802021468A4212D0002901D00C
:10F26000002A0BD1C0F880100FF22C10F2F7C3FF68
:10F270003068D0F88000F2F79AFF02E0012007F032
:10F2800099FA6878F021084202D09920F6F70AFC32
:10F290006878401E6870C0B2002801D1F6F769FC9A
:10F2A000F7F7C1FA012070BD38B50546294C207822
:10F2B000401C20706078F021084202D09920F6F7B7
:10F2C000F1FBF6F75CFC6078401C607029460FF299
:10F2D000DC00F2F790FF18480068C0F880501C4826
:10F2E000016805E08A68B2FBF5F26A43CA60096802
:10F2F0008142F7D16078F021084202D09920F6F7D8
:10F30000D1FB6078401E6070C0B2002801D1F6F7D2
:10F3100030FCBDE83140F7F786BA0D490A6808E0CD
:10F320001369012B01DAD368136113691B1A136186
:10F3300012688A42F4D17047F452012080520120B1
:10F340000080FFFF086000208C700020E84E012044
:10F3500078600020CC86002058206973206F766585
:10F360007200000059206973206F766572000000FA
:10F370005A206973206F766572000000554353541C
:10F38000282564294E5300006368616E676520720A
:10F390006174653200000000675F707453682D3E31
:10F3A0006354696D6572203D202564006374696D46
:10F3B0006572203D2025640038B504000D00144816
:10F3C0000078401C1249087012480078002802D0CA
:10F3D000A120F6F767FBF7F7E5F9607E662802D013
:10F3E0008220F6F75FFBF6F7CAFB05E03821200024
:10F3F00007F0E6F9F6F7C3FBE06821698842F5D02B
:10F400002900200007F0FEF9F7F70DFA31BD00BF23
:10F41000CC860020925301204FF0FF31801E01283E
:10F4200014D9C01E042811D9801F05280ED9083808
:10F430000CD0801E042809D9401F05D0401E10287A
:10F4400004D9113804D004E0072102E0012100E0D2
:10F4500003210846704780B501460020C91E1AD016
:10F46000C91E18D0C91E16D0C91E012913D90D39BD
:10F47000032910D9091F07D0491E0CD0C91F032921
:10F4800009D9C91F07D002BD1D210FF21000F2F7E4
:10F49000B2FE012002BD012002BD000050443A200E
:10F4A0004C4C53202564000038B504464FF0FF351E
:10F4B000F9F732FA2C2C36D8DFE804F03435323440
:10F4C0003432343432323534193217173435353258
:10F4D00035343434193432343234341C1F23272B5E
:10F4E0002E323232323230323400B4251BE04FF447
:10F4F0007A7518E0D0F8DC5415E000F2DC40856A3B
:10F5000011E000F2DC40056D0DE000F2DC40856F9B
:10F5100009E0D0F87C5506E00A2504E0052502E064
:10F52000142500E03C25284632BD38B5DFF8844A72
:10F53000F3F7A6F9E06207F0CDF9F9F7EDF92063EA
:10F54000002512E0DFF8701A0161DFF8701A4161DE
:10F55000DFF86C2A8261DFF86C2AC261DFF8682A62
:10F5600002624162406A80476D1C2D2D80F2188135
:10F57000216B05EB8500C000002242544018427008
:10F580004FF0FF32426000220272C2604272032DCD
:10F5900004D17431DFF8342A8A62E3E7022D03D103
:10F5A000DFF82C2A4A67DDE7002DCBD0042D04D1EB
:10F5B0007431DFF8202A0A65D4E7052D04D17431AF
:10F5C000DFF8142A8A67CDE7062D04D1DFF80C2A6C
:10F5D000C1F81421C6E7072D05D101F58A71DFF8BE
:10F5E000002A8A62BEE7082D05D101F58A71DFF88D
:10F5F000F4290A65B6E7092D05D101F58A71DFF80E
:10F60000E8298A67AEE70A2D9CD00B2D9AD0012DF0
:10F6100098D00C2D04D1DFF8D429C1F80422A1E739
:10F620000D2D05D101F50171DFF8C4298A6299E732
:10F630000E2D05D101F50171DFF8B8290A6591E7B2
:10F640000F2D05D101F50171DFF8AC298A6789E733
:10F65000102D04D1DFF8A429C1F8A42282E7122DCD
:10F660003FF470AF142D3FF46DAF132D3FF46AAF2C
:10F67000162D3FF467AF2B2D3FF464AF152D04D149
:10F68000DFF87C29C1F86C236CE7172D05D101F553
:10F690005B71DFF870290A6564E7182D05D101F563
:10F6A0005B71DFF864298A675CE71A2D05D101F2E6
:10F6B0000C41DFF858298A6254E71E2D05D101F26A
:10F6C000AC41DFF84C298A624CE7192D04D1DFF8F0
:10F6D0004429C1F80C2445E71F2D05D101F2AC41A6
:10F6E000DFF834290A653DE7202D05D101F2AC4150
:10F6F000DFF828298A6735E7212D04D1DFF8202992
:10F70000C1F84C252EE7222D05D101F24C51DFF82E
:10F7100014298A6226E7232D05D101F24C51DFF826
:10F7200008290A651EE71B2D05D101F20C41DFF8FF
:10F73000FC280A6516E71C2D05D101F20C41DFF803
:10F74000382A8A670EE71D2D04D1DFF8302AC1F868
:10F75000AC2407E7262D04D1DFF8242AC1F81426AB
:10F7600000E7272D05D101F21461DFF8182A8A621B
:10F77000F8E6292D05D101F21461DFF80C2A8A6719
:10F78000F0E62A2D04D1DFF8042AC1F8B426E9E610
:10F790002C2D7FF4D7AEDFF8F829C1F80427E1E675
:10F7A000012032BD0CB42DE9FF4706460F46012467
:10F7B00035461A2D4AD02C2D48D005EB85004FEA4E
:10F7C000C008DFF8F0970B2F20D1D9F8300008EBF4
:10F7D000000A9AF80100002818D03046FFF71CFEF6
:10F7E000012813DB3046FFF717FE9AF8011081421B
:10F7F0000CDB304600F0B4F90446D9F83000404440
:10F80000002141700FF69410F2F7F5FCD9F83000A2
:10F8100018F80010002950D108EB00014A78002A9E
:10F820004BD1002208F80020104648700CA983B084
:10F8300068461822F4F790F90EBC304600F085F8BF
:10F84000022835D0032838D1032436E00B2F16D1F7
:10F85000FFF7E2FD012812DB3046FFF7DDFD05EB87
:10F860008501DFF85027126B02EBC1014978814214
:10F8700005DB0FF63010F2F7BEFC022060E01A2D17
:10F8800004D13846C0B202F0E9F805E02C2D03D1CE
:10F890003846C0B207F044F90CA983B06846182274
:10F8A000F4F75AF90EBC304600F04FF8022801D1A7
:10F8B000022045E0032800D103240A2F0DD1DFF8F0
:10F8C000F496D9F8300005EB85014FEAC10818F825
:10F8D0000010491C08F8001017E00B2F15D1DFF8B5
:10F8E000D496032D07D1D9F8300090F8790000287C
:10F8F00001D101F004FB05EB85004FEAC008D9F8FF
:10F90000300040444178491C4170DFF8A896D9F88E
:10F910003000D9F82C1005EB85024FEAC208D1E976
:10F920001C23CDE90223C96E009108EB00014B783E
:10F9300018F8002029460FF67800F2F75CFC204604
:10F9400004B0BDE8F0075DF80CFB0EB42DE9F04102
:10F9500083B00546012400EB8001CE00DFF8547629
:10F960001A280BD02C2809D0C0B2FFF79DFD396BA7
:10F970007118486000200872C86011E0386B315C73
:10F9800000290DD130184078002809D12846C0B28E
:10F99000FFF78AFD396B7118486000200872C86053
:10F9A00009A984B068461822F4F7D6F80FBCD7F836
:10F9B00030C066443669B047022801D1022011E008
:10F9C000032801D103240CE0D7F82C80D8E91C6768
:10F9D000204600212A4608F0ABF930433943C8E9F4
:10F9E0001C012046BDE8FE015DF810FB2DE9FF4734
:10F9F00004460D460126274607EB87004FEAC0085C
:10FA0000DFF8B095D9F830001A2F59D02C2F57D0E5
:10FA100008EB000A9AF80100022814DB2046FFF7E1
:10FA2000FBFC01280FDB2046FFF7F6FC9AF80110DB
:10FA3000814208DB2046FFF7EFFC8AF801000FF255
:10FA40008470F2F7D8FBD9F8300018F800100029BC
:10FA500004D108EB00025278002A69D02A460A2A0B
:10FA600009D1002903D0491E08F8001017E0002131
:10FA700008F8001013E00B2A11D108EB00014A78B6
:10FA8000002A02D0521E4A7001E000224A70032F61
:10FA900005D190F87900002801D101F03FFAD9F89A
:10FAA000300018F80010002942D140444078002866
:10FAB0003ED1204600F054F8032839D1032637E020
:10FAC00018F80010002904D108EB00025278002A2F
:10FAD0002ED02A460A2A09D1002903D0491E08F847
:10FAE000001012E0002108F800100EE00B2A0CD1E3
:10FAF00008EB000A9AF80100002803D0401E8AF89B
:10FB0000010002E000208AF801001A2F04D12846E3
:10FB1000C0B201F0A3FF05E02C2F03D12846C0B2EC
:10FB200006F0FEFF204600F01BF8032800D1032654
:10FB3000D9F83000D9F82C10D1E91C23CDE90223E3
:10FB4000C96E009108EB00014B7818F80020394687
:10FB50000FF27860F2F74FFB304604B0BDE8F08753
:10FB60002DE9F04107460126B84608EB8800C5009C
:10FB7000DFF84044206B281840698047032800D1F3
:10FB80000326B8F12C0F07D1206B295C00290AD17C
:10FB900028184078002806D1384640B200F080F995
:10FBA000032800D10326206B295C002917D12818CF
:10FBB0004178002913D14FF0FF31416000210172DB
:10FBC000C160D4F82C80D8E91C4501203A4608F0E1
:10FBD000AFF824EA000025EA0101C8E91C0130461B
:10FBE000BDE8F08138B5044604EB8400C000DFF8BE
:10FBF000C453296B002242544018114641702046DC
:10FC0000FFF7AEFFE86AD0E91C2321460FF2D0507F
:10FC1000F2F7F1FA012032BD2DE9F041B6B0044609
:10FC20000E46B6B201208DF86400DFF888531AA89A
:10FC3000E96A6C22F3F790FF17951AA984B0684619
:10FC40006C22F3F789FF0FBC00F0F2F900270BE0FC
:10FC5000032803D1189703208DF86400286B4044D3
:10FC6000002101727F1C7FB22D2F2ADAEA6AD2E9C5
:10FC70001C013A4600F0EAFA00F0010011F0000120
:10FC800001D10028EED007EB87004FEAC008286BAF
:10FC9000404441680029E5D4027A521C0272D2B273
:10FCA000724389B28A42DDDB806980470228CFD166
:10FCB000189702208DF86400DDE91801C4E90001FD
:10FCC00003E0DDE91801C4E9000136B0BDE8F081C8
:10FCD00000210A3842F20772904200D20121084600
:10FCE00070472DE9F04383B00446002001900422C0
:10FCF00004F1090101A8F3F75AFF6168DFF8B46263
:10FD0000376B282505FB01704068019A904204D1A9
:10FD10000FF2DC40F2F76FFA68E01046FFF7D8FF09
:10FD2000002809D16168019B05FB017042680FF250
:10FD3000CC40F2F760FA59E0DFF858743868D0F830
:10FD4000008025E090F908906068316B05FB001099
:10FD5000C06820FA09F0C00717D54FF0FF300090B7
:10FD60000346012201994846FFF720F940B20028D6
:10FD70000BD1616801980090306B05FB010043686E
:10FD80004A460FF28C40F2F736FA4046D0F800802F
:10FD9000B842D7D13868D0F800801FE090F90890B9
:10FDA000C86820FA09F0C00715D54FF0FF330122CB
:10FDB00049684846FFF76AF940B200280BD16168EC
:10FDC00001980090306B05FB010043684A460FF232
:10FDD0005840F2F710FA4046D0F800806168326B64
:10FDE00005FB0121B842D9D101984860BDE8F783ED
:10FDF0002DE9F8438146002425466E4F21E005EBAE
:10FE00008500C600386B06EB0008002088F8090062
:10FE1000FA6AD2E91C012A4600F018FA00F0010043
:10FE200011F0000101D100280AD04846D8F81C1072
:10FE30008847002804D0386B3018012141720C46E5
:10FE40006D1C2D2DDBDB2046BDE8F2835948C16ACD
:10FE5000D1E91C23002B01D1002A0DD0002107E09D
:10FE600002EB8203026B02EBC30200235372491CB4
:10FE700049B20A462D2AF3DB704700B502464D48C9
:10FE8000C36AD3E91C0100F0E1F900F0010011F0B0
:10FE9000000101D1002801D0012000BD084600BDAD
:10FEA0002DE9F0478146012409EB8900C500414E48
:10FEB000306B2818C068002829D0DFF8D87238685D
:10FEC000D0F8008003E003244046D0F80080B84218
:10FED0001DD090F908A0306B2818C168012202FAE1
:10FEE0000AF2114021FA0AF149B20129ECD14FF08E
:10FEF000FF33012241685046FFF7C8F80028E2D0DE
:10FF0000524649460FF23830F2F775F9DCE72046E1
:10FF1000BDE8F08710B58AB004460020ADF8220095
:10FF200001900A208DF8080000208DF809008DF856
:10FF30000A00ADF82200600719D50520FFF79DFFE4
:10FF4000002807D004208DF800000520019000A8AB
:10FF5000F8F7D2FD0220FFF790FF002807D0042019
:10FF60008DF800000220019000A8F8F7C5FDE0061A
:10FF70000CD50820FFF781FF002807D003208DF85B
:10FF800000000820019000A8F8F7B6FD0AB010BDE7
:10FF900002460020092A00D0704780B5012902D10D
:10FFA00007F088FF012002BD02492C22F3F7D4BDDF
:10FFB00000000000B84C0120718C00086D8C000816
:10FFC000798C00087D8C0008818C0008C508010828
:10FFD000893801086D0201084D3601085B310308BC
:10FFE0001543030885340108037E010881050108D3
:10FFF00009300308F9240308453A0308CB400308F5
:020000021000EC
:100000002D4403085D46030821390308F92501083A
:10001000632D03081D3D0308BF9F0108FF4103082E
:10002000BB370308735D01083F5F01088532010893
:100030000FB41B9800990160019941600299816099
:100040000399C1600499016105994161BDF85A1095
:100050000183BDF85C104183BDF85E1081830C996B
:100060000162139941621499816204B070470000E3
:100070004168122903D1C17A002001F002B8132986
:1000800003D1017B012000F0FCBF142903D1417B87
:10009000022000F0F6BF152902D1C07A01F002B8A3
:1000A000172961D1817A1B2908D01C2932D01D293A
:1000B00011D0262928D02C293CD07047C17B01299A
:1000C00003D1B0F80B0003F00BB902294CD1B0F802
:1000D0000D0003F003B9017D012903D1B0F80B0035
:1000E00008F0D8B9022903D1B0F80D0008F0C6B95C
:1000F000042903D1B0F8170008F0CEB9032933D191
:10010000B0F8150008F0D4B9C17B01292CD1807B4F
:1001100008F0F1BA817B012902D1C07A08F0F7BC5E
:10012000022902D1007B08F0FCBC05291CD1407BD0
:1001300008F0D7BC417D012902D1C07B07F0FABA93
:10014000022902D1C08A07F0E1BA032902D1008B4B
:1001500007F0E6BA042902D1408B07F009BB052954
:1001600002D1808B07F0F6BA70470B4908607047E0
:1001700009480068704700005D8901081B84010878
:100180003D860108430E030851450308DD0F0308AF
:100190004776010874690020F8520120414C20453F
:1001A00058000000414C2045582D415400000000EB
:1001B000414C256420256420256420256420256C7D
:1001C0006C750000524C204558000000524C2564CC
:1001D00020256420256420256420256C6C75000092
:1001E0005445524D20256420256C6C75000000009C
:1001F0004558204C4D435231202564004558204C31
:100200004D435232202564202564202564000000DF
:100210004558204C4D435233202564202564202529
:1002200064202564000000004558204C4D435234A2
:10023000202564202564202564202564000000001A
:10024000534D52412025642025640000D2B2203A4B
:1002500022BF21FA02F0002170472032D141D04064
:1002600048409140D14048407047000038B5F8F709
:1002700053FB0446104DF2F703FB286004F0C4FE64
:1002800004F0C7FE686004F0FFFF0C48C4F8B0003B
:1002900004F1B0000A4941600A4981600A49C1601D
:1002A0000A490161012032BD03494968896808474C
:1002B0000148406800680047A0520120718C000886
:1002C0006D8C0008798C00087D8C0008818C0008FA
:1002D0002DE9F04786B0044601A81421F5F7A0FBEC
:1002E000F1F707FF05464FF00208002601E0761CF3
:1002F00076B20A2E80F29E80022EF8D0032EF6D01F
:10030000062EF4D0524850F82670787A002806D18C
:1003100007F10C00406D406880470028E7D008F8DE
:10032000046008F101084FFA88F8304609284FD8D0
:10033000DFE800F0050A4E4E10204E154E49C82148
:100340002846F2F7C3F843E04FF448712846F2F725
:10035000BDF83DE032212846F2F7B8F838E0072032
:100360008DF80400FF208DF8050032212846F2F7B1
:10037000ADF82DE03C212846F2F7A8F84FF0000A2E
:1003800007F10C09BAF1030F22DA0020D9F8541052
:100390000969884714212846F2F798F80120D9F80E
:1003A00054100969884714212846F2F78FF8BAF1EA
:1003B000020F05DA062101A8D9F8542052699047A6
:1003C0000AF1010ADEE74FF416712846F2F77EF8CB
:1003D00007F10C0999F8151001A8D9F854205269B1
:1003E0009047002819D0D9F80C00F96800EB010AF1
:1003F00099F8152001A95046F3F7D9FB3846FEF7C6
:100400000DFC99F81520514608EB0400F3F7CFFBDB
:1004100099F9150080444FFA88F8787A00287FF41B
:1004200066AFD9F854008068804700287FF45FAF3A
:10043000002009E0A8F10200ADF80000022200A9A6
:100440002046F3F7B4FB002006B0BDE8F0870000BB
:100450000860002038B505000C0094F84C006428B2
:1004600002D08020F5F71EFBF6F774F9F5F787FB4D
:10047000606928436061207C10F0F800082806D1EC
:10048000A0696169084202D02000F6F708FA07481F
:100490004078F021084202D09920F5F703FB034889
:1004A0004078002801D1F5F764FB31BDCC860020EF
:1004B0000FB480B5BDF80B0064494880022802DB08
:1004C000801E088001E0002008800C229DF90A109F
:1004D0000020F8F723FA032801D1022000E00120D0
:1004E00002BC5DF814FB59480121418000210180C4
:1004F00001207047564908707047000030B58DB034
:1005000002A8F8F76AFA514C2088401C20806188C4
:1005100080B2884231D300202080054627E0606801
:10052000D0F8EC01E840C00720D5284606F024FAB0
:1005300000281BD400EB80009FED430ADDED0B0A81
:1005400060EE800AFDEEE00A10EE901A00AA8152D9
:10055000DDED0C0A20EE800ABDEEC00A10EE101A86
:100560008218518000A94018012101716D1C172DBE
:10057000D5DBDDE9000106F008FA01200DB030BD41
:1005800080B5F8F7C9F9314948603249C0F8F0112F
:1005900000F5F87030494160304981600FF20D017B
:1005A000C1600FF225010161012002BD10B50024D8
:1005B000274890F90000002804D106F006FA002828
:1005C00000D00124204610BDF8B504460D4640F287
:1005D0004916287816FB004001210170287816FB87
:1005E00000404170287816FB00400C21817028786B
:1005F00016FB0040164991F90010002902D0022193
:10060000C17001E00121C170287816FB0040012172
:100610000171287816FB0040C180287816FB00473E
:10062000002006F073F93881287816FB004400207A
:1006300006F071F960812878401C28700C20BDE814
:10064000F24006F081B900000000C842F0870020A7
:1006500073530120B1040108E7040108FD040108F7
:100660000FB410B5032200210846F8F757F9022805
:1006700001D102201CE00FF24000F1F7BCFDDFF8D1
:10068000484C00206073608260629DF80C209DF8E9
:100690000B109DF80A0008F0CDFF58220021DFF86A
:1006A000BC0CF2F765FE00202074A073A06301204B
:1006B00010BC5DF814FB000050443A205374617282
:1006C000745065646F2D303632362D3100000000D5
:1006D00080B5032200210120F8F720F9032801D179
:1006E000032002BD012002BD30B58BB000A8F8F791
:1006F00074F905210320F8F7EEF9002802D1DFF89C
:10070000600C0890DFF8C04BE069C56F08F028FF67
:10071000207294F90800022806D13C2D04D114213E
:100720000320F8F75CF907E0012805D1142D03D167
:100730003C210320F8F753F9284680B2DDED081A72
:1007400000A991EC030A08F0D8FD206A281820625D
:1007500001200BB030BD10B5DFF86C4B94F90000F0
:1007600000283AD494F90A0094F90110814228D162
:10077000217B0818A07240B23D2801DB3C38A072F2
:1007800094F90A100FF26C00F1F735FD0020206299
:10079000DFF8D00B90F9010010F1010F01D1012019
:1007A00010BD94F90110081AF8F7E4FA21F000419D
:1007B00004F0FEFB40B2012801DB012010BD002047
:1007C00010BDDFF8A40B90F90120914203D0D4E9C9
:1007D0000023C0E90023002010BD206ADFF88C1B35
:1007E000884205DB0FF21800F1F705FD012010BD6E
:1007F000002010BD50443A204E54202564000000D3
:1008000050443A204E6F54696D6500002DE9F8435D
:100810000026DFF8B44A07E07A19A27252B23146D4
:100820000FF26C00F1F7E7FC94F90A50002E21D486
:100830006078461B76B294F90C70002EECD53046E9
:10084000F8F798FA21F0004102460B469046994687
:100850003846F8F78FFA42464B4605F027FCE3D2BC
:10086000EA1BA272002652B231460FF23800F1F7AD
:10087000C2FCD9E73C2D02DBA5F13C00A07294F943
:100880000A100FF23400BDE8F443F1F7B4BC0000E5
:1008900050443A20636F6D70312025642C2025640C
:1008A0000000000050443A20636F6D7032202564D0
:1008B0002C2025640000000050443A204355542069
:1008C0002564000010B5DFF8004A0020A073012065
:1008D0002072002060724FF0FF3020700F20E07215
:1008E0001420207300206073608260626074206353
:1008F000606328220146DFF87C0AF2F739FDF8F739
:100900000BF8E061F1F7F5FBA061E069DFF8681A28
:10091000C0F888108830DFF8641A4160DFF8601A88
:1009200081600FF28D21C1600FF659210161012014
:1009300010BD10B582B04FF46163C1EB0114A40087
:1009400013FB0043D3184FF47A746343DFF8244A4F
:100950002360DFF874391B7C009313460A46014676
:100960000FF20800F1F747FC13BD0000504420428D
:10097000542025642025642025642025640000007F
:100980002DE9F0412DED028BAAB0DFF8D069314698
:1009900084B068465822F3F7DFF80FBC00F096FCED
:1009A00010EE100AF8F7D0FA41EC100B9FED7E8B99
:1009B000DFF8C049656853EC102B51EC180BF8F7C1
:1009C000F1F904F0F5FA15FA80F060604FF6FF7562
:1009D000A84200D36560314684B068465822F3F7D8
:1009E000BBF80FBC00F028FC10EE100AF8F7ACFAC8
:1009F00041EC100BA76853EC102B51EC180BF8F7D7
:100A0000D1F904F0D5FA17FA80F0A060A84200D31B
:100A1000A5600020139002201290314684B06846F1
:100A20005822F3F799F80FBC00F09AFAA189401800
:100A3000A08180B2FF2801DBFF20A081002013905D
:100A400003201290314684B068465822F3F784F8A8
:100A50000FBC00F085FA216940182061A84200D33C
:100A600025610020139006201290314684B068461C
:100A70005822F3F771F80FBC00F072FAA18A4018FF
:100A8000A08280B2FF2801DBFF20A082002013900B
:100A900007201290314684B068465822F3F75CF87C
:100AA0000FBC00F05DFAE18A4018E08280B2FF28B6
:100AB00001DBFF20E08200201390082012903146D5
:100AC00084B068465822F3F747F80FBC00F048FAA4
:100AD000A1694018A061A84200D3A561002013902D
:100AE00009201290314684B068465822F3F734F852
:100AF0000FBC00F035FAE1694018E061A84200D36C
:100B0000E56114A808F030FDDFF8707DD7F830807B
:100B10002398F8F719FA0022DFF8443DF8F742F974
:100B200004F046FA58FA80F03863796B491C79630F
:100B3000B0FBF1F084F82000002013900120129007
:100B4000314684B068465822F3F706F80FBC00F02F
:100B500007FA616A40186062A84200D36562F87BB8
:100B600000F0E9FA2AB0BDEC028BBDE8F081DFF8B5
:100B700004088189002914D10169002911D1818AD1
:100B800000290ED1C18A00290BD18169002908D121
:100B9000C169002905D1406A401E8041C043C00F91
:100BA000704701207047000000000000000059401D
:100BB0002DE9F04FABB0814600254E46DFF8BC4C26
:100BC000A07B494688420BD0012E40F09F80E0690F
:100BD00090F9782090F979100FF6D840F1F70BFBD7
:100BE00014A808F0C1FCDFF874A728461390012070
:100BF0001290514684B068465822F2F7ADFF0FBC00
:100C000000F0AEF907469DED230ADAED0F0A30EE4B
:100C1000600A10EE100AF8F797F92A46DFF8403C10
:100C2000F8F7C0F804F0C4F980461FFA88F8BDF858
:100C30009A00BAF84A10A0EB010B5FFA8BFBE0694F
:100C400090F8D914002903D190F8D814002905D0C0
:100C5000E16A149A5118A26B891AE16200F5AF613A
:100C60004978002903D190F87825002A05D0A26A96
:100C7000149B9A18A36BD21AA262A269927A002AD4
:100C80001AD1A26A002A08D0002903D190F8780569
:100C9000002802D0012005F072F9E06A00280BD08C
:100CA000E06990F8D914002903D190F8D8040028FD
:100CB00002D0012009F0A3F9B9F1000F34D1002FBF
:100CC00002D15BEA080000D00125002020624FF02D
:100CD000FF302070DFF89026D4E90001C2E900015E
:100CE000DFF8B02BC2E90001DFF87826C2E9000185
:100CF000E07AA072A07B00284ED00020A073207C58
:100D0000002849D001206074054645E0B9F1000F84
:100D100004D10FF6B430F1F76EFA61E70FF6B43094
:100D2000F1F769FA2846E7E000F0A7F900281BD0A0
:100D300000A8F1F7FDFC204600A90522F2F7FCFE11
:100D400028466072DFF82026D4E90001C2E90001DC
:100D500094F9023094F9012094F900100FF69030C4
:100D6000F1F749FAFFF752FD00A8F1F7E1FC204640
:100D700000A90522F2F7E0FEFFF7EDFC00280BD0FA
:100D8000DFF8E025D4E90001C2E90001207C002859
:100D900001D0012060740125012E07D1A07B4946B6
:100DA000884203D000F036FA84F80E90012E58D114
:100DB000002F56D0DFF8DC9AE07B217C08430CD171
:100DC000012020740522214609F10800F2F7EFFE08
:100DD000A27861782078FFF7ACFD94F9010099F9C9
:100DE0000910401A411E222901D2012005E010F10C
:100DF000230F01DA012000E0002001282AD1002081
:100E000020636063FFF7B3FE002823D0282200216F
:100E1000DFF86005F2F7ACFAE07B401CE073C0B28B
:100E2000152809D10FF6E020F1F7E5F901206074EB
:100E30000020E07301250DE0207C401C2074A27886
:100E400061782078FFF775FD0522214609F1080039
:100E5000F2F7ADFEFFF794FD582214A95046F2F7C1
:100E6000A6FE607B012833D1608A002805D10FF6E9
:100E7000A820F1F7C0F9012523E0616A814218D268
:100E8000002F02D15BEA080000D00125DFF8049AA8
:100E900099F9020094F90220904212D0491C616233
:100EA0000FF68820F1F7A7F9D4E90001C9E900019C
:100EB00007E000206073608260620FF68020F1F727
:100EC0009AF9012E04D1207C002801D00120607401
:100ED0002846012801D100212162E16991F87910A9
:100EE000002906D100212162012801D100F092F9E8
:100EF00000251498A06328462BB0BDE8F08F10B5EC
:100F0000DFF8780900210162032205210020F7F7AC
:100F100005FD044600F007F8204610BD0322052118
:100F20000120F7F7FBBC00B597B000A808F01CFB48
:100F3000582200A9DFF84809F2F739FE012017B05E
:100F400000BDDFF83809806A7047DFF830090021FA
:100F500081627047DFF824090021C16270470000F8
:100F60000FB410B596B000249DF9BC0001280BD138
:100F700008F0F3FB1899884202D3441AE4B272E0F5
:100F80008038441AE4B26EE000A808F0EDFA9DF94A
:100F9000B800401E082866D8DFE800F02905111DBA
:100FA0002936424E5A0001981999884201D3441AB1
:100FB00059E0DFF8E4281018401A441C53E0029866
:100FC0001A99884201D3441A4DE0DFF8CC28101852
:100FD000401A441C47E003981B99884201D3441AE5
:100FE00041E0DFF8B4281018401A441C3BE0009898
:100FF0001899884201D3441A35E0DFF89C18081884
:101000001899401A441C2EE004981C99884201D378
:10101000441A28E0DFF880281018401A441C22E007
:1010200005981D99884201D3441A1CE0DFF868280E
:101030001018401A441C16E006981E99884201D3E5
:10104000441A10E0DFF850281018401A441C0AE037
:1010500007981F99884201D3441A04E0DFF8382822
:101060001018401A441C204616B010BC5DF814FB42
:10107000DFF80808012141727047DFF80008407A64
:10108000704708F083BA0146DFF8F027792902DBC0
:101090007820508200E05082012050730FF6B0009B
:1010A000F1F7A9B810B5040001D1012402E0072C22
:1010B00000DB062421460FF6AC00F1F79CF8641E15
:1010C000052C2DD8DFE804F0030A11181F26DFF8DD
:1010D000AC073721C1723C21017321E0DFF89C0786
:1010E0001921C1721E2101731AE0DFF890070F2148
:1010F000C1721421017313E0DFF880070A21C17265
:101100000F2101730CE0DFF874070721C1720C2175
:10111000017305E0DFF864070521C1720A2101733C
:10112000DFF85807C17A8172BDE81040FFF76EBB47
:10113000DFF83007704700EB80018800421CDFF8C1
:1011400024078C4992B20B681B0E1354521C92B2A6
:101150000B681B0C1354521C92B20B681B0A1354DD
:10116000521C92B20B681354521C92B24B681B0A69
:101170001354521C92B24B681354521C92B28B6897
:101180001B0A1354521C92B28B681354521C92B215
:101190008B891354521C92B20B691B0A1354521CB4
:1011A00092B20B691354521C92B28B8A1354521C84
:1011B00092B2CB8A1354521C92B28B691B0A1354FD
:1011C000521C92B28B691354521C92B2CB691B0A07
:1011D0001354521C92B2CB691354521C92B291F820
:1011E00020301354521C92B24B6A1B0A1354521CE7
:1011F00092B2496A1154DFF88406511C818270470B
:1012000010B5DFF87846A18A0FF26470F0F7F3FFAB
:10121000A08A10BD80B5282200215648F2F7A8F810
:10122000DFF858060021C173012181820021017479
:101230000163416301BD00000FB400B597B000A881
:1012400008F092F99DED090ADDED210AB4EE600A7D
:10125000F1EE10FA02DB30EE600A05E09FED441A71
:1012600071EE600A30EE800A10EE100AF7F76CFE9D
:10127000DFF8F425DFF8F43508F002FFF7F78CFE0D
:10128000F7F762FE0022DFF8E835F7F78BFD03F091
:101290008FFE00EE100AB8EEC00A10EE100AF7F743
:1012A00053FEDFF8C425DFF8CC35F7F77BFDDFF818
:1012B000C825DFF8E83508F0E3FEF7F76DFE00EE2D
:1012C000100A17B05DF814FB704B01200FB400B585
:1012D00097B000A808F048F99DED0E0ADDED260A4A
:1012E000B4EE600AF1EE10FA02DB30EE600A05E0BF
:1012F0009FED1F1A71EE600A30EE800A10EE100AA0
:10130000F7F722FEDFF86025DFF8603508F0B8FE59
:10131000F7F742FEF7F718FE0022DFF85435F7F72B
:1013200041FD03F045FE00EE100AB8EEC00A10EED3
:10133000100AF7F709FEDFF83025DFF83835F7F740
:1013400031FDDFF83425DFF8543508F099FEF7F762
:1013500023FE00EE100A17B05DF814FB14480120BC
:1013600000007A44B0520120A852012040771B00AF
:10137000002474499C4D012061060108D106010832
:10138000E90601082DE9F0472DED068BAAB00646C7
:101390000D4614A808F0E8F840F24914287814FB28
:1013A000006001210170287814FB0060DFF8CC7424
:1013B000797B01290ED103224270287814FB00604A
:1013C0000122C270012907D1788A002804D10020A7
:1013D000787301E001214170287814FB006003213B
:1013E0008170787C012820D1387C00281DD0297894
:1013F00014FB0161C0220A71DFF8681408702878B4
:1014000014FB0068FFF7FCFEA8F83000287814FBF6
:101410000064FFF78DFEC4F832002878401C287065
:10142000FFF7F8FE0020787415E20DF18C099FEDAE
:10143000868B9FED879BDFF8487400201390012076
:101440001290394684B068465822F2F785FB0FBCEB
:10145000FFF786FD0A28287814FB006080F0FC80E6
:1014600000210171287814FB006898F804A0084650
:10147000139002201290394684B068465822F2F741
:101480006BFB0FBCFFF76CFD40EA0A0088F8040014
:10149000287814FB0068002013900320129039462E
:1014A00084B068465822F2F757FB0FBCFFF758FD8F
:1014B00088F80500287814FB0068002013900420A9
:1014C0001290394684B068465822F2F745FB0FBCAB
:1014D000FFF746FD88F80600287814FB0068002016
:1014E000139005201290394684B068465822F2F7CE
:1014F00033FB0FBCFFF734FD88F80700394684B092
:1015000068465822F2F728FB0FBCFFF7DFFE10EE0B
:10151000100AF7F719FD41EC100B287814FB00684E
:1015200053EC102B51EC190BF7F73CFC03F040FD8A
:10153000A8F80E00287814FB00682398F7F704FD3C
:1015400053EC182BF7F72EFC03F032FD88F810004F
:10155000287814FB0060B9F80E104174394684B045
:1015600068465822F2F7F8FA0FBCFFF765FE10EE56
:10157000100AF7F7E9FC41EC1A0B287814FB006815
:1015800053EC1A2B51EC190BF7F70CFC03F010FD80
:1015900088F81200287814FB0068D9F80800F7F7DB
:1015A000D3FC53EC182BF7F7FDFB03F001FD88F893
:1015B0001300287814FB0068002013900620129076
:1015C000394684B068465822F2F7C6FA0FBCFFF7D6
:1015D000C7FC88F80800287814FB006800201390E6
:1015E00007201290394684B068465822F2F7B4FAC0
:1015F0000FBCFFF7B5FC88F80900287814FB0068D9
:101600000020139008201290394684B06846582272
:10161000F2F7A2FA0FBCFFF7A3FC88F80A002878BB
:1016200014FB00640020139009201290394684B006
:1016300068465822F2F790FA0FBCFFF791FCE0726F
:101640002878401C287004E10000000000002440BD
:10165000000000000000594080210171287814FB2F
:1016600000680020139002201290394684B068462A
:101670005822F2F771FA0FBCFFF772FCC8F80500A8
:10168000287814FB0068002013900320129039463C
:1016900084B068465822F2F75FFA0FBCFFF760FC8F
:1016A000C8F80900287814FB006800201390042073
:1016B0001290394684B068465822F2F74DFA0FBCB2
:1016C000FFF74EFCC8F80D00287814FB00680020D6
:1016D000139005201290394684B068465822F2F7DC
:1016E0003BFA0FBCFFF73CFCC8F81100394684B048
:1016F00068465822F2F730FA0FBCFFF7E7FD10EE0C
:10170000100AF7F721FC41EC100B287814FB006855
:1017100053EC102B51EC190BF7F744FB03F05EFC74
:10172000C8F82700287814FB00682398F7F70CFC0A
:1017300053EC182BF7F736FB03F03AFC88F82B0034
:10174000287814FB0060B9F80E1080F82C10394688
:1017500084B068465822F2F7FFF90FBCFFF76CFD22
:1017600010EE100AF7F7F0FB41EC1A0B454A464B16
:1017700004F0B4FC06D8454A454B04F097FC01D26E
:101780009FED47AB287814FB006853EC1A2B51EC03
:10179000180BF7F707FB03F00BFCA8F82D002878CF
:1017A00014FB0068D9F80800F7F7CEFB53EC182BB0
:1017B000F7F7F8FA03F0FCFB88F82F00287814FB01
:1017C00000680020139006201290394684B06846C5
:1017D0005822F2F7C1F90FBCFFF7C2FBC8F8150099
:1017E000287814FB006800201390072012903946D7
:1017F00084B068465822F2F7AFF90FBCFFF7B0FB90
:10180000C8F81900287814FB0068002013900820FD
:101810001290394684B068465822F2F79DF90FBC01
:10182000FFF79EFBC8F81D00287814FB0064002019
:10183000139009201290394684B068465822F2F776
:101840008BF90FBCFFF78CFBC4F821002878401CF3
:101850002870FFF768FB2AB0BDEC068BBDE8F08767
:1018600000002440582601207B14AE47E17A743FE3
:1018700000005940E17A843F2D431CEB704B01205E
:1018800014480120B81E85EB51B89E3F9A9999994A
:101890009999B93FD850012080969800E2361A3FB6
:1018A0009A9999999999B93F80B5C046C046012047
:1018B00002BD000050442052656620452825642959
:1018C0002C492825642900005044203A206C636488
:1018D0006F6E00005044203A206249734150536CAF
:1018E000656570696E672077726F6E67202564008A
:1018F00050443A54696D654E6F7469202564202503
:1019000064202564000000005044204254204246D8
:101910002046554C4C00000050443A20526571203E
:101920005065646F496E666F3100000050443A2084
:101930007574696D657220256400000050443A207A
:10194000526571205065646F496E666F3200000009
:1019500050443A20537461727420446174612025AC
:101960006400000050443A205554202564000000D3
:1019700050443A204241544C454E47544820256437
:101980000000000010B5DFF8AC4C4FF428720021C5
:101990002046F1F7EDFCFF202070E07284F862022F
:1019A000DFF8D00C0021417010BDF8B501240B28E0
:1019B00025D10B46012B0ED1DFF8783CD31893F9D3
:1019C00054522E46DFF8B07CD75DBE4210DA6D1C53
:1019D00083F8545231E0022B2FD1DFF8583CD31852
:1019E00093F95452012D03DB6D1E83F8545224E009
:1019F000DFF8403CD318002483F854421DE00A2845
:101A00001BD10B46012B08D1DFF8283CD31803F576
:101A100015735D796D1C5D710FE0022B0DD1DFF840
:101A2000143CD31803F5157393F90550012D02DB0F
:101A30006D1E5D7101E000245C71002C05D1134620
:101A400002460FF20C00F0F7D6FB2046F2BD000074
:101A500041542D25643A256420256400DFF8D41B09
:101A600081F85E0270470FB42DE9F04395B0012470
:101A7000DFF8005CE868DFF8BC6B90F81014002910
:101A800057D190F81104002853D10FF23820F0F705
:101A9000B2FBB4208DF8020046208DF803002046EA
:101AA0008DF8040000208DF82C0003200C900DF11F
:101AB000350000A91822F2F73FF80A208DF834000B
:101AC0000BA8F7F719F8002801D10220F4E000A8CC
:101AD000F0F72EFE9DF80000B0779DF90100F07739
:101AE0009DF9021086F82010BDF90320A6F82120E8
:101AF0009DF900304FF46167C0EB001C4FEA8C0089
:101B000017FB030040FA81F04FF47A7101FB0020CB
:101B1000C6F80200C6F80D000020A861E870287021
:101B2000A870687028712422014606F52870F1F724
:101B30001FFC9DF87270B846A146B8F1010F1DD187
:101B4000DDF87300202805D0D6F817100843C6F832
:101B500017000BE0204607E0D6F8171009FA00F24C
:101B60001143C6F81710401C0528F5DBF07E9DF9DF
:101B7000771009FA01F10843F07651E008EB06000E
:101B800090F9541200294BD190F95902002847D1FD
:101B9000B8F1020F2DD100A8F0F7CAFD9DF90000A1
:101BA0004FF461619DF90120C2EB02139A0011FB11
:101BB00000209DF9021040FA81F04FF47A71BDF9CE
:101BC000032001FB0020C6F89302C6F88F0206F13D
:101BD0002B0006F11E010522F1F7AEFF4FF49660CF
:101BE000B083DFF8D00CC6F8870200206861286156
:101BF00016E0B8F1030F13D1DDF87300C6F8230027
:101C0000BDF878004FF47A714843C6F827000020E9
